:020000040800F2
:1000000000060020E1010008E3010008E301000808
:10001000E3010008E3010008E3010008E301000830
:10002000E3010008E3010008E3010008652F000870
:10003000E3010008E3010008E3010008E301000810
:10004000E3010008E3010008E3010008E301000800
:10005000E3010008E30100080D3200083532000812
:100060005D32000885320008AD320008E301000867
:10007000E3010008E3010008E3010008E3010008D0
:10008000E3010008E3010008E3010008E3010008C0
:10009000E3010008E3010008E3010008D53200088D
:1000A000E3010008E3010008E3010008E3010008A0
:1000B000A9330008E3010008E3010008E301000898
:1000C000E3010008E3010008E3010008E301000880
:1000D000E3010008E3010008E3010008E301000870
:1000E00039330008E3010008E3010008E3010008D8
:1000F000E3010008E3010008E3010008E301000850
:10010000E3010008E3010008E3010008E30100083F
:10011000E3010008E3010008E3010008E30100082F
:10012000E3010008E3010008E3010008E30100081F
:10013000E3010008E3010008E3010008E30100080F
:10014000E3010008E3010008E301000819270008A3
:10015000E3010008E3010008E3010008E3010008EF
:10016000E3010008E3010008E3010008E3010008DF
:10017000E3010008E3010008E3010008E3010008CF
:10018000E3010008E3010008E3010008E3010008BF
:10019000E3010008E3010008E3010008E3010008AF
:1001A000E3010008E3010008E3010008E30100089F
:1001B000E3010008E3010008E3010008E30100088F
:1001C000E3010008E3010008E3010008E30100087F
:1001D000E3010008E3010008E3010008E30100086F
:1001E00002E000F000F8FEE772B6374880F30888B6
:1001F000364880F3098836483649086040F20000E6
:10020000CCF200004EF63471CEF200010860BFF36C
:100210004F8FBFF36F8F40F20000C0F2F0004EF638
:100220008851CEF200010860BFF34F8FBFF36F8F8C
:100230004FF00000E1EE100A4EF63C71CEF20001E4
:100240000860062080F31488BFF36F8F01F02CFF45
:1002500002F026FE4FF055301F491B4A91423CBF29
:1002600041F8040BFAE71D49184A91423CBF41F896
:10027000040BFAE71A491B4A1B4B9A423EBF51F83E
:10028000040B42F8040BF8E700201849184A914281
:100290003CBF41F8040BFAE701F00AFF02F054FEFC
:1002A000144C154DAC4203DA54F8041B8847F9E7A7
:1002B00000F042F8114C124DAC4203DA54F8041B22
:1002C0008847F9E701F0F2BE000600200022002076
:1002D0000000000808ED00E00000002000060020FB
:1002E0006837000800220020402200204022002021
:1002F000602E0020E0010008E0010008E001000895
:10030000E00100082DE9F04F2DED108AC1F80CD066
:10031000C3689D46BDEC108ABDE8F08F002383F3CF
:1003200011882846A047002001F072FAFEE701F08C
:1003300001FA00DFFEE7000038B500F0BBFB01F07A
:1003400083FE054601F0A6FE0446C8B90E4B9D4249
:1003500018D001339D4218BF044641F2883504BFCE
:1003600001240025002001F079FE0CB100F074F8A2
:1003700000F000FD284600F0BFF800F06DF8F9E746
:100380000025EFE70546EDE7010007B008B500F0EE
:1003900063FBA0F120035842584108BD07B541F264
:1003A0001203022101A8ADF8043000F073FB03B082
:1003B0005DF804FB38B5302383F3118817480368D0
:1003C0000BB101F0F1FA164A144800234FF47A7188
:1003D00001F0E0FA002383F31188124C236813B173
:1003E0002368013B2360636813B16368013B63606A
:1003F0000D4D2B7833B963687BB9022000F024FCE3
:10040000322363602B78032B07D163682BB902205A
:1004100000F01AFC4FF47A73636038BD402200206C
:10042000B50300086023002058220020084B1870F4
:1004300003280CD8DFE800F008050208022000F0CD
:10044000F9BB022000F0ECBB024B00225A6070475F
:100450005822002060230020234B244A10B51C465C
:10046000196801313FD004339342F9D16268A24246
:1004700039D31F4B9B6803F1006303F540439A4255
:1004800031D2002000F030FB0220FFF7CFFF194BE4
:100490001A6C00221A64196E1A66196E596C5A6425
:1004A000596E5A665A6E5A6942F080025A615A6908
:1004B00022F080025A615A691A6942F000521A61A8
:1004C0001A6922F000521A611B6972B64FF0E023DC
:1004D0003021C3F8084DD4E9003281F311889D46DC
:1004E00083F30888104710BD00C0000820C0000832
:1004F00000220020003802402DE9F04F93B0AA4BB3
:1005000000902022FF210AA89D6800F0DDFBA74A89
:100510001378A3B9A648012103601170302383F337
:10052000118803680BB101F03FFAA24AA0480023EA
:100530004FF47A7101F02EFA002383F31188009BA7
:1005400013B19D4B009A1A609C4A009C1378032BB0
:100550001EBF00231370984A4FF0000A18BF536063
:10056000D3465646D146012000F064FB24B1924B9D
:100570001B68002B00F01182002000F06DFA039040
:10058000039B002BF2DB012000F04AFB039B213B85
:10059000162BE8D801A252F823F000BFF905000895
:1005A00021060008B5060008670500086705000871
:1005B000670500083F0700080F0900082908000820
:1005C0008B080008B3080008D90800086705000870
:1005D000EB080008670500085D0900089906000897
:1005E00067050008A109000805060008990600082B
:1005F000670500088B0800080220FFF7C7FE0028E7
:1006000040F0F581009B0221BAF1000F08BF1C46A3
:1006100005A841F21233ADF8143000F03BFAA2E71E
:100620004FF47A7000F018FA071EEBDB0220FFF798
:10063000ADFE0028E6D0013F052F00F2DA81DFE8A9
:1006400007F0030A0D10133605230593042105A8AE
:1006500000F020FA17E054480421F9E75848042133
:10066000F6E758480421F3E74FF01C08404600F035
:100670003DFA08F104080590042105A800F00AFAE3
:10068000B8F12C0FF2D1012000FA07F747EA0B0B63
:100690005FFA8BFB4FF0000900F062FB26B10BF014
:1006A0000B030B2B08BF0024FFF778FE5BE74648DF
:1006B0000421CDE7002EA5D00BF00B030B2BA1D10D
:1006C0000220FFF763FE074600289BD0012000F0C0
:1006D0000BFA0220FFF7AAFE00261FFA86F8404612
:1006E00000F012FA044690B10021404600F01CFAD6
:1006F00001360028F1D1BA46044641F21213022114
:1007000005A8ADF814303E4600F0C4F92BE70120EF
:10071000FFF78CFE2546244B9B68AB4207D9284641
:1007200000F0E4F9013040F067810435F3E7234B32
:1007300000251D70204BBA465D603E46ACE7002E9A
:100740003FF460AF0BF00B030B2B7FF45BAF022089
:10075000FFF76CFE322000F07FF9B0F10008FFF6E1
:1007600051AF18F003077FF44DAF0F4A926808EBC2
:10077000050393423FF646AFB8F5807F3FF742AF9F
:10078000124B0193B84523DD4FF47A7000F064F901
:100790000390039A002AFFF635AF019B039A03F8F2
:1007A000012B0137EDE700BF002200205C23002071
:1007B00040220020B50300086023002058220020BA
:1007C00004220020082200200C2200205C220020AD
:1007D000C820FFF7DBFD074600283FF413AF1F2DAD
:1007E00011D8C5F1200242450AAB25F0030028BF0D
:1007F000424683490192184400F040FA019A804829
:10080000FF2100F061FA4FEAA8037D490193C8F384
:100810008702284600F060FA064600283FF46DAFD4
:10082000019B05EB830537E70220FFF7AFFD0028AA
:100830003FF4E8AE00F0A4F900283FF4E3AE00274F
:10084000B846704B9B68BB4218D91F2F11D80A9B22
:1008500001330ED027F0030312AA134453F8203CAF
:1008600005934046042205A900F0AEFA04378046FD
:10087000E7E7384600F03AF90590F2E7CDF8148042
:10088000042105A800F006F906E70023642104A866
:10089000049300F0F5F800287FF4B4AE0220FFF7CF
:1008A00075FD00283FF4AEAE049800F051F90590B4
:1008B000E6E70023642104A8049300F0E1F800288F
:1008C0007FF4A0AE0220FFF761FD00283FF49AAE4E
:1008D000049800F04DF9EAE70220FFF757FD0028E1
:1008E0003FF490AE00F05CF9E1E70220FFF74EFD27
:1008F00000283FF487AE05A9142000F057F9042121
:100900000746049004A800F0C5F83946B9E732203C
:1009100000F0A2F8071EFFF675AEBB077FF472AEBB
:10092000384A926807EB090393423FF66BAE022008
:10093000FFF72CFD00283FF465AE27F003074F4476
:10094000B9453FF4A9AE484600F0D0F8042105901F
:1009500005A800F09FF809F10409F1E74FF47A7057
:10096000FFF714FD00283FF44DAE00F009F9002810
:1009700044D00A9B01330BD008220AA9002000F0C2
:10098000ABF900283AD02022FF210AA800F09CF9F8
:10099000FFF704FD1C4800F041FF13B0BDE8F08FE5
:1009A000002E3FF42FAE0BF00B030B2B7FF42AAE7F
:1009B0000023642105A8059300F062F8074600288B
:1009C0007FF420AE0220FFF7E1FC804600283FF4D0
:1009D00019AEFFF7E3FC41F2883000F01FFF0598E5
:1009E00000F0F0F9464600F0BBF93C46BBE5064690
:1009F00052E64FF0000905E6BA467EE637467CE649
:100A00005C22002000220020A086010070B50F4B60
:100A10001B780133DBB2012B0C4611D80C4D296831
:100A20004FF47A730E6AA2FB03320146224628462F
:100A3000B047844204D1074B00221A70012070BDD8
:100A40004FF4FA7000F0EAFE0020F8E710220020D0
:100A5000082600209423002007B500230246012128
:100A60000DF107008DF80730FFF7D0FF20B19DF89A
:100A7000070003B05DF804FB4FF0FF30F9E700001A
:100A80000A4608B50421FFF7C1FF80F00100C0B29B
:100A9000404208BD30B4054C2368DD69044B0A466A
:100AA000AC460146204630BC604700BF0826002007
:100AB000A086010070B501F0CDF9094E094D3080D6
:100AC000002428683388834208D901F0BDF92B68D7
:100AD00004440133B4F5404F2B60F2D370BD00BF26
:100AE000962300206823002001F062BA00F1006024
:100AF00000F540400068704700F10060920000F58A
:100B0000404001F0EDB90000054B1A68054B1B8809
:100B10009B1A834202D9104401F096B90020704715
:100B2000682300209623002038B5084D044629B1DB
:100B300028682044BDE8384001F0A6B92868204460
:100B400001F08AF90028F3D038BD00BF68230020E7
:100B500010F003030AD1B0F5047F05D200F1005074
:100B6000A0F51040D0F80038184670470023FBE786
:100B700000F10050A0F51040D0F8100A70470000B6
:100B8000064991F8243033B10023086A81F82430F3
:100B90000822FFF7B1BF0120704700BF6C2300207F
:100BA000014B1868704700BF002004E070B5194B76
:100BB0001D68194B0138C5F30B0408442D0C0422A1
:100BC0001E88A6420BD15C680A46013C824213464D
:100BD0000FD214F9016F4EB102F8016BF6E7013A3A
:100BE00003F10803ECD181420B4602D22C2203F818
:100BF000012B0A4A05241688AE4204D1984284BFCC
:100C0000967803F8016B013C02F10402F3D1581A03
:100C100070BD00BF002004E08C3400087834000868
:100C2000022802BF024B4FF000429A61704700BF9A
:100C300000080240022802BF024B4FF400429A61B2
:100C4000704700BF00080240022801BF024A5369F2
:100C500083F40043536170470008024070B50446B6
:100C60004FF47A764CB1412C254628BF412506FB2E
:100C700005F000F0D3FD641BF4E770BD10B5002350
:100C8000934203D0CC5CC4540133F9E710BD00009B
:100C900010B5013810F9013F3BB191F900409C4279
:100CA00003D11AB10131013AF4E71AB191F90020E8
:100CB000981A10BD1046FCE703460246D01A12F9F6
:100CC000011B0029FAD1704702440346934202D027
:100CD00003F8011BFAE770472DE9F8431F4D14464E
:100CE00095F824200746884652BBDFF870909CB3E5
:100CF00095F824302BB92022FF2148462F62FFF7B8
:100D0000E3FF95F82400C0F10802A24228BF224662
:100D1000D6B24146920005EB8000FFF7AFFF95F891
:100D20002430A41B1E44F6B2082E17449044E4B2AB
:100D300085F82460DBD1FFF723FF0028D7D108E036
:100D40002B6A03EB82038342CFD0FFF719FF002801
:100D5000CBD10020BDE8F8830120FBE76C23002005
:100D6000024B1A78024B1A70704700BF9423002080
:100D70001022002010B5104C104800F0B5F82146A4
:100D80000E4800F0DDF82468626DD2F8043843F0B4
:100D90000203C2F804384FF47A70FFF75FFF084986
:100DA000204600F0D3F9626DD2F8043823F0020334
:100DB000C2F8043810BD00BF5835000808260020CE
:100DC000603500087047000030B5094D0A44914273
:100DD0000DD011F8013B5840082340F30004013BBB
:100DE0002C4013F0FF0384EA5000F6D1EFE730BD4A
:100DF0002083B8ED026843681143016003B11847CE
:100E00007047000013B5446BD4F894341A68117815
:100E1000042915D1217C022912D1197912890123C3
:100E20008B4013420CD101A904F14C0001F0F4FEF7
:100E3000D4F89444019B21790246206800F0D0F94F
:100E400002B010BD143001F077BE00004FF0FF3348
:100E5000143001F071BE00004C3001F049BF0000B9
:100E60004FF0FF334C3001F043BF0000143001F06D
:100E700045BE00004FF0FF31143001F03FBE0000CE
:100E80004C3001F015BF00004FF0FF324C3001F044
:100E90000FBF00000020704710B5D0F894341A68D6
:100EA00011780429044617D1017C022914D15979FB
:100EB000528901238B4013420ED1143001F0D8FD2A
:100EC000024648B1D4F894444FF4807361792068A5
:100ED000BDE8104000F072B910BD0000406BFFF794
:100EE000DBBF0000704700007FB5124B036000239A
:100EF0004360C0E90233012502260F4B0574044606
:100F00000290019300F18402294600964FF4807309
:100F1000143001F089FD094B0294CDE9006304F51A
:100F200023724FF48073294604F14C0001F050FE07
:100F300004B070BDAC340008DD0E0008050E0008DA
:100F40000B68302282F311880A7903EB82029061E8
:100F50004A79093243F822008A7912B103EB8203FD
:100F600098610223C0F894140374002080F3118860
:100F70007047000038B5037F044613B190F8543031
:100F8000ABB9201D01250221FFF734FF04F1140045
:100F900025776FF0010100F069FC84F8545004F1EA
:100FA0004C006FF00101BDE8384000F05FBC38BD77
:100FB00010B5012104460430FFF71CFF00232377FE
:100FC00084F8543010BD000038B5044600251430B4
:100FD00001F042FD04F14C00257701F011FE201DC7
:100FE00084F854500121FFF705FF2046BDE8384042
:100FF000FFF752BF90F8443003F06003202B07D175
:1010000090F84520212A4FF0000303D81F2A06D864
:1010100000207047222AFBD1C0E90E3303E0034AC7
:1010200082630722C26303640120704711220020FB
:1010300037B5D0F894341A681178042904461AD1C7
:10104000017C022917D11979128901238B4013429F
:1010500011D100F14C05284601F092FE58B101A9CA
:10106000284601F0D9FDD4F89444019B2179024629
:10107000206800F0B5F803B030BD0000F0B500EB1B
:10108000810385B09E6904460D46FEB1302383F38B
:10109000118804EB8507301D0821FFF7ABFEFB68C4
:1010A0005B691B6806F14C001BB1019001F0C2FDA9
:1010B000019803A901F0B0FD024648B1039B2946FF
:1010C000204600F08DF8002383F3118805B0F0BDB1
:1010D000FB685A691268002AF5D01B8A013B13404D
:1010E000F1D104F14402EAE7093138B550F8214062
:1010F000DCB1302383F31188D4F894241368527937
:1011000003EB8203DB689B695D6845B104216018CD
:10111000FFF770FE294604F1140001F0B3FC2046ED
:10112000FFF7BAFE002383F3118838BD7047000033
:1011300001F012B8012303700023C0E90133C36139
:1011400083620362C36243620363704738B5044637
:10115000302383F311880025C0E90355C0E9055504
:10116000416001F009F80223237085F311882846B5
:1011700038BD000070B500EB810305465069DA60A8
:101180000E46144618B110220021FFF79DFDA069FC
:1011900018B110220021FFF797FD31462846BDE81F
:1011A000704001F0B3B80000826802F00112826062
:1011B0000022C0E90422826101F034B9F0B400EBEE
:1011C00081044789E4680125A4698D403D43458138
:1011D00023600023A2606360F0BC01F04FB90000FF
:1011E000F0B400EB81040789E468012564698D404F
:1011F0003D43058123600023A2606360F0BC01F0E1
:10120000C9B9000070B50223002504460370C0E987
:101210000255C0E90455C564856180F8345001F079
:1012200011F863681B6823B129462046BDE8704069
:10123000184770BD0378052B10B504460AD080F816
:1012400050300523037043681B680BB10421984795
:101250000023A36010BD00000178052906D190F895
:101260005020436802701B6803B1184770470000A4
:1012700070B590F83430044613B1002380F8343050
:1012800004F14402204601F0EFF863689B68B3B9AB
:1012900094F8443013F0600535D00021204601F069
:1012A0008FFB0021204601F081FB63681B6813B1AE
:1012B000062120469847062384F8343070BD204626
:1012C00098470028E4D0B4F84A30E26B9A4288BFCD
:1012D000E36394F94430E56B002B4FF0300380F268
:1012E0000381002D00F0F280092284F8342083F37A
:1012F00011880021D4E90E232046FFF771FF002357
:1013000083F31188DAE794F8452003F07F0343EA7A
:10131000022340F20232934200F0C58021D8B3F597
:10132000807F48D00DD8012B3FD0022B00F0938056
:10133000002BB2D104F14C02A2630222E2632364C7
:10134000C1E7B3F5817F00F09B80B3F5407FA4D166
:1013500094F84630012BA0D1B4F84C3043F002038E
:1013600032E0B3F5006F4DD017D8B3F5A06F31D090
:10137000A3F5C063012B90D8636894F846205E689B
:1013800094F84710B4F848302046B047002884D07D
:101390004368A3630368E3631AE0B3F5106F36D0C4
:1013A00040F6024293427FF478AF5C4BA363022382
:1013B000E3630023C3E794F84630012B7FF46DAF5D
:1013C000B4F84C3023F00203C4E90E55A4F84C30B5
:1013D000256478E7B4F84430B3F5A06F0ED194F8E3
:1013E000463084F84E30204600F084FF63681B6866
:1013F00013B1012120469847032323700023C4E939
:101400000E339CE704F14F03A3630123C3E7237862
:10141000042B10D1302383F311882046FFF7C4FE3C
:1014200085F311880321636884F84F5021701B688D
:101430000BB12046984794F84630002BDED084F854
:101440004F300423237063681B68002BD6D0022121
:1014500020469847D2E794F848301D0603F00F0164
:1014600020460AD500F0F2FF012804D002287FF4BC
:1014700014AF2B4B9AE72B4B98E700F0D9FFF3E71B
:1014800094F84630002B7FF408AF94F8483013F0FE
:101490000F01B3D01A06204602D501F0A5FAADE738
:1014A00001F098FAAAE794F84630002B7FF4F5AEE5
:1014B00094F8483013F00F01A0D01B06204602D547
:1014C00001F07EFA9AE701F071FA97E7142284F8A6
:1014D000342083F311882B462A4629462046FFF7FD
:1014E0006DFE85F31188E9E65DB1152284F834209C
:1014F00083F311880021D4E90E232046FFF75EFE16
:10150000FDE60B2284F8342083F311882B462A460B
:1015100029462046FFF764FEE3E700BFDC340008FD
:10152000D4340008D834000838B590F83430044674
:10153000002B3ED0063BDAB20F2A34D80F2B32D81C
:10154000DFE803F0373131082232313131313131C6
:1015500031313737C56BB0F84A309D4214D2C36879
:101560001B8AB5FBF3F203FB12556DB9302383F3ED
:1015700011882B462A462946FFF732FE85F311884B
:101580000A2384F834300EE0142384F834303023F6
:1015900083F3118800231A4619462046FFF70EFEF2
:1015A000002383F3118838BD036C03B198470023EF
:1015B000E7E70021204601F003FA0021204601F070
:1015C000F5F963681B6813B1062120469847062386
:1015D000D7E7000010B590F83430142B044629D01A
:1015E00017D8062B05D001D81BB110BD093B022B23
:1015F000FBD80021204601F0E3F90021204601F04C
:10160000D5F963681B6813B1062120469847062365
:1016100019E0152BE9D10B2380F83430302383F304
:10162000118800231A461946FFF7DAFD002383F3D9
:101630001188DAE7C3689B695B68002BD5D1036C1E
:1016400003B19847002384F83430CEE700230375B4
:10165000826803691B6899689142FBD25A680360EB
:101660004260106058607047002303758268036908
:101670001B6899689142FBD85A6803604260106009
:101680005860704708B50846302383F311880B7DF6
:10169000032B05D0042B0DD02BB983F3118808BD83
:1016A0008B6900221A604FF0FF338361FFF7CEFF92
:1016B0000023F2E7D1E9003213605A60F3E700003B
:1016C000FFF7C4BF054BD9680875186802681A602F
:1016D000536001220275D860FEF714BE98230020E3
:1016E00030B50C4BDD684B1C87B004460FD02B4641
:1016F000094A684600F04EF92046FFF7E3FF009BD9
:1017000013B1684600F050F9A86907B030BDFFF783
:10171000D9FFF9E79823002085160008044B1A68C2
:10172000DB6890689B68984294BF00200120704756
:1017300098230020084B10B51C68D86822681A60EE
:10174000536001222275DC60FFF78EFF01462046C0
:10175000BDE81040FEF7D6BD9823002038B5074CF1
:1017600007490848012300252370656001F040FB0C
:101770000223237085F3118838BD00BF00260020A6
:10178000E43400089823002000F044B9034A51686B
:1017900053685B1A9842FBD8704700BF001000E006
:1017A0008B60022308618B82084670478368A3F12F
:1017B000840243F8142C026943F8442C426943F82C
:1017C000402C094A43F8242CC26843F8182C022202
:1017D00003F80C2C002203F80B2C044A43F8102CBD
:1017E000A3F12000704700BF1D03000898230020CC
:1017F00008B5FFF7DBFFBDE80840FFF761BF000059
:10180000024BDB6898610F20FFF75CBF9823002034
:10181000302383F31188FFF7F3BF000008B50146BA
:10182000302383F311880820FFF75AFF002383F346
:10183000118808BD064BDB6839B1426818605A60F0
:10184000136043600420FFF74BBF4FF0FF30704739
:10185000982300200368984206D01A6802605060FE
:1018600099611846FFF72CBF7047000038B5044651
:101870000D462068844200D138BD036823605C6057
:101880008561FFF71DFFF4E710B503689C68A2426D
:101890000CD85C688A600B604C6021605960996864
:1018A0008A1A9A604FF0FF33836010BD1B68121BC9
:1018B000ECE700000A2938BF0A2170B504460D463E
:1018C0000A26601901F08EFA01F07AFA041BA5428B
:1018D00003D8751C2E460446F3E70A2E04D9BDE84A
:1018E0007040012001F0C4BA70BD0000F8B5144B7F
:1018F0000D46D96103F1100141600A2A196982601D
:1019000038BF0A22016048601861A818144601F027
:101910005BFA0A2701F054FA431BA342064606D39A
:101920007C1C281901F05EFA27463546F2E70A2F9B
:1019300004D9BDE8F840012001F09ABAF8BD00BF13
:1019400098230020F8B506460D4601F039FA0F4AF3
:10195000134653F8107F9F4206D12A46014630466F
:10196000BDE8F840FFF7C2BFD169BB68441A2C1923
:1019700028BF2C46A34202D92946FFF79BFF2246E7
:1019800031460348BDE8F840FFF77EBF98230020AA
:10199000A823002010B4C0E9032300235DF8044B02
:1019A0004361FFF7CFBF000010B5194C236998427F
:1019B0000DD0D0E90032816813605A609A680A44F9
:1019C0009A60002303604FF0FF33A36110BD2346EC
:1019D000026843F8102F53600022026022699A4285
:1019E00003D1BDE8104001F0F7B9936881680B445A
:1019F000936001F0E5F92269E1699268441AA24214
:101A0000E4D91144BDE81040091AFFF753BF00BFE5
:101A1000982300202DE9F047DFF8BC8008F110077B
:101A20002C4ED8F8105001F0CBF9D8F81C40AA6819
:101A3000031B9A423ED81444D5E900324FF0000906
:101A4000C8F81C4013605A60C5F80090D8F81030F0
:101A5000B34201D101F0C0F989F31188D5E903310E
:101A600028469847302383F311886B69002BD8D020
:101A700001F0A6F96A69A0EB04094A4582460DD235
:101A8000022001F0F5F90022D8F81030B34208D155
:101A900051462846BDE8F047FFF728BF121A2244F6
:101AA000F2E712EB090938BF4A4629463846FFF7E4
:101AB000EBFEB5E7D8F81030B34208D01444211A31
:101AC000C8F81C00A960BDE8F047FFF7F3BEBDE809
:101AD000F08700BFA8230020982300200020704733
:101AE000FEE70000704700004FF0FF307047000035
:101AF00002290CD0032904D00129074818BF00206F
:101B00007047032A05D8054800EBC2007047044817
:101B100070470020704700BFBC350008202200201D
:101B20007035000870B59AB00546084601A91446FC
:101B300000F0C2F801A8FFF7BFF8431C5B00C5E93D
:101B400000340022237003236370C6B201AB023459
:101B50001046D1B28E4204F1020401D81AB070BD11
:101B600013F8011B04F8021C04F8010C0132F0E721
:101B700008B5302383F311880348FFF759FA00238F
:101B800083F3118808BD00BF0826002090F8443078
:101B900003F01F02012A07D190F845200B2A03D138
:101BA0000023C0E90E3315E003F06003202B08D1B9
:101BB000B0F848302BB990F84520212A03D81F2AC5
:101BC00004D8FFF717BA222AEBD0FAE7034A826358
:101BD0000722C26303640120704700BF182200205F
:101BE00007B5052917D8DFE801F0191603191920E0
:101BF000302383F31188104A01900121FFF7BAFACC
:101C000001980E4A0221FFF7B5FA0D48FFF7DCF9FB
:101C1000002383F3118803B05DF804FB302383F3C2
:101C200011880748FFF7A6F9F2E7302383F31188FC
:101C30000348FFF7BDF9EBE710350008343500081D
:101C40000826002038B50C4D0C4C0D492A4604F1ED
:101C50000800FFF767FF05F1CA0204F11000094907
:101C6000FFF760FF05F5CA7204F118000649BDE8E8
:101C70003840FFF757BF00BFD02A002020220020A5
:101C8000F0340008FA3400080535000870B5044641
:101C900008460D46FFF710F8C6B220460134037817
:101CA0000BB9184670BD32462946FEF7F1FF0028F1
:101CB000F3D10120F6E700002DE9F84F05460C4668
:101CC000FEF7FAFF2949C6B22846FFF7DFFF08B141
:101CD000013EF6B226492846FFF7D8FF08B1103674
:101CE000F6B2632E0DD8DFF88490DFF884A0214F80
:101CF000DFF888B0DFF888802E7846B92670BDE816
:101D0000F88F29462046BDE8F84F01F097BB252EF5
:101D100028D1072249462846FEF7BAFF40B9D8F82D
:101D200000302360B8F80430A38007350634E3E7B9
:101D3000082251462846FEF7ABFF98B90E4BA21C6D
:101D4000197809090232C95D02F8041C13F8011B55
:101D500001F00F015B45C95D02F8031CF0D1183496
:101D60000835C9E704F8016B0135C5E7DC35000823
:101D700005350008EB350008107AFF1F1C7AFF1F9D
:101D8000E4350008BFF34F8F024AD368DB03FCD46D
:101D9000704700BF003C024008B5094B1B7873B97F
:101DA000FFF7F0FF074B1A69002ABFBF064A5A60C7
:101DB00002F188325A601A6822F480621A6008BD03
:101DC0002E2D0020003C02402301674508B50B4B37
:101DD0001B7893B9FFF7D6FF094B1A6942F000420E
:101DE0001A611A6842F480521A601A6822F480520A
:101DF0001A601A6842F480621A6008BD2E2D002015
:101E0000003C02400B28F0B516D80C4C0C49237846
:101E10007BB90C4D0E460C234FF0006255F8047B45
:101E200046F8042B013B13F0FF033A44F6D101239B
:101E3000237051F82000F0BD0020FCE7602D002049
:101E4000302D0020FC350008014B53F8200070476E
:101E5000FC3500080C2070470B2810B5044601D94A
:101E6000002010BDFFF7CEFF064B53F82430184476
:101E7000C21A0BB90120F4E712680132F0D1043B19
:101E8000F6E700BFFC3500080B2810B5044621D842
:101E9000FFF778FFFFF780FF0F4AF323D360C300FB
:101EA000DBB243F4007343F002031361136943F49C
:101EB00080331361FFF766FFFFF7A4FF074B53F86A
:101EC000241000F0D9F8FFF781FF2046BDE810404C
:101ED000FFF7C2BF002010BD003C0240FC350008E7
:101EE000F8B512F00103144642D18218B2F1016F25
:101EF00057D82D4B1B6813F0010352D02B4DFFF721
:101F00004BFFF323EB60FFF73DFF40F20127032C6B
:101F100015D824F001046618244C401A40F2011729
:101F2000B142236900EB010524D123F001032361B1
:101F3000FFF74CFF0120F8BD043C0430E7E78307BE
:101F4000E7D12B6923F440732B612B693B432B6151
:101F500051F8046B0660BFF34F8FFFF713FF036860
:101F60009E42E9D02B6923F001032B61FFF72EFF7E
:101F70000020E0E723F44073236123693B4323619E
:101F80000B882B80BFF34F8FFFF7FCFE2D8831F8B5
:101F9000023BADB2AB42C3D0236923F001032361FE
:101FA000E4E71846C7E700BF00380240003C0240A3
:101FB000084908B50B7828B11BB9FFF7EDFE0123DE
:101FC0000B7008BD002BFCD0BDE808400870FFF77F
:101FD000FDBE00BF2E2D002010B50244064BD2B22C
:101FE000904200D110BD441C00B253F8200041F8CB
:101FF000040BE0B2F4E700BF502800400F4B30B5AF
:102000001C6F240407D41C6F44F400741C671C6FFD
:1020100044F400441C670A4C236843F48073236033
:102020000244084BD2B2904200D130BD441C00B2F1
:1020300051F8045B43F82050E0B2F4E70038024066
:10204000007000405028004007B5012201A900207F
:10205000FFF7C2FF019803B05DF804FB13B5044617
:10206000FFF7F2FFA04205D0012201A90020019450
:10207000FFF7C4FF02B010BD70470000034B1A68A1
:102080001AB9034AD2F874281A607047642D0020E8
:102090000030024008B5FFF7F1FF024B1868C0F3AB
:1020A000407008BD642D002070470000FEE700006E
:1020B0000A4B0B480B4A90420BD30B4BDA1C121AFB
:1020C000C11E22F003028B4238BF00220021FEF71E
:1020D000FBBD53F8041B40F8041BECE7A8370008CD
:1020E000602E0020602E0020602E002070B5D0E908
:1020F00015439E6800224FF0FF3504EB4213510157
:10210000D3F800090028BEBFD3F8000940F0804092
:10211000C3F80009D3F8000B0028BEBFD3F8000BAA
:1021200040F08040C3F8000B013263189642C3F8B8
:102130000859C3F8085BE0D24FF00113C4F81C380B
:1021400070BD0000890141F02001016103699B0617
:10215000FCD41220FFF71ABB10B5054C2046FEF741
:10216000E9FF4FF0A0436365024BA36510BD00BFBC
:10217000682D00205036000870B50378012B054605
:1021800050D12A4B446D98421BD1294B5A6B42F0D7
:1021900080025A635A6D42F080025A655A6D5A693C
:1021A00042F080025A615A6922F080025A610E217F
:1021B00043205B6900F022FC1E4BE3601E4BC4F819
:1021C00000380023C4F8003EC02323606E6D4FF436
:1021D0000413A3633369002BFCDA012333610C2061
:1021E000FFF7D4FA3369DB07FCD41220FFF7CEFAED
:1021F0003369002BFCDA0026A6602846FFF776FF3D
:102200006B68C4F81068DB68C4F81468C4F81C680C
:102210004BB90A4BA3614FF0FF336361A36843F0EE
:102220000103A36070BD064BF4E700BF682D0020DA
:10223000003802404014004003002002003C30C03F
:10224000083C30C0F8B5446D054600212046FFF734
:1022500079FFA96D00234FF001128F68C4F834385C
:102260004FF00066C4F81C284FF0FF3004EB431217
:1022700001339F42C2F80069C2F8006BC2F8080936
:10228000C2F8080BF2D20B686A6DEB65636210232B
:102290001361166916F01006FBD11220FFF776FACB
:1022A000D4F8003823F4FE63C4F80038A36943F47B
:1022B000402343F01003A3610923C4F81038C4F885
:1022C00014380A4BEB604FF0C043C4F8103B084B86
:1022D000C4F8003BC4F81069C4F80039EB6D03F191
:1022E000100243F48013EA65A362F8BD2C3600089F
:1022F00040800010426D90F84E10D2F8003823F460
:10230000FE6343EA0113C2F8003870472DE9F84331
:1023100000EB8103456DDA68166806F00306731E4C
:10232000022B05EB41130C4680460FFA81F94FEA68
:1023300041104FF00001C3F8101B4FF0010104F1F0
:10234000100398BFB60401FA03F391698EBF334EB0
:1023500006F1805606F5004600293AD0578A04F166
:102360005801490137436F50D5F81C180B43C5F885
:102370001C382B180021C3F8101953690127611E5E
:10238000A7409BB3138A928B9B08012A88BF5343B3
:10239000D8F85C20981842EA034301F1400205EBAB
:1023A0008202C8F85C00214653602846FFF7CAFE47
:1023B00008EB8900C3681B8A43EA845348346401EC
:1023C0001E432E51D5F81C381F43C5F81C78BDE8B4
:1023D000F88305EB4917D7F8001B21F40041C7F833
:1023E000001BD5F81C1821EA0303C0E704F13F03E2
:1023F00005EB83030A4A5A6028462146FFF7A2FEEE
:1024000005EB4910D0F8003923F40043C0F8003937
:10241000D5F81C3823EA0707D7E700BF0080001073
:1024200000040002826D1268C265FFF75FBE000003
:102430005831436D49015B5813F4004004D013F444
:10244000001F0CBF02200120704700004831436D7F
:1024500049015B5813F4004004D013F4001F0CBF73
:10246000022001207047000000EB8101CB68196A4F
:102470000B6813604B6853607047000000EB8103EA
:1024800030B5DD68AA691368D36019B9402B84BFE1
:10249000402313606B8A1468426D1C44013CB4FBFA
:1024A000F3F46343033323F0030302EB411043EAE5
:1024B000C44343F0C043C0F8103B2B6803F0030350
:1024C000012B09B20ED1D2F8083802EB411013F4F7
:1024D000807FD0F8003B14BF43F0805343F000539B
:1024E000C0F8003B02EB4112D2F8003B43F004433A
:1024F000C2F8003B30BD00002DE9F041244D6E6D67
:1025000006EB40130446D3F8087BC3F8087B380772
:102510000AD5D6F81438190706D505EB84032146E9
:10252000DB6828465B689847FA071FD5D6F8143849
:10253000DB071BD505EB8403D968CCB98B69488AC6
:102540005A68B2FBF0F600FB16228AB91868DA68FE
:1025500090420DD2121AC3E90024302383F311886C
:102560000B482146FFF78AFF84F31188BDE8F0810C
:10257000012303FA04F26B8923EA02036B81CB681F
:10258000002BF3D021460248BDE8F041184700BFB8
:10259000682D002000EB810370B5DD68436D6C6928
:1025A0002668E6604A0156BB1A444FF40020C2F880
:1025B00010092A6802F00302012A0AB20ED1D3F8E8
:1025C000080803EB421410F4807FD4F8000914BF0C
:1025D00040F0805040F00050C4F8000903EB421274
:1025E000D2F8000940F00440C2F80009D3F83408DA
:1025F000012202FA01F10143C3F8341870BD19B980
:10260000402E84BF4020206020682E8A8419013C1F
:10261000B4FBF6F440EAC44040F000501A44C6E768
:102620002DE9F8433B4D6E6D06EB40130446D3F89D
:102630000889C3F8088918F0010F4FEA40171AD02B
:10264000D6F81038DB0716D505EB8003D9684B693F
:102650001868DA68904230D2121A4FF000091A60F6
:10266000C3F80490302383F3118821462846FFF7EE
:1026700091FF89F3118818F0800F1CD0D6F83438F8
:102680000126A640334216D005EB84036D6DD3F8C6
:102690000CC0DCF814200134E4B2D2F800E005EB01
:1026A00004342F445168714515D3D5F8343823EAE2
:1026B0000606C5F83468BDE8F883012303FA04F27E
:1026C0002B8923EA02032B818B68002BD3D0214670
:1026D00028469847CFE7BCF81000AEEB01038342D1
:1026E00028BF0346D7F8180980B2B3EB800FE2D8B1
:1026F0009068A0F1040959F8048FC4F80080A0EB99
:1027000009089844B8F1040FF5D818440B449060B8
:102710005360C7E7682D00202DE9F74FA24C656D87
:102720006E69AB691E4016F480586E6107D0204672
:10273000FEF768FD03B0BDE8F04F00F047BC002E87
:1027400012DAD5F8003E98489B071EBFD5F8003E28
:1027500023F00303C5F8003ED5F8043823F0010345
:10276000C5F80438FEF778FD370505D58E48FFF724
:10277000BDFC8D48FEF75EFDB0040CD5D5F80838D9
:1027800013F0060FEB6823F470530CBF43F410539F
:1027900043F4A053EB6031071BD56368DB681BB9BA
:1027A000AB6923F00803AB612378052B0CD1D5F876
:1027B000003E7D489A071EBFD5F8003E23F0030374
:1027C000C5F8003EFEF748FD6368DB680BB176484C
:1027D0009847F30274D4B70227D5D4F85490DFF8A1
:1027E000C8B100274FF0010A09EB4712D2F8003BAD
:1027F00003F44023B3F5802F11D1D2F8003B002B16
:102800000DDA62890AFA07F322EA0303638104EB13
:102810008703DB68DB6813B1394658469847A36DD8
:1028200001379B68FFB29F42DED9F00617D5676D6E
:102830003A6AC2F30A1002F00F0302F4F012B2F582
:10284000802F00F08580B2F5402F08D104EB830380
:102850000022DB681B6A07F5805790426AD130037B
:10286000D5F8184813D5E10302D50020FFF744FE40
:10287000A20302D50120FFF73FFE630302D5022029
:10288000FFF73AFE270302D50320FFF735FE750355
:102890007FF550AFE00702D50020FFF7C1FEA1078A
:1028A00002D50120FFF7BCFE620702D50220FFF728
:1028B000B7FE23077FF53EAF0320FFF7B1FE39E7F0
:1028C000636DDFF8E4A0019300274FF00109A36DC9
:1028D0009B685FFA87FB9B453FF67DAF019B03EB4F
:1028E0004B13D3F8001901F44021B1F5802F1FD10B
:1028F000D3F8001900291BDAD3F8001941F09041F0
:10290000C3F80019D3F800190029FBDB5946606DA4
:10291000FFF718FC218909FA0BF321EA030323814D
:1029200004EB8B03DB689B6813B15946504698470C
:102930000137CCE7910708BFD7F80080072A98BF76
:1029400003F8018B02F1010298BF4FEA182884E7CF
:10295000023304EB830207F580575268D2F818C09F
:10296000DCF80820DCE9001CA1EB0C0C00218842FB
:102970000AD104EB830463689B699A6802449A60F5
:102980005A6802445A606AE711F0030F08BFD7F88B
:1029900000808C4588BF02F8018B01F1010188BFDE
:1029A0004FEA1828E3E700BF682D0020436D03EBD2
:1029B0004111D1F8003B43F40013C1F8003B7047CC
:1029C000436D03EB4111D1F8003943F40013C1F812
:1029D00000397047436D03EB4111D1F8003B23F4FC
:1029E0000013C1F8003B7047436D03EB4111D1F870
:1029F000003923F40013C1F80039704700F1604337
:102A000003F561430901C9B283F80013012200F004
:102A10001F039A4043099B0003F1604303F56143A0
:102A2000C3F880211A60704730B5039C01720433EB
:102A300004FB0325C0E90653049B03630021059BA7
:102A4000C160C0E90000C0E90422C0E90842C0E951
:102A50000A11436330BD0000416A0022C0E904113D
:102A6000C0E90A22C2606FF00101FEF7FFBE00005C
:102A7000D0E90432934201D1C2680AB9181D7047E7
:102A80000020704703691960C2680132C260C269E0
:102A9000134482690361934224BF436A03610021A6
:102AA000FEF7D8BE38B504460D46E3683BB162690F
:102AB000131D1268A3621344E362002007E0237A27
:102AC00033B929462046FEF7B5FE0028EDDA38BDB9
:102AD0006FF00100FBE70000C368C269013BC360FF
:102AE0004369134482694361934224BF436A43614B
:102AF00000238362036B03B11847704770B530231E
:102B0000044683F31188866A3EB9FFF7CBFF05467A
:102B100018B186F31188284670BDA36AE26A13F8DB
:102B2000015BA362934202D32046FFF7D5FF002347
:102B300083F31188EFE700002DE9F84F04460E46B5
:102B4000174698464FF0300989F311880025AA46A8
:102B5000D4F828B0BBF1000F09D141462046FFF759
:102B6000A1FF20B18BF311882846BDE8F88FD4E986
:102B70000A12A7EB050B521A934528BF9346BBF1E7
:102B8000400F1BD9334601F1400251F8040B43F8C2
:102B9000040B9142F9D1A36A40334036A362403519
:102BA000D4E90A239A4202D32046FFF795FF8AF31D
:102BB0001188BD42D8D289F31188C9E730465A46F8
:102BC000FEF75CF8A36A5B445E44A3625D44E7E7FA
:102BD00010B5029C0172043303FB0421C0E9061303
:102BE0000023C0E90A33039B0363049BC460C0E96C
:102BF0000000C0E90422C0E90842436310BD0000A0
:102C0000026AC260426AC0E904220022C0E90A22C4
:102C10006FF00101FEF72ABED0E904239A4201D1E8
:102C2000C26822B9184650F8043B0B607047002375
:102C30001846FAE7C368C2690133C36043691344A5
:102C400082694361934224BF436A43610021FEF7D6
:102C500001BE000038B504460D46E3683BB1236968
:102C60001A1DA262E2691344E362002007E0237A9E
:102C700033B929462046FEF7DDFD0028EDDA38BDE0
:102C80006FF00100FBE7000003691960C268013AB8
:102C9000C260C269134482690361934224BF436ADC
:102CA000036100238362036B03B118477047000080
:102CB00070B530230D460446114683F31188866AA9
:102CC0002EB9FFF7C7FF10B186F3118870BDA36A54
:102CD0001D70A36AE26A01339342A36204D3E169DF
:102CE00020460439FFF7D0FF002080F31188EDE77C
:102CF0002DE9F84F04460D46904699464FF0300AAC
:102D00008AF311880026B346A76A4FB94946204680
:102D1000FFF7A0FF20B187F311883046BDE8F88F98
:102D2000D4E90A073A1AA8EB0607974228BF1746C4
:102D3000402F1BD905F1400355F8042B40F8042B14
:102D40009D42F9D1A36A4033A3624036D4E90A23F5
:102D50009A4204D3E16920460439FFF795FF8BF3CB
:102D600011884645D9D28AF31188CDE729463A46DB
:102D7000FDF784FFA36A3B443D44A3623E44E5E77C
:102D8000D0E904239A4217D1C3689BB1836A8BB1FF
:102D9000043B9B1A0ED01360C368013BC360C36938
:102DA0001A44836902619A4224BF436A0361002383
:102DB00083620123184670470023FBE700F030B917
:102DC0004FF08043586A70474FF0804300225863A9
:102DD0001A610222DA6070474FF080430022DA6005
:102DE000704700004FF0804358637047FEE70000D3
:102DF00070B51B4B01630025044686B058608562A0
:102E00000E4600F0BFF804F11003C4E904334FF09C
:102E1000FF33C4E90635C4E90044A560E562FFF765
:102E2000CFFF2B460246C4E9082304F134010D4AC2
:102E3000256580232046FEF7B3FC0123E0600A4AA3
:102E40000375009272680192B268CDE90223074BC4
:102E50006846CDE90435FEF7CBFC06B070BD00BF77
:102E6000002600205C36000861360008ED2D0008C1
:102E7000024AD36A1843D062704700BF98230020EB
:102E80004B6843608B688360CB68C3600B694361A8
:102E90004B6903628B6943620B68036070470000F3
:102EA00008B5264B26481A6940F2FF110A431A61F9
:102EB0001A6922F4FF7222F001021A611A691A6B70
:102EC0000A431A631A6D0A431A651E4A1B6D11469E
:102ED000FFF7D6FF02F11C0100F58060FFF7D0FF7D
:102EE00002F1380100F58060FFF7CAFF02F15401DA
:102EF00000F58060FFF7C4FF02F1700100F580600B
:102F0000FFF7BEFF02F18C0100F58060FFF7B8FF0C
:102F100002F1A80100F58060FFF7B2FF02F1C401E1
:102F200000F58060FFF7ACFF02F1E00100F5806082
:102F3000FFF7A6FFBDE8084000F0EEB800380240F9
:102F4000000002406836000808B500F059FAFEF7A4
:102F500005FCFFF793F8BDE80840FEF773BE0000DC
:102F600070470000EFF3098305494A6B22F0010224
:102F70004A63683383F30988002383F31188704719
:102F800000EF00E0302080F3118862B60C4B0D4A50
:102F9000D96821F4E0610904090C0A43DA60D3F826
:102FA000FC20094942F08072C3F8FC200A6842F014
:102FB00001020A602022DA7783F82200704700BFFE
:102FC00000ED00E00003FA05001000E010B530232A
:102FD00083F311880E4B5B6813F4006314D0F1EE99
:102FE000103AEFF30984683C4FF08073E361094BBA
:102FF000DB6B236684F30988FEF790FB10B1064B68
:10300000A36110BD054BFBE783F31188F9E700BF0F
:1030100000ED00E000EF00E02F030008320300089D
:103020000F4B1A6C42F001021A641A6E42F0010250
:103030001A660C4A1B6E936843F0010393604FF0CD
:10304000804353229A624FF0FF32DA6200229A6183
:103050005A63DA605A6001225A611A60704700BFF1
:1030600000380240002004E04FF0804208B51169AA
:10307000D3680B40D9B2C9439B07116107D53023F0
:1030800083F31188FEF780FB002383F3118808BDCA
:103090001F4B1A696FEAC2526FEAD2521A611A695B
:1030A000C2F308021A614FF0FF301A695A69586179
:1030B00000215A6959615A691A6A62F080521A628B
:1030C0001A6A02F080521A621A6A5A6A58625A6A76
:1030D00059625A6A1A6C42F080521A641A6E42F0AF
:1030E00080521A661A6E0B4A106840F480701060A5
:1030F000186F00F44070B0F5007F1EBF4FF48030B1
:1031000018671967536823F40073536000F054B9CB
:103110000038024000700040334B4FF080521A6478
:10312000324A4FF4404111601A6842F001021A60BD
:103130001A689107FCD59A6822F003029A602A4B1C
:103140009A6812F00C02FBD1196801F0F9011960BC
:103150009A601A6842F480321A601A689203FCD5A9
:103160005A6F42F001025A671F4B5A6F9007FCD505
:103170001F4A5A601A6842F080721A601B4A5368EC
:103180005904FCD5184B1A689201FCD5194A9A606B
:10319000194B1A68194B9A42194B21D1194A1168D7
:1031A000194A91421CD140F205121A60144A136860
:1031B00003F00F03052BFAD10B4B9A6842F0020281
:1031C0009A609A6802F00C02082AFAD15A6C42F40A
:1031D00080425A645A6E42F480425A665B6E70476F
:1031E00040F20572E1E700BF003802400070004085
:1031F0000854400700948838002004E0116400203F
:10320000003C024000ED00E041C20F41074A08B512
:10321000536903F00103536123B1054A13680BB1ED
:1032200050689847BDE80840FFF7D0BE003C014019
:10323000E02D0020074A08B5536903F002035361EB
:1032400023B1054A93680BB1D0689847BDE80840A0
:10325000FFF7BCBE003C0140E02D0020074A08B546
:10326000536903F00403536123B1054A13690BB199
:1032700050699847BDE80840FFF7A8BE003C0140F0
:10328000E02D0020074A08B5536903F00803536195
:1032900023B1054A93690BB1D0699847BDE808404E
:1032A000FFF794BE003C0140E02D0020074A08B51E
:1032B000536903F01003536123B1054A136A0BB13C
:1032C000506A9847BDE80840FFF780BE003C0140C7
:1032D000E02D0020164B10B55C6904F478725A6139
:1032E000A30604D5134A936A0BB1D06A98476006C7
:1032F00004D5104A136B0BB1506B9847210604D5C7
:103300000C4A936B0BB1D06B9847E20504D5094A80
:10331000136C0BB1506C9847A30504D5054A936C08
:103320000BB1D06C9847BDE81040FFF74FBE00BF0F
:10333000003C0140E02D0020194B10B55C6904F4FD
:103340007C425A61620504D5164A136D0BB1506D6B
:103350009847230504D5134A936D0BB1D06D984758
:10336000E00404D50F4A136E0BB1506E9847A104C8
:1033700004D50C4A936E0BB1D06E9847620404D505
:10338000084A136F0BB1506F9847230404D5054AC0
:10339000936F0BB1D06F9847BDE81040FFF716BE92
:1033A000003C0140E02D002008B5FFF75DFEBDE8C0
:1033B0000840FFF70BBE0000062108B50846FFF7DE
:1033C0001DFB06210720FFF719FB06210820FFF748
:1033D00015FB06210920FFF711FB06210A20FFF744
:1033E0000DFB06211720FFF709FB06212820FFF718
:1033F00005FBBDE8084007211C20FFF7FFBA0000CD
:1034000008B5FFF745FE00F00BF8FDF791FEFDF75C
:1034100069FDFFF7A5FDBDE80840FFF7CFBC000040
:103420000023054A19460133102BC2E9001102F1AD
:103430000802F8D1704700BFE02D0020034611F8C4
:10344000012B03F8012B002AF9D1704753544D3357
:1034500032463F3F3F0053544D33324634307800BC
:1034600053544D3332463432780053544D33324640
:103470003434365858000000012033000010410059
:1034800001105A000310590007103100000000001D
:103490004C340008130400005634000819040000DE
:1034A00060340008210400006A34000800000000B5
:1034B000610E00084D0E0008890E0008750E000808
:1034C000810E00086D0E0008590E0008450E000818
:1034D000950E000800000000010000000000000040
:1034E00063300000E0340008F023002000260020B4
:1034F0004172647550696C6F740025424F415244AB
:10350000252D424C002553455249414C25000000D1
:1035100002000000000000007D100008E910000813
:1035200040004000A02A0020B02A00200200000035
:103530000000000003000000000000002D11000842
:103540000000000010000000C02A00200000000061
:103550000100000000000000682D002001010200B1
:10356000E11B0008F11A00088D1B0008711B000800
:10357000430000007835000809024300020100C042
:1035800032090400000102020100052400100105B7
:10359000240100010424020205240600010705821B
:1035A000030800FF09040100020A000000070501EA
:1035B00002400000070581024000000012000000E8
:1035C000C4350008120110010200004009124157E1
:1035D00000020102030100000403090425424F41D7
:1035E00052442500574647303031003031323334B1
:1035F00035363738394142434445460000400000E3
:1036000000400000004000000040000000000100F9
:1036100000000200000002000000020000000200A2
:103620000000020000000200000002000000000094
:103630007112000829150008D51500084000400047
:10364000C82D0020C82D002001000000D82D00202A
:103650008000000040010000030000006D61696E01
:103660000069646C650000000000802A0000000012
:10367000AAAAAAAA00000024FFFF00000000000080
:1036800000A00A000000000000000000AAAAAAAAE8
:1036900000000000FFFF000000000000000000002C
:1036A0000000004000000000AAAAAAAA0000000032
:1036B000FF7F00000000000000000000000000008C
:1036C00000000000AAAAAAAA00000000FFFF000054
:1036D00000000000000000000000000000000000EA
:1036E000AAAAAAAA00000000FFFF00000000000034
:1036F000000000000000000000000000AAAAAAAA22
:1037000000000000FFFF00000000000000000000BB
:103710000000000000000000AAAAAAAA0000000001
:10372000FFFF00000000000000000000000000009B
:10373000000000000A00000000000000030000007C
:103740000000000000000000000000000000000079
:103750000000000000000000000000000000000069
:103760000000000000000000FE0700000000000054
:1037700000400F0000000000FF009600000000085D
:10378000009600000000080004000000D835000882
:103790000000000000000000000000000000000029
:1037A0000000000000000000FFFFFFFFFFFFFFFF21
:1037B000FFFFFFFFFFFFFFFFFFFFFFFFFFFFFFFF19
:1037C000FFFFFFFFFFFFFFFFFFFFFFFFFFFFFFFF09
:1037D000FFFFFFFFFFFFFFFFFFFFFFFFFFFFFFFFF9
:1037E000FFFFFFFFFFFFFFFFFFFFFFFFFFFFFFFFE9
:10C000000006002099D20008157709087176090802
:10C01000DD76090871760908A97609089BD200081F
:10C020009BD200089BD200089BD20008F96F0B0836
:10C030009BD200089BD200089BD200089BD200082C
:10C040009BD200089BD200089BD200089BD200081C
:10C050009BD200089BD2000815820B083D820B087A
:10C0600065820B088D820B08B5820B08B12E0B0878
:10C07000D92E0B08052F0B08312F0B085D2F0B084D
:10C08000852F0B08B12F0B08352E0B089BD200080B
:10C090009BD200089BD200089BD20008DD820B08CF
:10C0A00015840B0819840B082D840B0831840B08A8
:10C0B00035840B0849840B085D840B083D350B085B
:10C0C000E5360B089BD200089BD200089BD20008E3
:10C0D0009BD20008B1830B08C5830B08D9830B08DA
:10C0E00041830B089BD200089BD2000881840B0877
:10C0F00085840B0899840B089D840B08DD2F0B08A1
:10C100009BD200089BD2000871840B089BD20008C8
:10C11000ED830B0801840B089BD200089BD200081A
:10C1200009300B0831300B085D300B0889300B08E3
:10C13000B5300B089BD200089BD200089BD20008A8
:10C140009BD200089BD200089BD2000825770B08E1
:10C15000DD300B0809310B0835310B089BD2000884
:10C160009BD200089BD200089BD200089BD20008FB
:10C170009BD200089BD200089BD200089BD20008EB
:10C180009BD200089BD200089BD200089BD20008DB
:10C190009BD200089BD200089BD200089BD20008CB
:10C1A0009BD200089BD200089BD200089BD20008BB
:10C1B0009BD200089BD200089BD200089BD20008AB
:10C1C0009BD200089BD200089BD200089BD200089B
:10C1D0009BD200089BD200089BD200089BD200088B
:10C1E0000DF500084D250108B1AC010835FB01082B
:10C1F000457C0208B9F70308158305081D89050861
:10C200003DF40508C94206088D4A0608C54D0608D2
:10C2100095AE060831CD0608FD62070899D10708DA
:10C22000E96F090809560A0875B70A088DDD0A087A
:10C23000DDE80A0855160B081D1C0B08000000005D
:10C2400081F0004102E000BF83F0004330B54FEAC7
:10C2500041044FEA430594EA050F08BF90EA020F34
:10C260001FBF54EA000C55EA020C7FEA645C7FEAC7
:10C27000655C00F0E2804FEA5454D4EB5555B8BFEA
:10C280006D420CDD2C4480EA020281EA030382EA5B
:10C29000000083EA010180EA020281EA0303362DED
:10C2A00088BF30BD11F0004F4FEA01314FF4801CC0
:10C2B0004CEA113102D0404261EB410113F0004FD2
:10C2C0004FEA03334CEA133302D0524263EB430389
:10C2D00094EA050F00F0A780A4F10104D5F1200E27
:10C2E0000DDB02FA0EFC22FA05F2801841F1000182
:10C2F00003FA0EF2801843FA05F359410EE0A5F156
:10C3000020050EF1200E012A03FA0EFC28BF4CF086
:10C31000020C43FA05F3C01851EBE37101F000453C
:10C3200007D54FF0000EDCF1000C7EEB00006EEB49
:10C330000101B1F5801F1BD3B1F5001F0CD34908D3
:10C340005FEA30004FEA3C0C04F101044FEA44522A
:10C3500012F5800F80F09A80BCF1004F08BF5FEAB1
:10C36000500C50F1000041EB045141EA050130BD91
:10C370005FEA4C0C404141EB0101013C28BFB1F5A3
:10C38000801FE9D291F0000F04BF01460020B1FAEE
:10C3900081F308BF2033A3F10B03B3F120020CDAC1
:10C3A0000C3208DD02F1140CC2F10C0201FA0CF09F
:10C3B00021FA02F10CE002F11402D8BFC2F1200C04
:10C3C00001FA02F120FA0CFCDCBF41EA0C019040BA
:10C3D000E41AA2BF01EB0451294330BD6FEA040403
:10C3E0001F3C1CDA0C340EDC04F11404C4F12002EE
:10C3F00020FA04F001FA02F340EA030021FA04F300
:10C4000045EA030130BDC4F10C04C4F1200220FA56
:10C4100002F001FA04F340EA0300294630BD21FA94
:10C4200004F0294630BD94F0000F83F4801306BF5A
:10C4300081F480110134013D4EE77FEA645C18BF4E
:10C440007FEA655C29D094EA050F08BF90EA020FE5
:10C4500005D054EA000C04BF1946104630BD91EADD
:10C46000030F1EBF0021002030BD5FEA545C05D1E0
:10C470004000494128BF41F0004130BD14F580041F
:10C480003CBF01F5801130BD01F0004545F0FE4193
:10C4900041F470014FF0000030BD7FEA645C1ABFC8
:10C4A000194610467FEA655C1CBF0B46024650EAFF
:10C4B000013406BF52EA033591EA030F41F400212B
:10C4C00030BD00BF90F0000F04BF0021704730B5B1
:10C4D0004FF4806404F132044FF000054FF0000186
:10C4E00050E700BF90F0000F04BF0021704730B547
:10C4F0004FF4806404F1320410F0004548BF40421C
:10C500004FF000013EE700BF42004FEAE2014FEA70
:10C5100031014FEA02701FBF12F07F4393F07F4F4B
:10C5200081F06051704732F07F4208BF704793F04E
:10C530007F4F04BF41F40021704730B54FF4607461
:10C5400001F0004521F000411CE700BF50EA010264
:10C5500008BF704730B54FF000050AE050EA01020D
:10C5600008BF704730B511F0004502D5404261EB7D
:10C5700041014FF4806404F132045FEA915C3FF4BE
:10C58000D8AE4FF003025FEADC0C18BF03325FEA5B
:10C59000DC0C18BF033202EBDC02C2F1200300FA0C
:10C5A00003FC20FA02F001FA03FE40EA0E0021FA31
:10C5B00002F11444BDE600BF70B54FF0FF0C4CF41F
:10C5C000E06C1CEA11541DBF1CEA135594EA0C0FD1
:10C5D00095EA0C0F00F0DEF82C4481EA030621EA0C
:10C5E0004C5123EA4C5350EA013518BF52EA033547
:10C5F00041F4801143F4801338D0A0FB02CE4FF0F9
:10C600000005E1FB02E506F00042E0FB03E54FF028
:10C610000006E1FB03569CF0000F18BF4EF0010E20
:10C62000A4F1FF04B6F5007F64F5407404D25FEA1C
:10C630004E0E6D4146EB060642EAC62141EA5551CF
:10C640004FEAC52040EA5E504FEACE2EB4F1FD0C11
:10C6500088BFBCF5E06F1ED8BEF1004F08BF5FEA8F
:10C66000500E50F1000041EB045170BD06F0004641
:10C6700046EA010140EA020081EA0301B4EB5C04EE
:10C68000C2BFD4EB0C0541EA045170BD41F48011E6
:10C690004FF0000E013C00F3AB8014F1360FDEBF0B
:10C6A000002001F0004170BDC4F10004203C35DAE7
:10C6B0000C341BDC04F11404C4F1200500FA05F36A
:10C6C00020FA04F001FA05F240EA020001F000420B
:10C6D00021F0004110EBD37021FA04F642EB060181
:10C6E0005EEA430E08BF20EAD37070BDC4F10C04AB
:10C6F000C4F1200500FA04F320FA05F001FA04F26F
:10C7000040EA020001F0004110EBD37041F100015A
:10C710005EEA430E08BF20EAD37070BDC4F1200565
:10C7200000FA05F24EEA020E20FA04F301FA05F2CD
:10C7300043EA020321FA04F001F0004121FA04F275
:10C7400020EA020000EBD3705EEA430E08BF20EA45
:10C75000D37070BD94F0000F0FD101F0004640007F
:10C7600041EB010111F4801F08BF013CF7D041EA01
:10C77000060195F0000F18BF704703F00046520005
:10C7800043EB030313F4801F08BF013DF7D043EAD6
:10C790000603704794EA0C0F0CEA135518BF95EA8C
:10C7A0000C0F0CD050EA410618BF52EA4306D1D113
:10C7B00081EA030101F000414FF0000070BD50EA32
:10C7C000410606BF1046194652EA430619D094EABC
:10C7D0000C0F02D150EA013613D195EA0C0F05D1A6
:10C7E00052EA03361CBF104619460AD181EA0301FA
:10C7F00001F0004141F0FE4141F470014FF00000B2
:10C8000070BD41F0FE4141F4780170BD70B54FF04C
:10C81000FF0C4CF4E06C1CEA11541DBF1CEA1355CC
:10C8200094EA0C0F95EA0C0F00F0A7F8A4EB0504AE
:10C8300081EA030E52EA03354FEA013100F08880A5
:10C840004FEA03334FF0805545EA131343EA12636E
:10C850004FEA022245EA111545EA10654FEA002623
:10C860000EF000419D4208BF964244F1FD0404F5DC
:10C87000407402D25B084FEA3202B61A65EB030538
:10C880005B084FEA32024FF480104FF4002CB6EBF5
:10C89000020E75EB030E22BFB61A754640EA0C0075
:10C8A0005B084FEA3202B6EB020E75EB030E22BFB5
:10C8B000B61A754640EA5C005B084FEA3202B6EBF6
:10C8C000020E75EB030E22BFB61A754640EA9C00B5
:10C8D0005B084FEA3202B6EB020E75EB030E22BF85
:10C8E000B61A754640EADC0055EA060E18D04FEA43
:10C8F000051545EA16754FEA06164FEAC30343EAE3
:10C9000052734FEAC2025FEA1C1CC0D111F4801FAF
:10C910000BD141EA00014FF000004FF0004CB6E7A8
:10C9200011F4801F04BF01430020B4F1FD0C88BF47
:10C93000BCF5E06F3FF6AFAEB5EB030C04BFB6EB52
:10C94000020C5FEA500C50F1000041EB045170BD45
:10C950000EF0004E4EEA113114EB5C04C2BFD4EB72
:10C960000C0541EA045170BD41F480114FF0000EF6
:10C97000013C90E645EA060E8DE60CEA135594EA72
:10C980000C0F08BF95EA0C0F3FF43BAF94EA0C0F75
:10C990000AD150EA01347FF434AF95EA0C0F7FF4EA
:10C9A00025AF104619462CE795EA0C0F06D152EA3E
:10C9B00003353FF4FDAE1046194622E750EA410622
:10C9C00018BF52EA43067FF4C5AE50EA41047FF433
:10C9D0000DAF52EA43057FF4EBAE12E74FF0FF3C98
:10C9E00006E000BF4FF0010C02E000BF4FF0010C69
:10C9F0004DF804CD4FEA410C7FEA6C5C4FEA430CE2
:10CA000018BF7FEA6C5C1BD001B050EA410C0CBF30
:10CA100052EA430C91EA030F02BF90EA020F002092
:10CA2000704710F1000F91EA030F58BF994208BFF9
:10CA300090422CBFD8176FEAE37040F001007047B6
:10CA40004FEA410C7FEA6C5C02D150EA013C07D10D
:10CA50004FEA430C7FEA6C5CD6D152EA033CD3D058
:10CA60005DF8040B704700BF8446104662468C4652
:10CA70001946634600E000BF01B5FFF7B7FF002885
:10CA800048BF10F1000F01BD4DF808EDFFF7F4FFAE
:10CA90000CBF012000205DF808FB00BF4DF808ED39
:10CAA000FFF7EAFF34BF012000205DF808FB00BF5C
:10CAB0004DF808EDFFF7E0FF94BF012000205DF87E
:10CAC00008FB00BF4DF808EDFFF7CEFF94BF012033
:10CAD00000205DF808FB00BF4DF808EDFFF7C4FF2C
:10CAE00034BF012000205DF808FB00BF4FEA410C75
:10CAF0007FEA6C5C02D150EA013C0AD14FEA430C58
:10CB00007FEA6C5C02D152EA033C02D14FF0000094
:10CB100070474FF0010070474FEA410212F50012D2
:10CB200015D211D56FF47873B3EB625212D94FEA74
:10CB3000C12343F0004343EA505311F0004F23FA5E
:10CB400002F018BF404270474FF00000704750EAB3
:10CB5000013005D111F0004008BF6FF00040704770
:10CB60004FF00000704700BF4A0011D212F50012CA
:10CB700011D20DD56FF47873B3EB62520ED44FEA35
:10CB8000C12343F0004343EA505323FA02F07047B5
:10CB90004FF00000704750EA013002D14FF0FF30F3
:10CBA00070474FF0000070474FEA4102B2F1E04396
:10CBB00024BFB3F5001CDCF1FE5C0DD901F0004C84
:10CBC0004FEAC0024CEA5070B2F1004F40EB8300D4
:10CBD00008BF20F00100704711F0804F21D113F100
:10CBE0003872BCBF01F00040704741F480114FEA39
:10CBF0005252C2F11802C2F1200C10FA0CF320FAC2
:10CC000002F018BF40F001004FEAC1234FEAD323DE
:10CC100003FA0CFC40EA0C0023FA02F34FEA430348
:10CC2000CCE77FEA625307D150EA01331EBF4FF0D1
:10CC3000FE4040F44000704701F0004040F0FE40EC
:10CC400040F40000704700BF80F0004002E000BFE9
:10CC500081F0004142001FBF5FEA410392EA030FE7
:10CC60007FEA226C7FEA236C6AD04FEA1262D2EB31
:10CC70001363C1BFD218414048404140B8BF5B4236
:10CC8000192B88BF704710F0004F40F4000020F0CF
:10CC90007F4018BF404211F0004F41F4000121F0E5
:10CCA0007F4118BF494292EA030F3FD0A2F101022F
:10CCB00041FA03FC10EB0C00C3F1200301FA03F16D
:10CCC00000F0004302D5494260EB4000B0F5000F90
:10CCD00013D3B0F1807F06D340084FEA310102F14F
:10CCE0000102FE2A51D2B1F1004F40EBC25008BF01
:10CCF00020F0010040EA03007047490040EB0000CB
:10CD0000013A28BFB0F5000FEDD2B0FA80FCACF1CB
:10CD1000080CB2EB0C0200FA0CF0AABF00EBC250F8
:10CD200052421843BCBFD0401843704792F0000FE6
:10CD300081F4000106BF80F400000132013BB5E739
:10CD40004FEA41037FEA226C18BF7FEA236C21D0AF
:10CD500092EA030F04D092F0000F08BF0846704714
:10CD600090EA010F1CBF0020704712F07F4F04D1E2
:10CD7000400028BF40F00040704712F100723CBFF5
:10CD800000F50000704700F0004343F0FE4040F41F
:10CD9000000070477FEA226216BF08467FEA2363DD
:10CDA0000146420206BF5FEA412390EA010F40F4C8
:10CDB000800070474FF0000304E000BF10F0004314
:10CDC00048BF40425FEA000C08BF704743F09643FB
:10CDD00001464FF000001CE050EA010208BF704716
:10CDE0004FF000030AE000BF50EA010208BF70479D
:10CDF00011F0004302D5404261EB41015FEA010CB2
:10CE000002BF84460146002043F0B64308BFA3F1A9
:10CE10008053A3F50003BCFA8CF2083AA3EBC2538B
:10CE200010DB01FA02FC634400FA02FCC2F12002AA
:10CE3000BCF1004F20FA02F243EB020008BF20F0E1
:10CE40000100704702F1200201FA02FCC2F1200247
:10CE500050EA4C0021FA02F243EB020008BF20EA3C
:10CE6000DC7070477BB972B90029BEBF00204FF05B
:10CE7000004106E008BF00281CBF6FF000414FF0E2
:10CE8000FF3000F007BAADF1080C6DE904CE0029BF
:10CE900009DB002B1ADB00F095F8DDF804E0DDE992
:10CEA000022304B07047404261EB4101002B1BDBC1
:10CEB00000F088F8DDF804E0DDE9022304B0404228
:10CEC00061EB4101524263EB43037047524263EB13
:10CED000430300F077F8DDF804E0DDE9022304B055
:10CEE000404261EB41017047524263EB430300F063
:10CEF00069F8DDF804E0DDE9022304B0524263EB97
:10CF00004303704753B94AB9002908BF00281CBF22
:10CF10004FF0FF314FF0FF3000F0BCB9ADF1080C1D
:10CF20006DE904CE00F04EF8DDF804E0DDE90223FF
:10CF300004B07047430803F05533C01A830803F068
:10CF4000333300F03330184400EB101000F00F3092
:10CF500000EB002000EB0040000E704707EE900A47
:10CF6000F5EEC07AF1EE10FA01D400F00BB8F1EE54
:10CF7000677A08B517EE900A00F004F8404261EBBA
:10CF8000410108BDD0B5FFF7BFFA0C4B00220646A1
:10CF90000F46FFF711FBFFF7E7FD0446FFF792FA94
:10CFA000074B0022FFF708FB02460B463046394686
:10CFB000FFF74AF9FFF7D8FD2146D0BD0000F03D4C
:10CFC0000000F0412DE9F047089D04468E46002BF5
:10CFD0004DD18A42944669D9B2FA82F252B101FA2D
:10CFE00002F3C2F1200120FA01F10CFA02FC41EA3D
:10CFF000030E94404FEA1C48210CBEFBF8F61FFAC2
:10D000008CF708FB16E341EA034306FB07F199425C
:10D010000AD91CEB030306F1FF3080F01F8199420F
:10D0200040F21C81023E63445B1AA4B2B3FBF8F0E9
:10D0300008FB103344EA034400FB07F7A7420AD970
:10D040001CEB040400F1FF3380F00A81A74240F298
:10D0500007816444023840EA0640E41B00261DB103
:10D06000D4400023C5E900433146BDE8F0878B4238
:10D0700009D9002D00F0EF800026C5E900013046F7
:10D080003146BDE8F087B3FA83F6002E4AD18B42D1
:10D0900002D3824200F2F980841A61EB030301207B
:10D0A0009E46002DE0D0C5E9004EDDE702B9FFDE67
:10D0B000B2FA82F2002A40F09280A1EB0C014FEA12
:10D0C0001C471FFA8CFE0126200CB1FBF7F307FB6F
:10D0D000131140EA01410EFB03F0884208D91CEB12
:10D0E000010103F1FF3802D2884200F2CB804346AF
:10D0F000091AA4B2B1FBF7F007FB101144EA01448E
:10D100000EFB00FEA64508D91CEB040400F1FF311C
:10D1100002D2A64500F2BB800846A4EB0E0440EA0A
:10D1200003409CE7C6F12007B34022FA07FC4CEA13
:10D13000030C20FA07F401FA06F31C43F9404FEA06
:10D140001C4900FA06F3B1FBF9F8200C1FFA8CFE1B
:10D1500009FB181140EA014108FB0EF0884202FA6F
:10D1600006F20BD91CEB010108F1FF3A80F0888030
:10D17000884240F28580A8F102086144091AA4B2ED
:10D18000B1FBF9F009FB101144EA014100FB0EFE6E
:10D190008E4508D91CEB010100F1FF346CD28E459D
:10D1A0006AD90238614440EA0840A0FB0294A1EB2E
:10D1B0000E01A142C846A64656D353D05DB1B3EB8B
:10D1C000080261EB0E0101FA07F722FA06F3F140BB
:10D1D0001F43C5E9007100263146BDE8F087C2F162
:10D1E0002003D8400CFA02FC21FA03F391400143DA
:10D1F0004FEA1C471FFA8CFEB3FBF7F007FB103613
:10D200000B0C43EA064300FB0EF69E4204FA02F4BE
:10D2100008D91CEB030300F1FF382FD29E422DD911
:10D22000023863449B1B89B2B3FBF7F607FB163346
:10D2300041EA034106FB0EF38B4208D91CEB0101C6
:10D2400006F1FF3816D28B4214D9023E6144C91A46
:10D2500046EA004638E72E46284605E70646E3E656
:10D260001846F8E64B45A9D2B9EB020864EB0C0E60
:10D270000138A3E74646EAE7204694E74046D1E76F
:10D28000D0467BE7023B614432E7304609E764441D
:10D29000023842E7704700BF02E000F000F8FEE706
:10D2A00072B6374880F30888364880F309883648D4
:10D2B0003649086040F20000CCF200004EF63471AE
:10D2C000CEF200010860BFF34F8FBFF36F8F40F2C3
:10D2D0000000C0F2F0004EF68851CEF20001086066
:10D2E000BFF34F8FBFF36F8F4FF00000E1EE100AD6
:10D2F0004EF63C71CEF200010860062080F31488DF
:10D30000BFF36F8FA9F0D6FEAAF020FE4FF0553084
:10D310001F491B4A91423CBF41F8040BFAE71D49E3
:10D32000184A91423CBF41F8040BFAE71A491B4ADC
:10D330001B4B9A423EBF51F8040B42F8040BF8E72E
:10D3400000201849184A91423CBF41F8040BFAE703
:10D35000A9F0B4FEAAF04EFE144C154DAC4203DA0F
:10D3600054F8041B8847F9E702F0C0F8114C124D3D
:10D37000AC4203DA54F8041B8847F9E7A9F09CBED5
:10D38000000600200022002000C0000808ED00E098
:10D39000000000200006002090140E08002200204B
:10D3A000AC2B0020B02B0020904C0120E0C10008E5
:10D3B0003CC200083CC200083CC200082DE9F04F06
:10D3C0002DED108AC1F80CD0C3689D46BDEC108AC3
:10D3D000BDE8F08F002383F311882846A047002082
:10D3E000A8F060FEFEE7A8F0CDFC00DFFEE700003D
:10D3F00001F0FF01102A2BDB10F0070F08D010F806
:10D40000013B013A8B422DD010F0070F42B3F6D109
:10D41000F0B441EA012141EA014122F007047FF022
:10D4200000070023F0E80256083C85EA010586EA79
:10D43000010685FA47F5A3FA87F586FA47F6A5FAB5
:10D4400087F68EB9EED1F0BC01F0FF0102F00702C1
:10D4500032B110F8013B013A83EA010313B1F8D16C
:10D460000020704701387047002D06BF354603384D
:10D47000073815F0010F07D1013015F4807F02BF86
:10D48000013015F4C03F0130F0BC0138704700BFD7
:10D4900010F8012B11F8013B012A28BF9A42F7D05E
:10D4A000D01A7047034613F8012B002AFBD1181A33
:10D4B0000138704738B50022002304460D46FFF7B7
:10D4C000EDFA28B920462946BDE8384000F00AB8F0
:10D4D000204605F1004100F005F8404261EB4101B2
:10D4E00038BD00BFD0B50C4B002206460F46FFF7F3
:10D4F00063F8FFF739FB0446FEF7E4FF074B002211
:10D50000FFF75AF802460B4630463946FEF79CFEB6
:10D51000FFF72AFB2146D0BD0000F03D0000F0419E
:10D52000036800221B6818477FB503914021054618
:10D5300079F012FC039A18B90124204604B070BD9A
:10D54000134E039296F98A33002BF5D05DF0D8FE86
:10D55000437A039A53B95DF0D3FE847A039A2CB9C7
:10D560000C4B4021284679F0FFFBE6E7D6F8D83C83
:10D57000B6F98C13B3F906309942DDDD064B009302
:10D580004021064B284679F0EFFB0024D5E700BF89
:10D59000B84B002070F60B088FF60B087DF60B08D1
:10D5A000F0B50D469DB02021044679F0D5FB00284A
:10D5B00000F09D804F4E96F98A33ABB1D6F8D82C47
:10D5C000B6F98C33B2F90A1003F10A02914203DD75
:10D5D00040F28D32934207DC474B2A4620212046F9
:10D5E00079F0C2FB002080E096F97933022B05D157
:10D5F000424B2A462021204679F0B6FBB6F84C3340
:10D60000A3F57A739BB241F6583293420DD83C4F42
:10D6100096EDEE7AD7F8403BD3ED097AB4EEE77A8F
:10D62000F1EE10FA03DD374BD7E7374BD5E796ED30
:10D63000EF7AD3ED0B7AB4EEE77AF1EE10FAF2DC82
:10D64000B6F98633002B01DC304BC6E796F8182478
:10D650000D2A06D80123934013F4215F01D02C4BEF
:10D66000BBE72C480EF0FAFD012806D1D7F84C0B89
:10D6700080F07EFB98B101281AD00021602204A816
:10D680000391ADF0CDFC2449D7F8480B642303AADD
:10D690007FF090FF00BB03AB0093204B02E0204BD8
:10D6A0000093204B2A462021204679F05DFB99E724
:10D6B00096F8EC3C73B11C4819214BF079FB48B14A
:10D6C0001948D6F8646319214BF098FB8642D4DDE3
:10D6D000164BE5E7164BE3E71649D7F8400B6423F2
:10D6E00003AA7CF027FE0028D5D01DB0F0BD012094
:10D6F000FBE700BFB84B002098F60B08ABF60B0811
:10D70000B86B0020E3F60B08D3F60B08FDF60B0808
:10D7100012F70B08E87E00208CF70B0890F70B0837
:10D7200057F70B0832F70B08B83A002076F70B08CA
:10D7300067F70B08A2F70B0807B5044881F070FEE5
:10D7400000F0010003B05DF804FB00BFDC760020B0
:10D750002DE9F043DFF844910446D9F89C000368B2
:10D76000A5B01B690D469847804614F031FB002197
:10D77000074660220CA80B91ADF052FC64230BAA63
:10D780004146384613F026FE064648B93A4A0BABE6
:10D790002946204679F0F0FC304625B0BDE8F083FC
:10D7A000A9F55B6067F028F8B8F1000F03D194F990
:10D7B0001E30012B0AD1314811F00CFB80B9304AE0
:10D7C0002946204679F0D8FC0026E5E710F0060F40
:10D7D000E2D0A9F5405011F0FDFA08B9294AEFE767
:10D7E00003A9384613F02CFC28B19DF80D305B06D8
:10D7F00001D5254AE4E7DFF8A880D8EDEA7AF5EE0E
:10D80000C07AF1EE10FA4FF00003C5DD08930993DA
:10D810000A930DF1200907AB019305AA06AB04A9F1
:10D82000CDF80090384613F0E9FF48462EF0D8FFB7
:10D83000D8EDEA7AB4EEE70AF1EE10FA01DB134A0A
:10D84000BEE79DED057AF4EEC77AF1EE10FA01D845
:10D850000F4AB5E79DED047AF4EEC77AF1EE10FABF
:10D8600001D80C4AACE79DED067AF4EEC77AF1EEEA
:10D8700010FA91D8084AA3E7A8F70B08B82B0020A4
:10D88000B1F70B08C8F70B08EEF70B08FCF70B080D
:10D8900011F80B0827F80B083DF80B08B85B0020BF
:10D8A000B84B002008B5064B93F8B5309B0704D55C
:10D8B000044A79F061FC002008BD0120FCE700BFAC
:10D8C000B85B002054F80B0870B50C4C0546D4F832
:10D8D0009C0003685B690E46984710B101242046FE
:10D8E00070BDA4F5405011F087FA04460028F5D128
:10D8F000034A3146284679F03FFCF0E7B85B002048
:10D9000064F80B082DE9F046464ED6F8C03093F87F
:10D91000CB509BB081468A4665B9434B1B68986AD9
:10D9200003685B6B9847044640B9404A51464846F5
:10D9300079F022FC28461BB0BDE8F0865DF0E0FCE3
:10D9400020215EF095FC58B15DF0DAFC1F215EF0FD
:10D950008FFC88B3364A5146484679F00DFC0024C6
:10D9600096F8923003F01403142B05D1314A514636
:10D97000484679F001FC0024514648467AF0A0FA66
:10D98000002188424FF0600202A808BF0C460191B6
:10D99000ADF046FBD6F8C000036801AA1B686421FD
:10D9A0009847054680B9244A01AB5146484679F06C
:10D9B000E3FB2C462546BDE75DF0A2FCA5215EF009
:10D9C00057FC0028C6D1CBE7002CF3D0D9F808309B
:10D9D0003BB9D9F8003051465B6B4846984704463E
:10D9E000E8E751464846FFF7DBFD51460746484603
:10D9F000FFF758FF3840C4B251464846FFF794FD40
:10DA0000514604404846FFF75FFF514604404846F0
:10DA100079F0DAFB5146044048467AF069FA04404E
:10DA2000C8E700BFB85B0020E880002078F80B084A
:10DA30008FF80B08A9F80B08C1F80B0808B5FFF719
:10DA400061FF054A92F8901060F3041182F890107B
:10DA5000024A907108BD00BFB85B0020A58200207B
:10DA6000F7B505460F4679F0B3F9044678B10221BF
:10DA7000284679F071F9064648B1154881F0D0FC86
:10DA8000C205C0F30723C0F3002403D53446204663
:10DA900003B0F0BD9B07F9D50D4881F0CFFC0D4BCD
:10DAA00003F52F63D3ED007AF8EEE77A30EE670ADC
:10DAB000DFED097AB0EEC00AB4EEE70AF1EE10FA33
:10DAC000E4DD064B3A460221284679F04DF9DEE7BF
:10DAD000DC760020B86B00200000C842CCF80B08B0
:10DAE000F8B504460F4679F025FC1021054620467E
:10DAF00079F032F958B12046FFF71EFE064630B9DC
:10DB0000044B3A461021204679F02EF93546284636
:10DB1000F8BD00BFE0F80B0870B505460E4679F079
:10DB2000BFF8044678B18021284679F015F950B144
:10DB3000074B93F8153643B1064B324680212846F1
:10DB400079F012F90024204670BD0446FBE700BFBF
:10DB5000B85B0020F4F80B0838B50D4D0446D5F835
:10DB60004C0B80F005F9012810D0D5F84C0B80F053
:10DB7000FFF8022804D02046BDE8384079F092B87A
:10DB800004480EF06BFB0128F5D138BD0020FCE7FE
:10DB9000B86B0020E87E0020F0B5134C04F500536C
:10DBA00085B0D3F8D02C0092D3F8D42C0192D3F8BE
:10DBB000D82C0292D3F8DC3C03936A4606460F4603
:10DBC0007AF030F939460546304679F027F904F500
:10DBD0004054284094F8903060F3C303C3F3C0006E
:10DBE00084F8903005B0F0BDB82B00202DE9F84343
:10DBF00006462748DFF8A890DFF8A8800F4666F0B1
:10DC0000FBFD0446D9F89C0003681B69984705464C
:10DC100030B914F0060F03D1D9F8D030022B09D156
:10DC20003946304679F0CCF9054618B9002488F811
:10DC300007400AE039463046FFF78AFD04460028CF
:10DC4000F4D02DB9012388F807302046BDE8F883C9
:10DC50000821304679F080F80028F3D00D4821F0F3
:10DC600099FF0028EED00C4B93F8E423B02101FB80
:10DC7000023203F50053B2F8EE21B3F97A339A4237
:10DC8000E0DD064B3A460821304679F06DF8CDE7E5
:10DC9000084E0020D82C0020B82B002008F90B08D3
:10DCA000B85B0020A58200202DE9F3410E46054611
:10DCB00014F08EF8804613F085F9044640B9514AB5
:10DCC0000121284679F058FA204602B0BDE8F081DB
:10DCD0004D4FD7F89C00036831469B69984704462E
:10DCE00058B9D7F89C0003681B6C9847474A03460D
:10DCF0000121284679F040FAE6E7AB68002BE3D033
:10DD00001021284679F028F820B3D8ED937A98EDC1
:10DD1000920A20EE270AAAF021FFDFED3D7AA7F54F
:10DD2000805320EE270AB3F94C33DFED3A7A20EE28
:10DD3000270A07EE903AF8EEE77AB4EEE70AF1EE3A
:10DD400010FA07DD344B01221021284679F00CF837
:10DD50000024B9E74021284678F0FEFF38B3012EB1
:10DD60001ED0232E1CD0042E1AD02C4CD4F8D83C14
:10DD7000B3F9083000EE103AA4F50050B8EEC00A2E
:10DD800000F0BCFBB5EEC00AF1EE10FA1DDD244B2D
:10DD900000930122234B4021284678F0E5FFD7E786
:10DDA000D7F89C000368DB6B98470028DDD01E4B3A
:10DDB0001B68D86A0368DB6998470128014619D1B6
:10DDC0001A4A284679F0D8F9C2E7D7F89C000368C8
:10DDD0005B69984730B1D4F8D83CB3F90830002BD0
:10DDE000E5DDD4E7D7F89C0003681B6898470B284B
:10DDF000DDD1F0E73146284602B0BDE8F04179F0C8
:10DE000061BD00BF18F90B08B85B002029F90B08A9
:10DE1000E02E65420000C8423DF90B08B84B0020D7
:10DE20008FF60B0845F90B08E880002051F90B0824
:10DE300070B505460E46FFF78BFC084B0446D871BB
:10DE400031462846FFF740FD31460028284608BFE6
:10DE5000002479F0CFFE204070BD00BFA5820020D5
:10DE60002DE9F0414E4F3B78002B40F096804D4C11
:10DE7000D4F8C05095F8CB5001263E701DB13B70D0
:10DE80002846BDE8F0817AF0DBF8054630B9464A0D
:10DE90003870137843F001031370F1E753F0E4F89E
:10DEA000314652F049FAA4F5405006F097FC3F4B3A
:10DEB0001E710B2646F03AFD013E46F0D5FC16F0E9
:10DEC000FF06F7D13A4800F06FFF13F081FFD0F85A
:10DED0000022C4F8E82090F87C32DA074DD413F021
:10DEE000EFFA53F0C1F83C2152F0FAFF0023C4F8D6
:10DEF000A83000212E482F4E00F0DCFF2C4810F0F7
:10DF000069FF01462C4885F0FDF92C4B1B68D86A47
:10DF1000036801211B689847D4F8C00003689B6A16
:10DF200098470121D4F8C00082F034FA53F09CF8ED
:10DF30008046D4F89C0003681B68984796F80C2329
:10DF40000146404652F0B8FBA6F5005006F038FCFA
:10DF500050F0FCFA4FF038FE00233B7089F010FCC3
:10DF6000B4F8923006F5005623F4087343F020030A
:10DF7000C6F8580BA4F8923082E79B07B9D4314613
:10DF80000B4804F0D7FC0E4881F058FADFED0D7A0B
:10DF900020EE270A84ED2A0AABE7002570E700BFD0
:10DFA000B02B0020B85B0020C4820020A582002096
:10DFB000B82B0020B84B00202C570020E880002010
:10DFC000DC7600200AD7233C2DE9F043374DD5F805
:10DFD000C03093F8CB3087B0002B64D062B10129F8
:10DFE00001D0232908D195F99030002B04DB0024BF
:10DFF000204607B0BDE8F0837AF0CEF8044600284A
:10E00000F5D013F0E5FE07461AF0F6FB80463846D9
:10E0100012F0EAFCD8B198F92430022B17D100266F
:10E020004FF00009F1B203AA38460191CDF80C90E7
:10E03000CDF81090CDF8149013F068F8019918B14C
:10E0400003AA40461AF088F80136032EEAD1184890
:10E05000012106F031FE1648012106F061FD002184
:10E06000D5F8C00082F096F9124831F09DF852F0D0
:10E07000FBFF002152F060F90F4B1B68D86A036860
:10E0800000211B68984795F89230D5F89C100B48F2
:10E090006FF3451385F892300B1A594259413C30C1
:10E0A00087F094FDA4E70124A2E700BFB85B00203D
:10E0B000B82B00201C790020E8800020B87A0020CE
:10E0C00010B5064CD4F89C0003685B6A984718B1F9
:10E0D000D4F8C03093F8CB0010BD00BFB85B00206F
:10E0E00030B52DED028B89B00C46B0EE408AFFF7BB
:10E0F000E7FF0546002838D0B4EE488AF1EE10FA62
:10E100007CBFDFED1C8ADFED1C7A226863689FED1F
:10E110001A0A68BFDFED198A029278BF68EE288A72
:10E1200002A878BF68EEA78AD4ED027A0393F1EED5
:10E13000677ACDED047A2DF055FFB4EE488A0022BF
:10E140000123F1EE10FACDE900238DED050ACDEDA6
:10E15000060A9FED0A0A0A488DED071AF0EE680AD2
:10E1600068BF134605A90CF057F9284609B0BDEC65
:10E17000028B30BDE02E65420000C8420000000066
:10E180008C7D002007B50191FFF79AFF30B101990E
:10E19000044803B05DF804EB00F0F0BA03B05DF89A
:10E1A00004FB00BFB82B0020014866F0B1BC00BFE3
:10E1B000084E002008B500F5405090F89030C3F3A9
:10E1C00040128A420BD061F3451380F8903031B190
:10E1D00052F04AFFBDE808400F2152F081BE08BD51
:10E1E00070B500F540560546D6F8D0308B420C4647
:10E1F00012D0012911D0022916D059B952F034FF9A
:10E200001B2152F06DFE0D4A05F5395006213430C0
:10E2100054F026FFC6F8D04070BD52F025FF1A21F9
:10E2200052F05EFE064AEFE7012100F043FE52F095
:10E230001BFF1D2152F054FE024AE5E7BCF90B0812
:10E24000D1F90B08CCF90B0810B500F540520C467B
:10E2500092F8B53003F00101A14209D064F3000344
:10E2600082F8B530DB0704D405F09AFE024B9C72AD
:10E2700010BD06F069F8F9E7A582002000F54050CE
:10E2800090F8B53061F3410380F8B530014B197354
:10E29000704700BFA582002010B504465DF030F83D
:10E2A00020215DF0E5FF04F54053003893F89220FB
:10E2B00018BF012060F3820283F8922010BD000095
:10E2C00010B5044650F042F904F54052436FD2F8BD
:10E2D000C02004F58044D360D4F8402B9366D4F872
:10E2E000482BC2F8FC32D4F8400B03685B6D9847AA
:10E2F000D4F8400B0368BDE810409B6D1847000040
:10E3000070B52DED028B00F540550446D5F8C030B0
:10E3100093F8CB30002B72D095F99030002B6EDB48
:10E3200000F5804696F8883C002B68D1D5F89C0013
:10E3300003685B699847002861D1324BD3F89C0091
:10E3400003681B6898470B2859D0D6F8483B9FEDC7
:10E350002E7AD3EDDB7AF0EEE77AF4EEC77AF1EEBF
:10E3600010FA4CD5D5F8C000443054F08FFA03466B
:10E37000DFED260A93ED000A9F20B7EE001A2AF07F
:10E3800023FCB5EEC00AF1EE10FA38DD04F5964034
:10E39000243081F05FF8DFED1E7AB0EEC00AB4EEF3
:10E3A000E70AF1EE10FA2AD504F58054D6F8400BAE
:10E3B000D4F8503607EE903A0368D3F89830B8EEA8
:10E3C000E78A984738EE400ADFED127AB0EEC00ACD
:10E3D000B4EEE70AF1EE10FA11D5D4F8543640F253
:10E3E000E63203F2F313934209D8BDEC028BD5F861
:10E3F000C0009FED090ABDE8704083F0B5BABDECDE
:10E40000028B70BDB85B00200000003400000000EB
:10E41000000070420000FA430AD7233C08B500F51B
:10E420004050D0F8C00003681B699847F6EE007AA8
:10E4300020EE270AB5EEC00AF1EE10FA48BF9FEDB4
:10E44000010A08BD0000000038B52DED028B00F573
:10E4500080450446D5F8403BDFED110A93ED370ABD
:10E4600004F540547120B7EE001A2AF0ADFBD4F841
:10E47000C000D5F8485B03681B69B0EE408A984736
:10E4800038EE400ABDEC028BDFED067A05F5057526
:10E49000284620EE270ABDE8384070F063BD00BF73
:10E4A0000000000000007A4400F5A250D0ED9A5A16
:10E4B000D2ED007AD0ED9D6A91ED006A26EEE77A02
:10E4C00067EEA57AA6EE257AE6EE267A81ED007A49
:10E4D000C2ED007A7047000000F50050B0F9243C0E
:10E4E00033B9B0F986030028B8BF404280B2704704
:10E4F00083EAE370A0EBE370F8E7000070B52DED60
:10E50000028B00F5405382B093F8B51011F001066C
:10E51000044605D09FED2E0A02B0BDEC028B70BD03
:10E520008DED010A5CF0ECFE037F002BF2D0DFEDF5
:10E53000298ADFED270A9DED010AB0EE681A4E2008
:10E540002AF042FB04F500554FF4C8723146B5F984
:10E550008E03B0EE408A2AF075FBA5F88E032046A4
:10E5600010F0E2F9B5F98E3307EE900AB8EEE77ACB
:10E5700007EE903AF8EEE77A77EE676AB4EEE68A4D
:10E58000F1EE10FA0DD52046FFF7A6FF07EE900A30
:10E5900038EE668AB8EEE70A20EE088A88EE260A88
:10E5A000BAE777EE877AB4EEE78AF1EE10FAB1DDDA
:10E5B000B5F9863300EE103A38EE678AB8EEC00A35
:10E5C00078EEE77A20EE088A88EE270AA4E700BFF3
:10E5D0000000000000007A440020704700207047CF
:10E5E0007047000000F50E501C307047004870471F
:10E5F00064290C0800F54050D0F89C0003681B68A3
:10E6000018470000034808602F21117008221A6083
:10E61000704700BF68FD0B0800F54050D0F89C0023
:10E620000368DB6C1847000000F54050D0F89C00F0
:10E6300003689B6C1847000000F5405300F59A40B2
:10E64000D3F89C3028301B1A5842584170470000BC
:10E6500010B500F540500C46D0F89C000368DB6D07
:10E66000984707EE900A9FED057AF8EE677A012049
:10E6700067EE877AC4ED007A10BD00BF0AD7233C4D
:10E6800010B500F540500C46D0F89C0003689B6D17
:10E69000984707EE900A9FED057AF8EEE77A012099
:10E6A00067EE877AC4ED007A10BD00BF0AD7233C1D
:10E6B00010B500F540500C46D0F89C0003681B6E66
:10E6C0009847DFED047A20EE270A012084ED000A46
:10E6D00010BD00BF0AD7233C5FF054BA63F0F8B90D
:10E6E0005EF0F6BD4FF07CBE27F0D2BE51F08ABF7F
:10E6F00017F064B95CF056BA5AF006BC0FF0ACBD26
:10E7000010F00ABA06F010BD11F01CBA05F09CBC5E
:10E7100005F0E8B905F00EB960F0B4BF0EF03CBCEE
:10E72000FFF7EEBD0FF0DCBE10F04EB903F07AB883
:10E730000FF060BE0FF0D8BD5CF030BD22F0C8BC59
:10E7400006F0B8B802F03EBC10F05CB906F0A2BC0E
:10E7500004F0DCB806F0FCBD05F07EB906F05AB94D
:10E760000FF006BDFFF7ACBD28F084BA05F06ABE15
:10E7700009F0AEBE09F0A8BD09F03CBD1FB500F51B
:10E7800040530446D3F89C00039103685B6A9847A2
:10E7900060B1DFED070A0399002304F5A34000935D
:10E7A000B0EE600A1A4654300BF08CFC04B010BD79
:10E7B0000000000010B52DED028B00F5405304461B
:10E7C000D3F89C0003685B6AB0EE408A984720B992
:10E7D0000024BDEC028B204610BD9FED080A04F515
:10E7E000A34028EE000A54300AF036FF0446002801
:10E7F000EED003480121FFF7DDFCEAE70000C84244
:10E80000B82B00200A4A92F99020002A0B4605DA1C
:10E8100000228A604A600A600120704700F580404B
:10E82000D0F8402B783207CA83E80700F4E700BF2E
:10E83000B85B002070B5224B036000F50055214BFA
:10E84000C5F8743E00F540530446586A08B119F003
:10E850000BFA1D4B236095F834303BB92D6B2DB16D
:10E86000284626F0DBFB284619F0FAF904F59B5000
:10E8700077F0A6FD04F5935008305EF05DFF04F6D6
:10E88000B46504F65466B54204D0183D284626F017
:10E890001BF8F8E70D4BC4F8983804F6F81053F05D
:10E8A000D1FC04F6CC1053F0CDFC04F62C1053F040
:10E8B000C9FC04F5106053F0C5FC204670BD00BFD4
:10E8C00024010C0890060D086CE70C082CAF0C080E
:10E8D00038B5474B044640F8043B5FF073FA04F147
:10E8E000100016F00DFD04F168004FF007FB04F571
:10E8F000907021F077F804F5866015F00DFB04F2B6
:10E90000545019F0B3F904F6980027F007FC04F509
:10E9100063605FF035F804F570604AF06FF904F554
:10E920008D50103051F068FC04F5935008305EF0C3
:10E93000EBFE04F59550043017F0DEFF04F59B5014
:10E9400077F02AFD04F59B501C304FF099FE04F53A
:10E950009E50103060F0E0FB04F580530025254AFE
:10E9600083F8F45304F5A05004F59F531433043096
:10E97000136045F0EDFD04F5A2502946183011F062
:10E9800019FD04F5D65070F0ABFB04F5F6500430D9
:10E9900074F048FD04F5FE501C3076F057FE04F587
:10E9A000015077F08DFA04F50250183011F004FB95
:10E9B00004F50750383071F049F804F5095010306B
:10E9C00065F0BEFD04F5005304F50C5083F80C53BC
:10E9D000094D243078F0B4F82B6813B1074888F05B
:10E9E0009DFE2046064948F0F1FE2C60204638BDC9
:10E9F0006CE70C081C8C002080830020E0F90B08D9
:10EA000094E60C0810B50FF003FF5CF079FC036886
:10EA1000BDE810405B681847FFF7F4BF10B5044627
:10EA200006F096F8204610F0FFF9204603F0BCFDF2
:10EA30002046BDE8104003F01FBF0000FFF7EEBF07
:10EA400070B500F543552C350446284616F032FBC8
:10EA500019F0D2FE90F9213093B390F840337BB394
:10EA600004F5405304F25456D3F8C000443053F038
:10EA70000DFF0346DFED130A93ED000A9F20B7EE6A
:10EA8000001A2AF0A1F894F98835012B284608BF0E
:10EA900086ED0E0A002116F0D3F8DFED0B7A04F2B2
:10EAA000AC7494ED287A20EE270ADFED087AA7EE01
:10EAB000270A304684ED280ABDE8704019F0ACBD45
:10EAC00070BD00BF00000000CDCCCC3D6666663F47
:10EAD000FFF7B6BF10B50121044610F0E1F960B1AF
:10EAE000114BD3F89C0003689B6A984728B92046CD
:10EAF00002F06EF9204602F07BF94FF40011204637
:10EB000010F0CEF918B129F0EBFA27F00FFA4FF414
:10EB10008021204610F0C4F928B129F0E1FABDE8BF
:10EB2000104027F007B910BDB85B0020FFF7D2BF37
:10EB30007FB500F580460446D6F8400B9FED550A98
:10EB40006C302DF04FFA04F5A25001A918308DED6C
:10EB5000010ACDED020A8DED031A11F0D7FA022158
:10EB6000204610F09DF970B10121204610F098F96F
:10EB700048B9494BD3F89C0003689B6A984710B981
:10EB8000204602F025F90121204610F089F948B904
:10EB9000414BD3F89C0003689B6A984710B9204604
:10EBA00002F026F90121204610F07AF910B920462A
:10EBB00002F078F94FF40031204610F071F930B1CD
:10EBC00004F54053D3F8C00003685B6C98474021BC
:10EBD000204610F065F968B104F58D5510352846CA
:10EBE00050F0E0FE04F5805393F9683213B12846E3
:10EBF00051F01AF84FF48061204610F051F920B11D
:10EC000004F58D50103050F067FF2021204610F0A1
:10EC100047F958B104F54055D5F89C0003681B69C5
:10EC20009847C0B1D6F8480B7DF000FC8021204603
:10EC300010F036F9E0B129F053FA27F09FF81021CF
:10EC4000204610F02DF910B3D6F8400B04B0BDE803
:10EC500070407AF031B920460CF0EEF80028E1D18E
:10EC6000D5F89C0003685B6998470028DAD0DDE797
:10EC70004FF48021204610F013F90028DBD14FF427
:10EC80000021204610F00CF90028D4D1D7E704B0B9
:10EC900070BD00BFE02E6542B85B0020FFF748BFA3
:10ECA00010B50121044610F0FBF810B1204602F027
:10ECB000F9F88021204610F0F3F858B14FF4802184
:10ECC000204610F0EDF828B929F00AFABDE8104006
:10ECD00027F030B810BD0000FFF7E2BF10B50446C2
:10ECE00005F084FC204605F0E3FA204605F0C4FC5C
:10ECF000204610F097FF2046BDE8104003F030BCDE
:10ED0000FFF7ECBF70B54FF6FF71044610F0C8F87E
:10ED100004F5405528B1D5F890200721204602F08F
:10ED2000F3F8D5F8C03093F8CB308BB92046FFF715
:10ED3000B3FAD5F8C00004F50053026893F818142C
:10ED4000166A93F8A223B047D5F8C00082F0D8FD28
:10ED50005DF0E8FF5DF074FD204610F061FF95F86E
:10ED600090300F4A04F58044DB43D4F8405BC3F392
:10ED7000C01353712B681E6F4FF0E8FB4FF050F833
:10ED80002846B047D4F8484B4FF0E0FB04F5057433
:10ED90004FF046F82046BDE870406FF049BF00BF15
:10EDA000A5820020FFF7AEBF70B500F5805606F5CE
:10EDB0008B6300F54054D3F85022C4F8D420D3F824
:10EDC0005C32C4F8D8300546D6F8580600F58C40B9
:10EDD000503029F0CDFED4F8D430C4F8E030D4F867
:10EDE000D830C4F8DC00C4F8E4304FF6FF71284690
:10EDF00010F056F838B1D6F8582628460921BDE853
:10EE0000704002F057B870BD30B500F54053D3F8EC
:10EE1000D040002C4CD093F89120D10748D56FF307
:10EE2000000283F8912000F50052012CD2F8D01C8A
:10EE3000D2F8D45CB1F908400BBFD3ED365AD3ED0C
:10EE4000395AD3ED357AD3ED387A07EE104AB5F951
:10EE5000084006EE904A0CBFF8EEE66AF8EEE66A65
:10EE6000B8EEC77A25EEE66A00F5A250A7EE276A4B
:10EE700067EEA67AD0ED9A6AE7EE257A90ED9D7A54
:10EE800027EE877AA6EE267ABDEEC77A17EE103AFD
:10EE90000B8190ED9A7AD2F8D43C67EE877A90EDA8
:10EEA0009D7AE6EE477AFDEEE77A17EE902A1A8110
:10EEB00030BD000038B505462DED028B00F54054FD
:10EEC00071B128460FF02CFBD4F8DC301B1A03F28A
:10EED000F31340F2E63293420CD8BDEC028B38BDFE
:10EEE000D4F8D030022BF8D10FF0FEFAB0F57A7FCB
:10EEF000E7D2F2E7C4F8DC0000F58C405030642320
:10EF000090FBF3F308EE103ADFED097AB8EEC88A09
:10EF100028EE278AB0EE480AA9F066FC84ED380A8C
:10EF2000B0EE480AA9F0B6FD84ED390AD5E700BF76
:10EF300035FA8E3C00F5A2500121183012F0BABE0D
:10EF4000FFF7F8BF10B504460FF0F4FC102120467F
:10EF50000FF0A6FF70B1204601F092FE4FF40011B1
:10EF600020460FF09DFF28B929F0BAF8BDE81040FF
:10EF700026F0DCBF10BD0000FFF7E4BFF8B5044683
:10EF8000254606F00DF9224B45F83C3B214BA46584
:10EF9000C4E91734204BC4E91934204BE36604F16B
:10EFA000800018F0F5FA04F19C0018F0F1FA04F171
:10EFB000B80018F0EDFA4FF6FF76194BC4F8CC30D4
:10EFC000A4F8D06004F1D40018F0E2FA4FF0FF3753
:10EFD000144B1549C4F8307128461D6048F0F6FB03
:10EFE000A4F87870A4F8946004F5A27018F0D0FA30
:10EFF00004F5B07018F0CCFA04F5BE7018F0C8FA39
:10F00000002384F89031C4F8B4312046F8BD00BF25
:10F01000C8540C0871E7000875E7000879E7000894
:10F020000000FFFF74820020ECBC0C0810B5044601
:10F0300006F0B6F80A4B23600123A38704F14000D1
:10F0400018F0A6FA04F1500018F0A2FA04F16000DA
:10F0500018F09EFA04F1700018F09AFA204610BDDC
:10F06000705C0C082DE9F043044689B0FFF730FCD2
:10F07000A04B236004F50F50043004F5005502F056
:10F080007FF804F50E53103304F53357C5F8E43C0C
:10F09000062385F8E83C4FF07C5805A907F13400B9
:10F0A000CDF8148053F054FC07F14C0087F032FD8A
:10F0B00004F596460023243604F5345785F8243D9C
:10F0C000192304A985F8303DC5F82C6D07F13C00E3
:10F0D000CDF8108053F03CFC07F1540087F01AFD86
:10F0E0004FF00108182304F5365004F5375785F81A
:10F0F000783D343785F86C8DC5F8746D0C305DF053
:10F1000015FF384677F0D8FD06AE7B4BC5F8F43DC9
:10F110003146381D8DF8188049F076F904F53850DD
:10F120002C3077F0B3FD754B754FC5F82C3E04F5C8
:10F13000395031460430069753F00AFC04F5395033
:10F1400031461030069753F003FC04F53950314630
:10F150001C3004F53959069709F1340953F0F8FBCE
:10F16000684BC5F8743E09F1080087F0D3FC04F53C
:10F170003A5704F53C58203708F10408384614374C
:10F1800058F0BAF84745F9D104F540580723C8F8B4
:10F1900028300023A8F82C304FF4CB7018F05EFD17
:10F1A000C8F824004046303087F0B4FC04F54150E4
:10F1B000343087F0AFFC544B1A680AB9C3F800909A
:10F1C00004F5A747514BC5F8743E3C3704F542504F
:10F1D000C8F89C70203078F0FFFF4D4B07934FF03C
:10F1E0007E554C4BC8F8D450C8F8E05006940093B4
:10F1F00004F5435096E80C004FF400712C3015F0E4
:10F20000D7FB04F55850183069F026F904F59540FD
:10F2100003A97430039553F0C1FB04F5964003A98C
:10F220000830039553F094FB04F5964004F58045AF
:10F23000143018F0ADF905F6243300261E605E6028
:10F240009E6005F5336304F596401E605E609E6027
:10F2500004F5A2531833C5F83C3B002385F85D3B09
:10F260004FF40041603016F02FF904F597406030FC
:10F2700067F080FA04F598401C3049F0FBF9264B02
:10F28000C5F81C3C04F59840244B2549303004F562
:10F290009848186008F1500848F098FAFF2385F85C
:10F2A000603C85F8683C1F49404648F08FFA1E4A8A
:10F2B000136813B11D4888F031FA1D491D48C2F882
:10F2C000008004F59842783208604FF0140E1FFA5F
:10F2D00083FC0EFB0C010133097C0029F7D1164B8E
:10F2E000A3F800C0154BD3F80080B8F1000F29D067
:10F2F0001348E0E724010C0868F90B08A8F90B088B
:10F300000000A04090060D089C860020A4010C0877
:10F310006DE7000814010C08B8F90B08208C0020D8
:10F3200018130D089C970D08B08C0020F4F90B08F9
:10F330004083002058430C083E830020FC820020BC
:10F3400015FA0B0804F599401A6003A9564B03936C
:10F350000C3053F0FDFA04F599402C3005F020FFF5
:10F36000524BC5F8AC3C04F599406C3005F018FFE1
:10F370004F4BC5F8EC3C04F59A4004F59E49283003
:10F38000FFF7FCFD484605F00BFF4A4BC5F8003F70
:10F3900009F13C0085F0A2F8474BC5F83C3F04F565
:10F3A000A14004F5A045403005F0FAFE434BC5F8F6
:10F3B000C03004F5A240043005F0F2FE404BC5F821
:10F3C000043104F5A24085F84081443005F0E8FEA0
:10F3D0003C4BC5F8443104F5A34005F0E1FE3A4B3F
:10F3E000C5F8803104F5A340C5F8BC61C5F8C0611B
:10F3F000C5F8C461543005F0D3FE344BC5F8D431A0
:10F4000004F5A440C5F81082183005F0C9FE304B51
:10F41000C5F8183204F5A440603005F0C1FE2D4B4C
:10F42000C5F8603204F5A5401C3005F0B9FE2A4B42
:10F43000C5F89C3204F5A640C5F81463C5F81863F6
:10F440003030FFF7F3FD384605F0AAFE234BC5F830
:10F45000BC3304F5A740783005F0A2FE204BA5F898
:10F46000348404F5A840C5F8F8334830FFF7DEFDD2
:10F470001C4BC5F84834012385F8D13405F59B634E
:10F4800004F5A9401E605E609E60643005F088FE51
:10F49000154BC5F8E43405F2245520462E606E6005
:10F4A00009B0BDE8F08300BFCDCC4C3DC4510C0881
:10F4B00068520C086C550C08FC550C08B8560C0822
:10F4C00058570C08F8570C0890580C0830590C087D
:10F4D000C0590C08585A0C08F85A0C08CC5D0C0896
:10F4E000685F0C08285D0C082C600C0838B5054BCB
:10F4F0001C6823680A461D68034B01462046A8473E
:10F50000002038BDE8800020B82B002010B587F01F
:10F5100067FD064C064B18602046FFF7A3FD20460A
:10F52000044A0549BDE81040A9F038B8B82B0020BE
:10F53000E880002094E3002035E8000801207047AF
:10F5400090F890308B4286BF00EB8100D0F8940099
:10F550000020704790F890308B4286BF00EB81000E
:10F56000D0F8940000207047FA207047014B93F8C0
:10F5700052037047B84B0020034BD3F8D000431E12
:10F5800058425841704700BFB85B0020034BD3F886
:10F59000D000831E58425841704700BFB85B00201E
:10F5A000034BD3F8C00008B180F0ECBF01487047AE
:10F5B000B85B002090010C0838B5036A2E4D43F467
:10F5C000E0520262426A42F4E0524262826A42F4CB
:10F5D000E0528262D5F8482B0446E2B143F4F84386
:10F5E0000362D5F8480B7CF0E1FA38B1636A43F462
:10F5F00080436362A36A43F48043A362D5F8480B57
:10F600007CF0F6FB38B1636A43F400536362A36A8B
:10F6100043F40053A362194B1D6845B119212846D4
:10F6200049F0C6FB18B1236A43F480732362144B7C
:10F6300093F8EC3C6BB1636A43F48073636245B149
:10F640001921284649F0ECFB18B1A36A43F48073F2
:10F65000A362236A43F080432362636A43F08043DA
:10F660006362084BD3F8C03093F8C1301BB9A36A6A
:10F6700043F08043A36238BDB86B00204C83002068
:10F68000B84B0020B85B002013B54FF44470CDE9AF
:10F69000002118F0DDFA044628B1DDE900215AF016
:10F6A00081FB024B2360204602B010BDE4030C082E
:10F6B0000020704770470000032070470820704703
:10F6C000014B93F854037047B84B0020034B93F958
:10F6D0000C04003818BF0120704700BFB84B002051
:10F6E000014B93F956037047B84B00207047000058
:10F6F0007047000008B50C4BD3F8480B70B91023C5
:10F700000A4AD2F8C02043F0400022B192F8CB2040
:10F710000AB143F0C00040F0010008BD7CF046FA99
:10F720000028ECD01823EBE7B86B0020B85B002072
:10F7300038B5C5780B46352D044628BF352535220A
:10F7400000211846ABF06CFC2A4604F10C01BDE820
:10F750003840ABF01BBC00001FB5184C94F8E61104
:10F7600004F1980010F014FC78B194F8E61104F15B
:10F77000980010F00FFC40B194F8E61104F19800E5
:10F7800004B0BDE8104010F007BC002301930293C1
:10F79000039312F01DFB01A912F0F4F820B101A8A7
:10F7A0002DF01EF804B010BD21F0D0FC90F8C4324A
:10F7B000B02202FB030090ED2F0AF3E7B84B0020C4
:10F7C00008B50D4BD3F8C000A8B1443053F05EF833
:10F7D000034693ED000ADFED090A9F20B7EE001AF9
:10F7E00029F0F2F9DFED067A20EE270ABDEEC00A15
:10F7F00010EE103A18B208BDB85B002000000000FF
:10F800000000C8422DE9F04FDFF8D880344F8DB0AA
:10F810000446042508F5005617F8019BB8F9AC33E7
:10F8200009F1FF3A43FA0AF3D90742D5207C54F094
:10F83000A5FB8346207C55F0A5FA00F121039B45EA
:10F8400005D2207C0DB0BDE8F04F53F013BEBAF1E5
:10F85000030F2ED8DFE80AF00234393ED6F8400B09
:10F8600003689B68984700F194035A69D3F800A095
:10F87000D3F804E0D8681969D3F818C008925A6A16
:10F880001B6ACDF82520CDF8293062222123CDE94D
:10F89000003206900791207CCDF80CA0192303AA12
:10F8A000C221CDF810E0CDF814C08DF8249054F0AA
:10F8B000CFFB013D15F0FF05AED10DB0BDE8F08FD7
:10F8C000D6F8400B0368DB68CCE7D6F8400B03683A
:10F8D0001B69C7E7D6F8483B03F52A73C5E700BFA5
:10F8E000B0040C08B84B002013B50446074801913A
:10F8F00008F032FC30B90199204602B0BDE8104052
:10F9000055F064BC042002B010BD00BFE0780020B8
:10F91000014808F07BBA00BFE078002059F0A2B996
:10F9200010B588B0044656F0DDFD0C4BD3F8C0008E
:10F9300038B90B4A0621204608B0BDE8104056F001
:10F94000B9BD69461E2280F021FE064A6B4606219B
:10F95000204656F0AFFD08B010BD00BFB85B0020D8
:10F96000DC010C083A4F0C08034A92F8CC3C0133F6
:10F9700082F8CC3C55F0BABEB84B002007B508461B
:10F98000019117F0DBFE38B10448019902F09CFCAC
:10F99000002003B05DF804FB0420FAE7F4800020A7
:10F9A000162A10B40C4605D0542A03D05DF8044B37
:10F9B00055F02ABC0323237001205DF8044B7047E7
:10F9C00008B555F0C7FD40F41C6040F00D0008BDBF
:10F9D00010B5044618F044F9204610BD10B50C4C83
:10F9E00094F99030002B0FDBD4F89C000368DB6C9B
:10F9F000984758B9D4F89C0003689B6C9847002836
:10FA00000CBF0220032010BD0120FCE70420FAE710
:10FA1000B85B002010B44C69012C05D101465DF89B
:10FA2000044B034802F0CEBF5DF8044B55F078BE9E
:10FA3000B82B00202DE9F341B1F90430002B064624
:10FA40000C46154635DB4FF00008CDE900281A4F6B
:10FA5000B1F902209FED190AD7F8D01C4FF47A7340
:10FA600059F0DAFB0123CDE900539FED140AB4F9F4
:10FA70000020D7F8D41C4FF47A73304659F0CCFBF1
:10FA80009FED0F0AB4F90420D7F8D81C434630463E
:10FA9000CDE9005859F0C0FBCDE900589FED070AA9
:10FAA000B4F90620D7F8DC1C4FF47A73304659F0CD
:10FAB000B3FB02B0BDE8F081B84B00200000FA446F
:10FAC00000007A44044B187820B9044B93F8920054
:10FAD000C0F38010704700BF44820020B85B002054
:10FAE0000B4B93F815267AB993F8B52092060BD1F3
:10FAF00093F99020002A09DB93F8913013F0200F3E
:10FB000014BF042001207047052070470320704770
:10FB1000B85B002008B5074B93F9A033032B03D043
:10FB2000BDE8084056F03EBD034A022156F0C2FC33
:10FB3000042008BDB84B0020F4010C08094BD3F891
:10FB40001024920701D455F051BB03F5005303F67E
:10FB5000183393ED000ADFED047AB8EEC00A20EE08
:10FB6000270A7047B84B00200AD7233C10B594B041
:10FB7000044603A817F00CFD1C4BD3F89C00036847
:10FB800003A95B6D984778B3002103A817F098FD8F
:10FB900050B3247C87F0F4FD059BDDED047A0893D7
:10FBA000069B09930023F8EEE77A9FED117A0B93F9
:10FBB0000C930D930E930F931093119312934FF692
:10FBC000F853ADF84C300023962267EE877A8DF813
:10FBD0004E303323CDE90032079007AA5721204643
:10FBE000CDED0A7A54F034FA14B010BDB85B0020A1
:10FBF0000AD7233C30B52DED0A8B774C0546D4F857
:10FC00009C00036899B05B6A984700285BD004F5B4
:10FC10000054D4F81032062B00F2C980DFE803F05C
:10FC20000404045788AB53006C489FED6D8A0AF0BA
:10FC300011FC9FED6C0A0168426883680D930BA864
:10FC40000B910C922CF0CEF9F0EE489AB0EE40CA2F
:10FC5000F0EE60BAB0EE419AB0EE48AAF0EE488AF3
:10FC6000F0EE48AAB0EE48BA40F6F8542D7C87F082
:10FC700087FD00231593169301238C228DF85E30A7
:10FC80003323CDE900320B90B1EE499AF1EE688A48
:10FC9000B1EE488A0BAA552128468DED0CCACDED50
:10FCA0000DBA8DED0E9A8DED0FBACDED10AACDEDFA
:10FCB000118A8DED12AACDED139A8DED148AADF84F
:10FCC0005C4054F0C5F919B0BDEC0A8B30BD434817
:10FCD0000AF0C0FB9FED430A0168426883680D93F8
:10FCE0000BA80B910C922CF07DF93C48F0EE60BA19
:10FCF000B0EE419AB0EE40CA0AF0B0FB9FED390A6F
:10FD00002CF070F93548B0EE40BAF0EE60AAF0EE93
:10FD1000418A0AF0A7FB9FED330A2CF063F94FF4F8
:10FD20004064B0EE40AAF0EE609AB0EE418A9DE7E2
:10FD30002A489FED2B9A0AF091FB9FED2A0A2CF09E
:10FD400051F92648B0EE40BAF0EE60AAF0EE418AD2
:10FD50000AF088FB9FED230A2CF044F9F0EE49BA33
:10FD6000B0EE40AAF0EE609AB0EE418AB0EE49CA19
:10FD700040F607447AE71948DFED198A0AF072FB6A
:10FD80009FED180A2CF02EF9F0EE68AAB0EE40AA0A
:10FD9000F0EE609AB0EE418AB0EE68BAB0EE689AC2
:10FDA000F0EE68BAB0EE68CA40F63F445EE79FEDF9
:10FDB0000C8A0024F0EE489AB0EE48AAF0EE488A89
:10FDC000F0EE48AAB0EE48BAB0EE489AF0EE48BA63
:10FDD000B0EE48CA4AE700BFB85B00208C7D002027
:10FDE000000000000AD7233C2DE9F0412DED068BE1
:10FDF0003B4D95F8913099068CB004466AD505F5CF
:10FE000080579FED380AD7F8400BDFED378A6C300A
:10FE10002CF0E8F88DED041A21EE281AD5F89C6034
:10FE20008DED020ABDEEC11ACDED030A11EE103AB6
:10FE30001DB2336894F810809B6D304660EE289AAE
:10FE400020EEA89A984707EE900AF8EEE77A304637
:10FE500067EEA87AFDEEE77A17EE903A1CB23368A7
:10FE6000DB6D984707EE900AB8EE678AD7F8483BF3
:10FE7000DFED1E7A93ED0FAA336828EE288A1B6EF9
:10FE8000B4EEE78AF1EE10FA58BFB0EE678A30465A
:10FE90009847BCEEC88A0023089318EE103AB722A0
:10FEA0002AEE28AA20EE280AADF82C301A23CDE934
:10FEB00000323E2105AA4046CDED059A8DED069A09
:10FEC0008DED07AA8DED090AADF82850ADF82A404E
:10FED00054F0BEF80CB0BDEC068BBDE8F08100BF5D
:10FEE000B85B00209F0CB3450AD7233C00FF7F4737
:10FEF0002DE9F04F2DED028B1A4B047CD3F8403BDB
:10FF00008DB0D3F88480D3F88870D3F88C60D3F8A0
:10FF1000905093ED258AD3F898B0D3F89CA0D3F8ED
:10FF2000DC9087F02DFC00238DF82C301622252341
:10FF3000CDE90032029002AA532120468DED078AB6
:10FF4000CDF820B0CDF824A0CDF82890CDF80C80C5
:10FF500004970596069554F07BF80DB0BDEC028B26
:10FF6000BDE8F08FB86B0020054BD3F8C0302BB143
:10FF700093F8CA00002808BF02207047022070478B
:10FF8000B85B002008B5034BD3F89C0003681B68DE
:10FF9000984708BDB85B0020024B93F89100C0F36E
:10FFA00040107047B85B002070B52C4E2DED028BD1
:10FFB0000546D6F89C0091ED018A036886B05B6A1D
:10FFC0000C46984750B9BDEEC88A18EE103ADB07C8
:10FFD00004D4022006B0BDEC028B70BDD4E904014C
:10FFE00029F0AAFE0028F4D002A817F0D1FA02AA3C
:10FFF0002146284659F080F80028EAD0184902A87E
:020000040801F1
:1000000017F0A8FB03460028E3D1DFED160A0090A5
:100010000246B0EE600A144802A90AF053F8D8B1BB
:10002000D6F89C0003685B6A9847044608B1002034
:10003000D0E70E480222042105F04AFC60B1DFED52
:10004000090A094800942346B0EE600A224602A934
:100050000AF038F80028EAD10420BBE7B85B00209A
:10006000CC760020000000008C7D0020B82B002002
:1000700008B591F82030032B1CD1D1ED027A9FED09
:100080000E7A91ED060A0D4BF0EEE77AF4EEC77AA0
:10009000DFED0B7AD3F89C00F1EE10FA4CBF012192
:1000A000002120EE270A0FF00BFA002814BF0020D1
:1000B000042008BD0220FCE700000034B85B0020EB
:1000C0000000C84210B52DED028BD1ED007AF5EE9F
:1000D000C07AF1EE10FA82B00C4604DA042002B0C5
:1000E000BDEC028B10BD9FED197AF4EEC77AF1EEEC
:1000F00010FAF3D891ED030A9FED158AF0EEC07A5D
:10010000F4EEC87AF1EE10FA19D5D4ED037A11485D
:10011000D4ED010A94ED000AF4EEC87AD4ED027A27
:10012000FDEEE77AF1EE10FACDED017A9DF90410BB
:10013000ACBF0122002202F029F80020CFE7F7EE41
:10014000000A28F03DFC0028C8D0DEE70000B443D8
:1001500000000034F480002091ED010AB5EEC00AE1
:10016000F1EE10FA08B501DC042008BD9FED107A0D
:10017000104BD1ED007AD3F89C0020EE070A9FEDDA
:100180000E7A0368F4EEC77AF1EE10FA05DDDB6E45
:1001900098470028E8D00020E7E79FED087AF4EEC2
:1001A000C77AF1EE10FACCBF9B6E5B6EF0E700BF32
:1001B0000000C842B85B00209A9939403333F33FBE
:1001C00008B5D1ED007A9FED157AF0EEE77AF4EEFE
:1001D000C77AF1EE10FA1DD5D1ED017AF0EEE77A8B
:1001E000F4EEC77AF1EE10FA14D50D48022203217D
:1001F00005F06EFB80B10A480121FDF7DBFF0948DD
:1002000090F8683D012B03D000F664502FF022FADD
:10021000002000E0022008BD0420FCE700000034BC
:10022000B82B0020B86B002010B5D1ED007AFCEEA1
:10023000E77A17EE903A9CB2012C02D0022C06D03D
:100240004CB9064821465FF0DFFA002010BD044893
:1002500003F064F9F9E70420F8E700BFE87700202D
:10026000B82B00201FB5D1ED017A0B7CFCEEE77AAC
:10027000CDED027AD1ED007A0093FCEEE77AD1ED74
:10028000030ACDED037A91ED020A9DF808309DF83E
:100290000C20014602480DF0D1FE05B05DF804FBCC
:1002A000B82B002010B50A4C94F8B530DB070CD4FD
:1002B00002220521A4F5405005F00AFB28B90222CC
:1002C0001146A4F5405005F003FB002010BD00BF0F
:1002D000B85B002010B5D1ED007AFCEEE77A044659
:1002E00017EE903A13F0FF030FD10F4BD3F89C0099
:1002F00003689B6F984708B1002010BD0B4A204649
:10030000062156F0D7F80420F7E7012B09D1064B58
:10031000D3F89C000368DB6F98470028ECD1044AAF
:10032000EDE70220E9E700BFB85B002018020C08E7
:1003300028020C089FED0B7A01F10C03F1EC017A15
:10034000F4EE677AF1EE10FA0AD6F0EEE77AF4EE00
:10035000C77AF1EE10FA03DC9942EFD10120704721
:100360000020704700007A4430B52DED028B8DB02F
:100370000023054603930493059311F029FD03A977
:1003800011F000FB58B311F023FD00F55A7393E808
:10039000070006AC84E80700DDED060A9DED070ABC
:1003A0002D7CF1EE600AB1EE400AA8F03FFC204639
:1003B000B0EE408A2CF014FADFED0B7A089B0B9319
:1003C000012228EE278A0C23CDE90032A82109AAB0
:1003D00028468DED098A8DED0A0A53F039FE0DB0DD
:1003E000BDEC028B30BD00BFE02E6542242938B53C
:1003F00005460FD003D81B2907D1012412E040295C
:10040000FBD0A1F14203012BF7D92846BDE83840C3
:1004100059F034BA0C2153F03FF8044610B1284685
:10042000FFF7A2FF204638BD38B5194C94F8B53017
:10043000DB070D460AD4D4F8C03093F8CB303BB973
:1004400001221146A4F50370FDF70AFD002038BD16
:1004500094F99030002B4FF0020212DA0521A4F536
:10046000405005F035FA0028F0D095ED000ADFED98
:10047000097AD4F89C0020EE270A01210FF020F819
:10048000E4E70921A4F5405005F022FADEE700BFB9
:10049000B85B00200000C84210B5214C94F8B5307C
:1004A000DB070ED4D4F8C03093F8CB304BB194F9BD
:1004B0009030002B07DA01220821A4F50370FDF724
:1004C00083FD002010BDD1ED007A9FED167AF0EE8D
:1004D000E77AF4EEC77AF1EE10FA0BD51248022251
:1004E000112105F0F5F9A0B9022211460E4805F0D8
:1004F000EFF9E6E7D4F89C0003681B6898470428E6
:10050000DFD0D4F89C0003681B6898471428E5D115
:10051000D7E7064840F6C41108F0F8FAD1E700BF63
:10052000B85B002000000034B82B0020787C00204D
:1005300070B58B8BC12B05460C463CD8BB2B0CD819
:10054000542B6AD02ED8113B99B2052918D92146CF
:100550002846BDE870405AF029B8BC3B052BF6D8B8
:1005600001A151F823F000BF5506010863060108F8
:100570004F0501084F050108FF050108090601089C
:10058000052BE4D801A151F823F000BF3F06010874
:100590004F0501084F0501084F060108B105010884
:1005A0001B060108732B22D0B22B24D0552BCED1A1
:1005B0000222092145E04AF21146B34237D00AD857
:1005C000D12B26D0B3F5967F35D0D02BBFD1BDE847
:1005D0007040FFF729BE4AF21246B34223D04AF2D6
:1005E0001346B342B3D1BDE87040FFF755BFBDE835
:1005F0007040FFF767BDBDE87040FFF7ADBD214615
:10060000BDE87040FFF7D0BC2146BDE87040FFF761
:1006100061BEBDE87040FFF725BE21462846BDE813
:100620007040FFF725BDBDE87040FFF7FDBEBDE897
:100630007040FFF737BEBDE87040FFF7C1BD022232
:1006400005210A4805F044F948B9042070BD02228A
:100650000621F6E70221064806F0A6FAF4E7002094
:10066000F4E70221024806F069FAEDE7B82B002012
:10067000E078002008B591ED007AF6EE007AB4EE4D
:10068000E77AF1EE10FA06DD044801220521FDF7B4
:100690009BFC002008BD0420FCE700BFAC590020F3
:1006A00030B52DED028BCD7893B0272D28BF2725AF
:1006B0000C462722002108A8AAF0B2FC2A4604F121
:1006C0000C0108A8AAF062FC424BD3F89C00036816
:1006D0005B6A9847002841D09DF8465068063DD493
:1006E00000244FF07E532906049307940694059442
:1006F00027D504A82AF04EFFEA0701940294039438
:1007000005F006032ED4002B2ED10D9B01930E9BDA
:1007100002930F9B0393304809F082FA9DED100A73
:10072000044630B340F2ED40B7EE001AFFEE000A87
:1007300028F04AFA2848234601AA04A909F078FAC1
:100740000CE0099B04930A9B05930B9B069304A85A
:100750000C9B07932AF024FF0028CDD113B0BDECE9
:10076000028B30BD062BD6D001211B4809F0F4F9CD
:10077000F4E7DFED1A0A4FF49E60B7EE001A28F096
:1007800023FAF6EE000AB0EE408A28F019F9E8B92B
:10079000B6EE000A124BB4EEC08AF1EE10FAD3F8AE
:1007A0004C3B08DD38EE400A30EE008A93ED070A34
:1007B00028EE000ABEE730EE480AD3ED087A30EEA4
:1007C000000AF0EEE77A27EEC00AB3E79FED030ACE
:1007D000B0E700BFB85B00208C7D00200000000067
:1007E000B86B00202DE9F0439DB0814608460EA964
:1007F000FEF79EFF844BD3F89C0003685B6A984722
:1008000050B19DF86C30012B09D0DA1F022A06D9AD
:100810007E48012109F0A0F91DB0BDE8F083BDF8C4
:100820006840A20504F0070604F0380704F4E075F8
:1008300001D5002DF0D04FF00008CDF81480CDF890
:100840001880CDF81C803EBB9FED716A9DED107A3B
:10085000DDED117ADDED0F6A27EE067A67EEC67AD6
:1008600066EE866A083B012BCDED056A8DED067AB2
:10087000CDED077A04D8674806AA05A9FDF714FE4E
:100880009DF86C30073B022B06D863487EF0D2FD02
:10089000014605A82BF0C6FBCDF82080CDF82480BA
:1008A000CDF82880F7B9DDED147A129B0893F1EEAC
:1008B000677A139B099308A94846CDED0A7AFFF79A
:1008C00039FD0028A4D09FED520A08A82BF0DEFBCA
:1008D0009DF86C30083B012B04D84E4809AA08A9A2
:1008E000FDF7E2FDCDF82C80CDF83080CDF83480D6
:1008F000EDB99FED476A9DED167ADDED177ADDEDD6
:10090000156A9DF86C3027EE067A67EEC67A66EEB9
:10091000866A083B012BCDED0B6A8DED0C7ACDED8F
:100920000D7A04D83B480CAA0BA9FDF7BDFD14F4C1
:10093000806233D1DFED397A9DED180A9DF86C1095
:1009400020EE270ADFED327A0839012920EE270A46
:100950008CBF0021012114F4006305BFDFED2F7A65
:10096000DDED190ADFED2E0A60EEA70A04BFDFED08
:10097000287A60EEA70AAEB9002F35D1B3FA83F317
:10098000B2FA82F25B0952090291019300920BAB19
:1009900008AA05A91D4809F04DFA3DE79FED200A78
:1009A0000021D8E77FB9B3FA83F35B0901200093F4
:1009B000B2FA82F3CDE901105B0914480BAA08A929
:1009C00009F0D0FC28E7002D7FF422AF0120B3FA14
:1009D00083F3B2FA82F2CDE900105B090B485209A9
:1009E0000BA909F067FC17E7002D3FF411AFB3FA2C
:1009F00083F3B2FA82F2CDE900165B09520905A928
:100A0000024809F099FA07E7B85B00208C7D0020C6
:100A10000000C842B82B0020DC760020E02E6542A2
:100A2000000000002DE9F047A2B08046084614A956
:100A3000FEF77EFE7E4BD3F89C0003685B6A984706
:100A4000C0B1BDF88040A30504F0070904F4E077C5
:100A500000D57FB10CAE304616F09AFDB9F1000F0B
:100A600029D1DDE9150129F067F930B97148012173
:100A700009F072F822B0BDE8F0879DF8841009AA49
:100A8000404658F023FB0028F0D0DDED177A9FEDAB
:100A90006A7A099B009367EE877A10ADFDEEE77ADC
:100AA000DDE9151217EE903A284616F091FD95E80B
:100AB0000F0086E80F00002514F0380A0695079508
:100AC000089514D1DDED1A7A189B0693F1EE677A3A
:100AD000199B079306A94046CDED087AFFF72AFC3B
:100AE0000028C3D09FED540A06A82BF0CFFA099531
:100AF0000A950B959FB99FED506A9DED1C7ADDED2F
:100B00001D7ADDED1B6A27EE067A67EEC67A66EE81
:100B1000866A8DED0A7ACDED096ACDED0B7A14F473
:100B2000806805BFDFED457A9DED1E0A9FED440A02
:100B300020EE270A04BFDFED407A20EE270A14F4E6
:100B4000006405BFDFED3D7ADDED1F0ADFED3C0AF5
:100B500060EEA70A04BFDFED387A60EEA70AB9F1AC
:100B6000000F31D1BAF1000F52D13046CDED050A58
:100B70008DED040A16F03CFD03289DED040ADDED21
:100B8000050A3FF473AF10A93046CDED050A8DED8F
:100B9000040A10951195129516F08AFE00283FF46C
:100BA00065AFB4FA84F46409B8FA88F3DDED050A98
:100BB0009DED040ACDF804A000945B0906AA10A9D3
:100BC0001C4809F0A7F955E7BAF1000F0FD101232E
:100BD000B4FA84F4CDE901A36409B8FA88F315489E
:100BE00000945B0909AA06A909F0BCFB42E7002FA3
:100BF0007FF43CAF0123CDE90073B8FA88F2B4FA70
:100C000084F30C485B09520909A909F053FB31E749
:100C1000002F3FF42BAFB4FA84F3B8FA88F2CDF882
:100C200000905B0952093146024809F04BFA21E76E
:100C3000B85B00208C7D00200000C842E02E654299
:100C40000000000010B44B7A8C7ACA7A43EA04237D
:100C500043EA0243542B07D0562B09D0522B0BD119
:100C60005DF8044BFFF71CBD5DF8044BFFF7BABD00
:100C70005DF8044BFFF7D6BE5DF8044B58F02EBB71
:100C80002DE9F0432DED028B00F540560446D6F8D1
:100C90009C00DFED4C8A036891B05B69984704F5CE
:100CA00080490027002840F08880D9F8483BD3EDE0
:100CB000DE7A93EDD88AFDEEE77A28EE288A17EEE1
:100CC000903A1DB204F5355808F13C0801A9404698
:100CD0000DF09CFF18B950F0C7F93B4B0193372238
:100CE000002102A8AAF09CF9A3238DF808309523CF
:100CF0008DF8093086F04CFDD9F8403BCDF80B005B
:100D0000D6F8C000D3F8DC20D3F8E030CDF80F10CF
:100D10004430CDF81320CDF8173051F0B7FD03461D
:100D2000DFED2A0A93ED000AB7EE001A9F2027F0A4
:100D30004BFF10EE103AD6F8C000CDF81B30036818
:100D40001B69984710EE103A04F59646CDF81F300F
:100D5000243618EE103A3046CDF823307EF06EFB84
:100D600020EE280A404610EE103ACDF82730D9F888
:100D7000F03ACDF82B30019BCDF82F300DF068FF05
:100D800010EE103A3046CDF83330CDF83770ADF86C
:100D90003B507EF05FFBBDEEC00A04F58D5010EEB7
:100DA000103A372202A91030ADF83D304FF0DCFA8E
:100DB00011B0BDEC028BBDE8F08308EE107A00257F
:100DC00080E700BF0AD7233C2292CA7F00000000C0
:100DD00010B500F58044D4F8400B77F017FAD4F83A
:100DE000481BD4F8400BBDE8104077F075BA0000FE
:100DF00070B54FF4805105460EF052F800284FD0E0
:100E000005F5804605F58D54D6F8400B03689B68C0
:100E10009847103400F19402692120464FF054F9AC
:100E2000D6F8400B0368DB6898476A2100F194020A
:100E300020464FF049F9D6F8400B03681B699847E4
:100E40006B2100F1940220464FF03EF9D6F8482B72
:100E50006C21204602F52A724FF036F920212846EF
:100E60000EF01EF8E0B105F54053D3F89C0003687E
:100E70001B69984778B1D6F8482B204690326E21EE
:100E80004FF022F9D6F8482B2046BC32BDE870401E
:100E90006F214FF019B9284609F0CEFF0028EAD19A
:100EA00070BD000008B510F093FFBDE8084010F0D9
:100EB0001BBD00007FB50E464FF6FF710446154678
:100EC0000DF0EEFFE8B1102200216846AAF0A8F864
:100ED000A3238DF8003095238DF8013003238DF87E
:100EE000023086F055FC1022CDF8030004F58D5039
:100EF000CDF80710104469468DF80B6003954FF04C
:100F0000B3FA04B070BD00007FB50E464FF6FF7116
:100F1000044615460DF0C4FFE8B1102200216846D2
:100F2000AAF07EF8A3238DF8003095238DF80130C8
:100F300004238DF8023086F02BFC1022CDF803003C
:100F400004F58D50CDF80710104469468DF80B60FC
:100F500003954FF089FA04B070BD000030B52DED57
:100F6000048B87B004460D46182200216846B0EE77
:100F7000409AF0EE608AB0EE418AAAF051F8A323BD
:100F80008DF8003095238DF8013006238DF802305E
:100F900086F0FEFBCDF8030004F58D50CDF8071068
:100FA0001822694610308DF80B508DED039ACDED67
:100FB000048A8DED058A4FF0D7F907B0BDEC048B9C
:100FC00030BD000010B54FF4801104460DF068FFED
:100FD00030B104F5A2501830BDE810400FF070B9E0
:100FE00010BD00002DE9F0438FB014460546894638
:100FF0003122002101A8DDE916769846AAF010F802
:10100000A3238DF8043095238DF8053008238DF83F
:10101000063086F0BDFB2368049363680593A368DC
:1010200006933B68CDF81D307B68CDF82130BB6856
:10103000CDF825303368CDF80700CDF8293005F517
:101040008D507368CDF80B10CDF82D303122B36878
:101050008DF80F9001A910308DF81C80CDF831303B
:101060004FF082F90FB0BDE8F083000070B52DEDB0
:10107000068B8CB0144605460E462C22002101A892
:10108000B0EE409AF0EE608AB0EE418AB0EE61AA0E
:10109000F0EE429AA9F0C4FFA3238DF80430952303
:1010A0008DF805300B238DF8063086F071FBDFEDEF
:1010B0001A7A94ED007ACDF8070027EE277A29EE08
:1010C000279A8DED077A94ED017ACDF80B1027EE73
:1010D000277A68EEA78A8DED087A94ED027A8DF86A
:1010E0000F6028EE278A05F58D5067EE277A2C22AF
:1010F00001A910308DED049ACDED058A8DED068A9B
:10110000CDED097A8DED0AAACDED0B9A4FF02CF9B1
:101110000CB0BDEC068B70BDE02E6542A020704780
:1011200030B5154B044689B004F58D55D3F8C00091
:10113000694610351E227FF029FA6A460F49284673
:101140004FF096FA04F54053D3F89C0003681B68EF
:10115000984704F50053014693F80C2328464FF0B6
:10116000ABFA04F5A250183011F070F804F5907045
:101170001FF056F809B030BDB85B00203A4F0C089C
:101180002A4B2B4A70B54360002343618361C361DE
:10119000C363284B426303644FF08042264B436491
:1011A00004468263583059F02BFF244E244BA3652C
:1011B000A82560195AF0DAF866513035B5F56A7F1E
:1011C000F7D104F56A705BF08DFC002104F5F66040
:1011D00081F0CCFD1B4BC4F864389FED1B1ADFED8A
:1011E0001B0A9FED1B0A04F6780077F001FE9FEDC5
:1011F000161A9FED180AF0EE410A04F5096077F01F
:10120000F7FD9FED111A9FED130AF0EE410A04F667
:10121000A80077F0EDFD20460F4946F0D7FA2046AA
:101220000E4946F0D3FA204670BD00BFE8390020D1
:101230000000C8410AD7233C0000E040A44C0C0841
:10124000B84C0C08F47A0020000000009A99993EEE
:101250000000B44300804A4368400C08C8420C08B0
:1012600070B54C4D4C49ADF50E7DD02206465AA8BE
:10127000A9F08CFE0FCD0EAC0FC40FCD0FC40FCD57
:101280000FC495E80F0084E80F0000245AAB18192A
:101290000021B7EE000A103445F066FDD02CF5D1E0
:1012A0003E4B0FCB02AC84E80F0001A9204645F06D
:1012B0000FFD90B19DF90430DFED396AE06807EE6B
:1012C000103AB8EEC77AF0EE007AE7EE267AB7EE7B
:1012D000000A80EE270A46F021FE00240EAB181902
:1012E00000211034B7EE000A45F03EFD402CF5D148
:1012F0002C49902236A8A9F049FE0022092136A8DF
:1013000045F0DEFD96F9AC69D6B9274D0FCD1EAC80
:101310000FC40FCD0FC40FCD0FC495E80F0084E8A4
:101320000F00324604211EA845F0CAFD9FED1F0A9A
:101330001F4846F0F3FD1F48B7EE000A46F0EEFDE9
:101340001D4C9FED1E0A0FCC06AD0FC594E80F0093
:1013500085E80F00002106A845F006FD9FED170A5D
:101360000021284645F000FD04F1100160221EA86E
:10137000A9F00CFE00241EAB18190021B7EE000ADC
:10138000103445F0F1FC602CF5D15BF0BFF90DF5A0
:101390000E7D70BD04F30B0834F20B0844F30B0808
:1013A000CDCCCC3D54F30B08E4F30B080000000057
:1013B000503F0C085F3F0C0824F40B080000344237
:1013C0002DE9F04790B00DF106011D205BF090FA79
:1013D000002800F09E809DF80630614A0133DBB2A0
:1013E00011210BA88DF8063085F0BAFB00220DF113
:1013F00007010BA845F0F2F99DF80630594A112172
:1014000005460BA885F0ACFB00220DF107010BA8E7
:1014100045F0E4F99DF80630534A112106460BA821
:1014200085F09EFB00220DF107010BA845F0D6F9CF
:101430009DF806304D4A03F03F03112107460BA8E3
:1014400085F08EFB00220DF107010BA845F0C6F9CF
:101450008046002D5DD0002E5BD0002F59D0002893
:1014600057D0284645F0D2FB002852D1304645F0EF
:10147000CDFB00284DD1384645F0C8FB002848D1A7
:10148000404645F0C3FB002843D1394C94E80F0097
:101490000DF10C0C10348CE80F0094E80F000DF1E6
:1014A0001C0989E80F0002A9604645F011FC98B3B9
:1014B000BDF8084002A9484645F00AFC00284AD079
:1014C000BDF8083054BB23B340F2E2449C420FFA0B
:1014D00084FA0FFA83F927D80DF10A013046ADF8E6
:1014E0000A9047F011F80DF10A012846ADF80AA05C
:1014F00047F00AF80DF10A013846ADF80AA047F0A6
:1015000003F800230DF10A014046ADF80A3047F018
:1015100015F810B0BDE8F0870024CBE740F2D662A2
:10152000002B08BF1346D1E70DF10A013046ADF894
:101530000AA046F0E9FF0DF10A012846ADF80A902D
:1015400046F0E2FF0DF10A013846ADF80A9046F088
:10155000DBFF0123D6E7002CDBD040F2D663B5E7F2
:10156000703F0C087C3F0C08883F0C08953F0C0826
:10157000A4F40B0837B500F50D517822103104465C
:101580004DF008FB00220C21254845F099FC20462F
:10159000FFF716FF04F50D500022B7EE000A0221F6
:1015A000243045F015FD012504F509511D4A00952B
:1015B00000231031452045F087FC1B4A1368D907EA
:1015C00005D41A49156004F5075338330B6004F548
:1015D0000F5016490122043045F0C8FC012504F5DE
:1015E0008D51134A009500231031FD2045F06CFC0D
:1015F000104B1A68D20705D40F4A1D6004F59B549E
:101600001C3414600C48012145F0CCFC46F0E4FA8F
:101610000A4A138843F00103138003B030BD00BFB2
:10162000A83F0C08F4910D08EC8000200022002057
:10163000FCED0C08F08000200C22002030830020FC
:101640000F299DBF302303FB01005030002070475D
:10165000014B93F997037047B84B0020024B93F866
:10166000B50000F001007047B85B0020044BB3F8F0
:101670005C33DB075ABF0069C0F34010002070479D
:10168000B84B0020014BD3F8DC0C7047B84B00205E
:1016900008B503689B68984730B9044B93F9B400C8
:1016A000B0FA80F0400908BD0020FCE7B85B0020DC
:1016B00038B50D1E2DDB174C94F8E82CEBB29A428E
:1016C00027D3D4F8E43C0122595DA4F5005004F07E
:1016D000FFF8F0B159F014FE03215AF0C9FDC0B96A
:1016E00059F00EFE0D215AF0C3FD90B994F97C33E8
:1016F000EB40DB075CBF94F99613E940A4F500507A
:1017000048BF0221BDE8384058BF01F00101FCF795
:1017100067BD38BDB84B0020022A10B50C4605D174
:10172000BDE810400948352204F0D2B8084BD3F880
:101730009C0003681B689847A04205D159F0E0FD62
:10174000BDE8104059F066BD10BD00BFB82B0020A9
:10175000B85B002029B1022907D1044BC3F89410CB
:101760007047024B0122C3F894207047B85B0020F9
:1017700031B1022907D1044B012283F89820704728
:10178000014B83F898107047B85B002010B500F546
:101790000053DFED186AD3F8D42CD3F8D03CB2F95B
:1017A0000820B3F908309FED147A07EE902AF8EE7E
:1017B000E77A0446C7EEA60A00F5A25001211830C8
:1017C00007EE903AF8EEE77A60EE870A87EEA60A0F
:1017D00020EE070A10F09AFB4FF046FC26214FF04E
:1017E0007FFB04F53950054ABDE81040062134302E
:1017F00051F036BC0000C84235FA8E3C744A0C08E1
:1018000000F58042002382F85C3B044A00F5395021
:1018100013720621024A343051F022BCA582002006
:10182000804A0C0870B500F58045044695F85C1BAD
:10183000002957D02C4B2D4AD3F89C00904204D15C
:10184000D3F8C03093F8CB3023B92046BDE87040C0
:10185000FFF7D6BF264E95F85D0B04F540530122E5
:1018600093F990303272D0BB002B3BDB85F85D2BB7
:101870000139C9B204F5005385F85C1BD3F8D42CA8
:10188000D3F8D03CB2F90820DFED1A6AB3F908307A
:101890009FED197A07EE902AF8EEE77AB1FA81F116
:1018A000C7EEA60A04F5A2504909183007EE903A8F
:1018B000F8EEE77A60EE870A87EEA60A20EE070ABE
:1018C00010F024FB95F85C3B63B904F53950337292
:1018D0000A4ABDE870400621343051F0C1BB002BEC
:1018E000C6DAB2E770BD00BFB85B0020747F00208D
:1018F000A582002000007A4535FA8E3C944A0C08F7
:101900006D2900F3E380012901DC5AF0FFBA8B1E38
:101910006B2BFAD80FF2040C5CF823F02B1B010898
:10192000251B01082B1B01082B1B01080B190108A3
:101930002B1B01080B1901080B190108251B0108B5
:101940000B1901082B1B0108251B0108251B010889
:101950000B1901082B1B01082B1B01082B1B01086D
:101960000B1901080B190108251B01082B1B010885
:10197000251B01080B190108251B0108251B01085F
:101980000B1901080B1901080B1901080B190108A3
:101990000B190108251B01082B1B01080B19010855
:1019A0000B1901080B1901082B1B01080B19010861
:1019B000251B01080B1901080B1901082B1B010835
:1019C000251B01080B1901080B1901080B19010847
:1019D0002B1B01082B1B01082B1B01080B190108ED
:1019E0000B1901082B1B01080B1901080B19010821
:1019F0002B1B01082B1B01082B1B01080B190108CD
:101A00000B1901082B1B01082B1B01080B190108DE
:101A10000B1901080B1901080B1901080B19010812
:101A20000B1901082B1B01082B1B01082B1B01089C
:101A30002B1B01082B1B01082B1B01080B1901088C
:101A4000251B0108251B01080B1901080B190108AA
:101A50000B1901080B1901080B1901080B190108D2
:101A60002B1B0108251B01080B1901080B19010884
:101A70000B1901080B1901080B1901080B190108B2
:101A80000B1901080B1901080B1901080B190108A2
:101A90000B1901080B1901080B1901080B19010892
:101AA0002B1B01080B1901080B1901080B19010860
:101AB0000B1901080B1901080B1901080B19010872
:101AC0000B1901080B190108251B0108A12921DCAC
:101AD00096297FF71AAFA1F197030A2B3FF615AFAE
:101AE0000FF2040C5CF823F02B1B01082B1B0108E0
:101AF0000B1901082B1B01080B1901080B19010810
:101B00000B1901080B190108251B0108251B0108E9
:101B10002B1B0108B42908D0DB2903D0B2297FF49C
:101B2000F4AE704700235AF0C3B9704770B563290B
:101B30008AB000F3D180012904DC0AB0BDE870400E
:101B400059F086BF8B1E612BF7D801A454F823F0FF
:101B50004F1D0108631D0108831D01088B1D01082D
:101B60003B1B0108BF1D01083B1B01083B1B010873
:101B7000711E01083B1B01083B1B0108711D010878
:101B8000971E01083B1B01086D1E0108D11E0108AC
:101B9000DF1E01083B1B01083B1B0108EF1E01086B
:101BA000FD1E01080B1F01083B1B01082D1F01082A
:101BB0003F1F01083B1B01083B1B01083B1B0108A1
:101BC0003B1B01083B1B0108511F01086B1F01084B
:101BD0003B1B01083B1B01083B1B01086F1F010851
:101BE0003B1B01083B1B01083B1B01083B1B010879
:101BF000731F01083B1B01083B1B01083B1B01082D
:101C00003B1B01083B1B01083B1B01083B1B010858
:101C10003B1B01083B1B0108831F01083B1B0108FC
:101C20003B1B0108E31E0108E71E0108EB1E01082B
:101C30003B1B01083B1B01083B1B01083B1B010828
:101C40003B1B01083B1B01083B1B01083B1B010818
:101C50003B1B01083B1B0108771F01087B1F010884
:101C60007F1F01083B1B0108871F01088B1F01080C
:101C70003B1B0108CD1F01088F1F01083B1B0108FA
:101C80003B1B01083B1B01083B1B01083B1B0108D8
:101C90003B1B01083B1B01082F2001083B1B0108CF
:101CA0003B1B01083B1B01083B1B01083B1B0108B8
:101CB0003B1B01083B1B01083B1B01083B1B0108A8
:101CC0003B1B01083B1B01083B1B01083B1B010898
:101CD0003B1B0108452001089F291DDC96297FF741
:101CE0002CAFA1F19703082B3FF627AF01A454F8BE
:101CF00023F000BF492001084D2001083B1B0108CB
:101D0000612001083B1B01083B1B01083B1B01082C
:101D10003B1B01083D200108B42900F0DB80DB29D2
:101D200017D0B2297FF409AF002A00F07981022A86
:101D30000FD1AF4BD3F89C0003689B6F984740B915
:101D400058F012F8AB4A042151F08AF901E0022A56
:101D500001D0012430E035220E21A74803F0B8FD60
:101D6000F7E7111E18BF0121A348FCF739FAF0E785
:101D7000012A04D0022A14BF00210221F4E71146EF
:101D8000F2E70621FFF7C8FCE3E7022AE1D1984D0C
:101D9000D5F89C000368DB6A984704460028D8D031
:101DA000A5F58053D3F8D83CB3F90830002BD0D137
:101DB000A5F54050FFF7EAFC20460AB070BD022AA4
:101DC000C7D18B4E8D4AD6F89C109142C1D0D6F81F
:101DD000C02092F8CB20002ABBD006F58054A6F58F
:101DE0008056B4F9982D2AB9D6F8D83CB3F9083002
:101DF000002BAED01C22002103A805ADA9F010F9DC
:101E0000284615F0C5FBB4F9983D93B91623ADF8F3
:101E10000E30D4F8183B7A48642BB8BF642303A96A
:101E200006932BF089F820B14FF01EF927214FF0CF
:101E300057F804F6143494E80F0085E80F00D6F83C
:101E4000D83C6F48B3F90830002BCCBF10231523C2
:101E500003A9ADF80E302BF06FF800283FF479AFEE
:101E60004FF002F927214FF03BF872E7032189E791
:101E7000022A644D03D0002385F8EC3C69E7192160
:101E8000A5F5885046F094FF04460028F3D00123BE
:101E900085F8EC3C90E7012A0BD0022A11D0002AE9
:101EA0007FF457AF574B83F8C0234FF0DDF82B2159
:101EB000D9E7544B019283F8C0234FF0D5F82C2179
:101EC000D1E7504B83F8C0234FF0CEF82D21CAE75D
:101ED0000F2157E74C48114684F040F839E70921B3
:101EE00050E704214EE705214CE717214AE7901EF1
:101EF0004142414145485DF087FC2AE7022A7FF4D0
:101F000028AF3D4801F00AFB23E7012A06D0022A48
:101F100007D0002A7FF41DAF1146EBE7114601926E
:101F2000E8E73A4801215DF06FFCEAE7384B911E83
:101F3000D3F8403B4A424A4183F8202009E7931EE8
:101F400059425941324BD3F8400B78F05DF800E725
:101F5000274B013A93F89210012A8CBF00220122EC
:101F600062F3041183F89210F3E611210AE71221BB
:101F700008E7152106E7002104E7102102E7022106
:101F800000E70121FEE60721FCE60B21FAE6022A22
:101F90001F4B0ED1012483F8884C4FF065F84A217D
:101FA0004EF09EFF57F0E0FE1A4A062151F058F815
:101FB00002E7002283F8882C4FF056F84B214EF0B0
:101FC0008FFF57F0D1FE144A0621BDE6012A09D041
:101FD000022A0AD0002A7FF4BCAE01210F480CF07F
:101FE0004DFEB6E601920021F8E71146F6E700BF84
:101FF000B85B0020CF4A0C08B82B0020E078002006
:102000001C790020B84B0020F47A0020E8770020EB
:10201000B86B0020AC4A0C08BD4A0C0834590020AB
:10202000184BD3F89C000368DB6F984791E6114684
:10203000FFF790FB144803F0F7FF8AE61146FFF71D
:1020400097FB86E61B219DE61C219BE6022A7FF476
:1020500080AE0E48FCF7A8FE57F086FE0C4AB3E7A8
:10206000114659F015FC0B4874F06AFE044600282E
:102070003FF46FAE034A92F8933043F0020382F8C4
:10208000933099E6B85B002064780020B82B0020DC
:10209000E84A0C08AC59002010B5044604487DF00D
:1020A000CBF904F10801BDE8104027F0C3BD00BF23
:1020B000DC76002038B504462DED028B11487DF00A
:1020C000C1F9054629F0F2FC0F48B0EE408A0CF049
:1020D00081FE90B1DFED0D7AB4EEE78AF1EE10FAF1
:1020E0000BDDD5ED000A95ED010AA6F09FFDDFEDB1
:1020F000087A20EE270A84ED080ABDEC028B94EDE5
:10210000080A38BDDC760020B82B002000401C46B1
:10211000E02E6542074B93F97D03022805D0032882
:1021200006D0003818BF0120704781F001007047C9
:1021300004207047B84B002003688B4216D0042956
:10214000C0E9001302D007290ED07047084B9FED5D
:10215000097A03F5CB63D3ED007AF8EEE77A67EE00
:10216000877AC0ED087A704700238362704700BF0A
:10217000B83B00200AD7233C08B50246FFF7CAFF48
:10218000BDE8084001461046FFF7D6BF70B52DEDFB
:10219000048B0446F0EE408AB0EE608A0D46164687
:1021A00085F0EEFA9FED329ADFED329AE06176B378
:1021B000236843B9304B03F5CB63D3ED007AF8EED7
:1021C000E77AC4ED097A68EE898A002DB7EE000A35
:1021D000FFEE007AB8BFB0EE670A68EE808AC4ED01
:1021E000058A264BB4EEE98AF1EE10FAD3F8400BDB
:1021F00030DA76F0E7FE20EE090A84ED060ABDEC3F
:10220000048B20460321BDE87040FFF795BF94ED95
:10221000090A98EE890A26F081FC002D84ED050A52
:102220000BDAB4EEE90AF1EE10FADADBDFED147A3C
:1022300030EE670A84ED050AD3E7D2D0DFED117ADC
:10224000B4EEE70AF1EE10FACBD8DFED0D7A30EEFE
:10225000270AEFE776F0B6FEB4EE480AF1EE10FA80
:1022600048BFB0EE408A28EE098A84ED068AC6E7A8
:102270000000C84200000034B83B0020B86B0020CA
:1022800000A00C47000000B410B52DED028B0446F1
:10229000B0EE608AF0EE408A85F072FADFED090A4E
:1022A000E06168EEA08A68EE200AC4ED098ABDEC00
:1022B000028BC4ED0A0A20460621BDE81040FFF754
:1022C0003BBF00BF0000C84208B54A680346084645
:1022D00042B98A6832B9C96821B9BDE808400748DF
:1022E000FFF74ABF03F1080115F0E2FA28B1BDE893
:1022F000084002480221FFF71FBF08BDF4800020FC
:1023000008B50721FFF718FF80ED0A0A08BD000095
:1023100008B50368032B23D1D0ED057A9FED127A1F
:10232000F0EEE77AF4EEC77AF1EE10FA1AD50F4B19
:1023300090ED090A03F5CB63D3ED007AF8EEE77A66
:1023400037EEC00A26F0EAFBDFED097AB0EEC00AEC
:10235000B4EEE70AF1EE10FA94BF0120002008BDA8
:102360000120FCE70020FAE700000034B83B002021
:102370000000484330B50368023B85B00446082B93
:102380006DD8DFE803F0050D30374B613F61610028
:10239000FFF782FE84ED090A94ED090A05B030BD0D
:1023A00085F0EEF9E369DFED310AE061C31A07EE6B
:1023B000903AF8EE677A94ED050A67EEA07AD4EDCC
:1023C000060AF12020EEA71A67EEE00A26F0FCFBD1
:1023D000D4ED057A77EEC07AC4ED057AD4ED097AAA
:1023E00037EE800AD6E7FFF765FEDFED217A20EEB3
:1023F000270ACFE71F4BD3ED3A7AF8EEE77AC0ED24
:10240000097AC9E71C4DD5F8540B7BF0AFF90028C9
:10241000C2D0D5F8543B1B6B6362BDE785F0B0F9C1
:10242000E3699FED127AD4ED0A6AE061C31A07EE00
:10243000903AF8EE677A67EE877A94ED097AA6EE1D
:10244000A77A84ED097AA7E70B4B9FED0C0AD3F826
:10245000400B6C3029F0C6FD84ED091A9CE7064B51
:10246000D3F8483BD3F84433D6E700BF6F12833A22
:102470000000C842B85B0020B86B00209F0CB34539
:102480000368092B08D8DFE803F0050A05050505F0
:10249000070705100023836290ED0A0A7047044B7A
:1024A000D3F8483BD3F84833F5E7C36AF3E700BFF6
:1024B000B86B0020F8B50023214FCB6297F8B530F8
:1024C000204E13F0010F04460D462DD1D7F89C0085
:1024D00003685B6F984738B3D7F89C0003F0AEFBF6
:1024E000DFED197A85ED0B0AB0EEC00AB4EEE70A0B
:1024F000F1EE10FA03D409213046FFF71DFE114812
:10250000FFF738FF0F4884ED000AFFF7B9FF336883
:1025100084ED010A0A2B0FD8DFE803F00C1010102D
:102520001010100C100C0C003368092BE7D1054873
:102530000021E2E70223A3602046F8BD0123FAE769
:10254000B85B0020F480002000000034034B01221F
:102550001A6000229A60DA601A617047F4800020E5
:1025600013B501A904460CF0D1FA04F5804320B953
:10257000012283F8052C02B010BDDDED017ADFEDFC
:10258000096A03F6F832B8EEE77AD2ED007A67EE20
:10259000A67AB4EEE77AF1EE10FA54BF01220022D7
:1025A000E7E700BF0000C8422DE9F04F2DED068B94
:1025B00000F5005B00F5A2599BF9CE338DB00546BE
:1025C00000F5804409F1180933B100F54058D8F8F6
:1025D000C03093F8CB707FB90021A4F87C1C48462A
:1025E0000FF05CFE94F87D1C48460DB0BDEC068BE8
:1025F000BDE8F04F0FF05CBE85F0C2F80190D4F852
:10260000480B9FED958A90EDDBAA79F0CFFA09AEE1
:10261000002800F0CC80D4F8483B03F55C7393E8C5
:10262000070086E8070030468DED0B8A2AF0D8F8BF
:10263000B0EE409A28460CF0CDFB05F5964A0AF11B
:10264000240A002800F0B68050467CF0FBFE07C844
:1026500086E8070030468DED0B8A2AF0C1F8F0EECF
:10266000409AD8F89C0003681B689847122840F0ED
:10267000AA80002384F87C3CD8F89C0003685B693E
:10268000984728B1DBF8D83CB3F90830002B0DDCB3
:1026900098F99030002B09DA019BC4F8803C504631
:1026A0007CF0CCFE04F6844383ED000A94F87C3C75
:1026B0005BB1019BD4F8800C181A41F28833984220
:1026C00040F28F80002384F87C3CD4F8400B9FEDCF
:1026D000630A6C3029F086FC8DED090ACDED0A0AFB
:1026E0008DED0B1A96E8070006AB03AE9FED5C0A72
:1026F00083E8070086E80700304629F073FC284687
:10270000B0EE408AF0EE608A8DED060ACDED070A44
:102710008DED081A0CF05EFB002874D0DFED517AC5
:10272000F4EEE79AF1EE10FA94BF01250025D4F8F3
:10273000480B79F03BFA30B1DFED4A7AB4EEE79A14
:10274000F1EE10FA09D9002D64D1D8F89C00036885
:102750001B689847022864D00027D4F8480B79F00A
:1027600047FB0546002873D0B5EEC0AAF1EE10FA7B
:102770006DD5DFED3D7AB4EEE7AAF1EE10FAACBF0D
:102780000126002650467CF065FE5EB9DFED377A03
:10279000B0EEC00AB4EEE70AF1EE10FA5AD8002DF6
:1027A00008BF002794F87C1C84F87D7C17E7B0EE06
:1027B000489A3FE728460CF0DFFA00287FF444AF40
:1027C000DFED259A4DE7D8F8C03093F8CB30002BD9
:1027D0003FF452AF98F99030002BBFF64DAF012374
:1027E00048E750467CF02AFE04F68443D3ED007A95
:1027F00030EE670ADFED1E7AB4EEE70AF1EE10FA6A
:102800003FF760AF61E728460CF0B6FA05460028AE
:1028100084D18CE7D4F8480B79F0C8F9002894D11A
:102820009BE7B0EE680AA5F0DFFFF0EE408AB0EE5D
:10283000480AA5F0D9FFDFED0F7A20EE280AB4EEA2
:10284000E70AF1EE10FACCBF0127002785E7002543
:102850002E4697E73746A5E7000000009F0CB345DA
:10286000D30237390000FA420000C8C200007042AB
:102870000000484255CF7D3F38B504460CF0AAFA17
:1028800004F5A255183548B920460CF075FA0146F2
:1028900020B92846BDE838400EF082BF04F5405408
:1028A000D4F89C0003689B6C984720B9D4F89C002E
:1028B0000368DB6C98470146EBE7000030B504463F
:1028C00089B0684604F5A25514F062FE183504A8D4
:1028D00014F05EFE694628460FF01CF898B104A972
:1028E00028460FF067F870B1059B0193236800221A
:1028F000DB6C69462046984728B104F52D5001212C
:10290000343080F0FFFC09B030BD000000F580528B
:1029100092F8D426D2070BD400F54052D2F8C0204A
:1029200092F8CB1009B1FFF7C9BF03689B6C184739
:102930007047000030B587B0044602A8019114F03A
:1029400027FE04F5A25002A918300EF0E3FF019A09
:1029500018B90025284607B030BD236802A9DB6CF2
:102960002046984705460028F3D004F52D50012154
:10297000343080F0C7FCEDE7F0B5044685B004F5CF
:10298000A256684618360F46154614F001FE6946F1
:1029900030460FF00FF810B9002005B0F0BD3946F1
:1029A00030460EF06FFE0028F6D0002DF5D004F56D
:1029B0008054284694F8D43643F0020384F8D43681
:1029C000EBE700002DE9F04F2DED0A8BBDB004467A
:1029D00024220D4618A80021A8F022FB2422002161
:1029E00021A8A8F01DFB242200212AA8A8F018FB8A
:1029F00004F540562422002133A8A8F011FB00233F
:102A0000CDE90D330F9396F8913013F0080839D1C2
:102A100004F5005943F0080399F8CC2C079286F886
:102A2000913015F0E9FE90F9213003B390F840336E
:102A3000EBB104F25457384615F0EEFDC34694F856
:102A400076355FFA8BF18B421FD9384615F0C2FDFF
:102A50000BF1010B82460028F1D1C94A0221284618
:102A600053F028FD96F891306AF3C30308E0C54A95
:102A70000221284653F01EFD96F891306FF3C303F0
:102A800086F891304FF001083EE304F537533433B4
:102A9000012118460BEE903AFBF77EF8824608B902
:102AA000B94ADBE720460BF0B3FED9F8D83CB3F9BE
:102AB00008A0BAF1000F01D0B44AD9E796F99030D6
:102AC000002B01DBB24AC9E7204601F087FE04F57E
:102AD00043532C33184652460CA90CEE103A12F010
:102AE000FFF8002814BF022301230393F123CDE94B
:102AF000133A8F210A23CDE9003113AA287CADF8BF
:102B000054A003234D2151F0A3FAA24B9FEDA28ABA
:102B100001225A720621A14A284653F0CBFC039B9E
:102B2000022B0CBF9E4A9F4A062128464FF0000AFE
:102B300053F0C0FC89F88AA35146384615F0B6FC1C
:102B400094F876355FFA8AF18B420CD913AA38468D
:102B50008DED138A8DED148A8DED158A0AF1010A27
:102B600015F026FBECE7384615F056FD4FF0000A4D
:102B70004FF07C0B94F876255FFA8AF94A4519D90B
:102B80004946384615F006FAC0B20BFB00403CAA95
:102B90000C2300F2E45003FB092C07C8ACF1900CA5
:102BA0008CE807003CAA02EB890909ED2F8A0AF19B
:102BB000010ADFE741F288310AA821F0D1FFD6F8F7
:102BC000C0009FED759A03689FED77AA9B6ADFEDC1
:102BD00077AA9847D6F8C00001217DF0DBFB744B43
:102BE0001B680293D86A036801211B68984784F028
:102BF000C7FD059084F0C4FDF0EE499A06900026CA
:102C000004F50059079A99F8CC3C934240F0D880DB
:102C100094F89618384615F0DDFC002800F0D080B6
:102C200004F5405BDBF8C03093F8CB300493002B05
:102C300000F0C68041F288310BA821F091FF84F0AA
:102C40009FFD059BC01A132840F2D98084F098FD9F
:102C5000059020460BF0DCFD5AF064F8824659F0EE
:102C6000FBFFD9F8D83CDBF8C000B3F9083000EE20
:102C7000103AB8EEC00A20EE0A0A7FF065F8504616
:102C800059F0F2FF384615F0C7FC1CEE100A12F09E
:102C900011FAD9F8D83CDFED400AB3F9083000EE5C
:102CA000103AB8EEC00AA22020EE0A0AB7EE001AC7
:102CB00025F08AFFB4EEE90AF1EE10FA1CEE100AD4
:102CC0004FF000020CA958BFF0EE409AF0EE408A97
:102CD00012F006F808B900230C939DED0C8ADFED85
:102CE000357AB4EE498AF1EE10FAF4EEE78A48BF7D
:102CF000B0EE498AF1EE10FA80F28F809FED2E9AA5
:102D0000DFED2E8A4FF0000A94F876355FFA8AFBE1
:102D10005B4540F296814FF00C0918AB09FB0BF9AB
:102D200003EB0900B0EE490A29F05CF95946384630
:102D3000CDED110A8DED121A8DED100A15F02AF95C
:102D40007C23C0B203FB0040B0EE680A00F2E450FE
:102D500029F048F93CAB13A910A899448DED130A4A
:102D6000CDED140A8DED151A29F010F90AF1010ABA
:102D700009ED240A49ED230A09ED221AC4E700BF30
:102D8000E54C0C08D44C0C08E3600C08F34C0C0820
:102D9000054D0C08A582002000000000104D0C0815
:102DA000254D0C088FF60B086F12833A0000C842BD
:102DB000E880002000000034A4707D3F0AD7233C47
:102DC00004F54059D9F8C00003689B6A9847D9F8C0
:102DD000C00000217DF0DEFA029BD86A0368002162
:102DE0001B689847002E40F05F812846C94A05219C
:102DF00053F060FB3146384615F058FB70E1029BFA
:102E0000986A036805215B6898470BA821F0B4FE17
:102E1000B0EE498AB0EE489AF2E64FF000094FF062
:102E20000C0B04F5B26A94F876255FFA89F39A429E
:102E300022D919463846089315F0ACF8089B0BFBCD
:102E400003F13CAB5A18A2F16C034FF07C0CC0B2FA
:102E5000CDE908320CFB00A018AB1944543029F01E
:102E6000ABF8089B099A09F1010902ED1B0AC3EDB1
:102E7000010A83ED021AD6E7039B012B4FF0000AEB
:102E800046D19FEDA5BA9FEDA59A4FF00C0B94F893
:102E900076355FFA8AF6B34240F286800BFB06F67F
:102EA0003CAB03EB0609A9F14803089321ABB0EE54
:102EB000680A981929F0A6F8089B09ED120AC3EDD3
:102EC000010A83ED021A33ABB0EE4B0A981929F0D0
:102ED00089F82AAB98198DED100AB0EE490ACDEDAC
:102EE000110A8DED121A29F07DF813A910A88DEDA5
:102EF000130ACDED140A8DED151A29F05DF80AF1CB
:102F0000010A09ED090A49ED080A09ED071ABEE7A9
:102F10009FED819A9FED81BAF0EE088A94F876359C
:102F20005FFA8AF94B4564D99DED0C0AB4EEE80AC4
:102F3000F1EE10FA35DB0C2303FB09F93CAB03EB94
:102F4000090621AB03EB090029F05CF833AB46ED31
:102F5000110A06ED101A06ED120A03EB0900B0EE95
:102F6000490A29F03FF82AAB03EB09008DED100A5E
:102F7000B0EE4B0ACDED110A8DED121A29F032F8A0
:102F800013A910A88DED130ACDED140A8DED151AB5
:102F900029F012F806ED090A46ED080A06ED071AAF
:102FA000049E0AF1010AB9E74FF000094FF00C0A3C
:102FB00094F876355FFA89F6B34241D933AB0AFB10
:102FC000063029F00DFC1BEE900AF0EE408A73F0FB
:102FD000B3FE07EE900AB8EE677A3CABC8EE877A8C
:102FE00003EB860609F1010967EEAA7A46ED2F7A0E
:102FF000DEE74FF0000A4FF00C0B94F876355FFADD
:103000008AF94B451DD933AB0BFB093029F0E8FB9E
:10301000C8EE297A0AF1010A1BEE900A67EE808A4F
:1030200073F08AFE07EE900AB8EE677A3CABC8EE02
:10303000877A03EB890967EEAA7A49ED2F7ADCE7F4
:10304000049E84F09DFB069BC01AB0F5FA7F27D939
:1030500084F096FB04F50053DDED0D7AD3F8D83CEF
:103060000C9A1B891392FCEEE77A339A1492ADF80E
:103070005C30349A159217EE903A359A1692ADF864
:103080005E30F0221423CDE90032B121069013AA5C
:10309000287C50F0DDFF6CF09DFC297C6CF094FBEB
:1030A0000BA821F069FDB5E60399384615F0FEF945
:1030B00000264FF00C0A94F87635F1B28B4207D90E
:1030C00033AB0AFB0132384615F072F80136F2E7ED
:1030D000384615F07FF8124A0621284653F0EAF9DF
:1030E000104B002520465D7201F06AFB04F50E507E
:1030F0000A3044F041FC99F8913065F3C30389F834
:1031000091300AA821F038FD40463DB0BDEC0A8B55
:10311000BDE8F08F05E20D08A4707D3F0AD7233C7F
:103120002D4D0C08A58200207FB54C4BD3F8983C60
:10313000DB07044600F18F8000F54055D5F8C0301C
:1031400093F8C120002A40F0868093F8CB30002B02
:103150007ED095F99030002B7ADB00F5804696F80A
:10316000883C002B77D1D6F8400B9FED3D0A6C30A0
:1031700028F038FFCDED020A60EEA00ADFED397AC3
:103180008DED010AE0EE000A8DED031AF4EEE70A78
:10319000F1EE10FA5CDCD6F8403B9FED337AD3EDCC
:1031A000377AF4EEC77AF1EE10FA04D5D5F8C030CC
:1031B0001B7A002B4CD0B5EE007AF4EEC77AF1EE14
:1031C00010FA45D404F5964024307CF043F9DFED45
:1031D000277AB4EEE70AF1EE10FA39D8D6F8403B78
:1031E0009FED237AD3ED367A67EE877AB3EE0E7AC7
:1031F000F4EEC77AF1EE10FA2ADA1E4AB4F9A410F6
:10320000138801339BB2138019B9B4F8A210A4F843
:10321000A410B4F8A41099421DD8002616804DF0D1
:1032200023FF012219214DF07BFED5F8C000036871
:103230005B699847431C04F539500F4A31463430D6
:103240004FF00EFFD5F8C030012283F8C12002E014
:10325000084B00221A8004B070BD00BFB84B00209C
:103260009F0CB3454054094A6666663F000000B4AF
:10327000E02E65422E810020444D0C0870B52DEDE6
:10328000028B4A4BD3F8983C9B0784B004461FD46A
:1032900000F58045DFED468AD5F8400B03681B69D1
:1032A0009847D0ED017AF4EEE87AF1EE10FA0FDBF0
:1032B00004F5405304F59946D3F8C02092F8C110A4
:1032C0000C3649B1002303A9304603934FF0E0FACE
:1032D00004B0BDEC028B70BD92F8CB20002AF1D077
:1032E00093F99030002BEDDB95F8883C002BE9D169
:1032F000D5F8400B03681B699847D0F8A430D5F87F
:10330000400B039303681B69984704F58C7200F126
:10331000A40130464FF02AFBDDED037AB0EEC08AFF
:10332000F0EEE77AF4EEC87AF1EE10FA03D503A9CD
:1033300030464FF0ADFAD5F8400B03681B6998474B
:10334000D0ED040AF4EEE80AF1EE10FAC0DBF6EE76
:10335000087A60EEA77AF4EEC87AF1EE10FA1DD57D
:1033600084F00EFAD5F8983C42F21072C31A9342D8
:10337000AED9DFED107AC5F8980C68EE277A04F51F
:10338000395417EE900AF9F7BFF83434CDE900014B
:10339000094A002120464FF063FE99E79DED030A9C
:1033A00025F00EFB0028DBD192E700BFB84B0020D0
:1033B000000000340000C842604D0C0810B50446FF
:1033C00000F5984030305CF031FA04F59840012166
:1033D000BDE81040503064F0FBBE0000F8B500F5C9
:1033E0008045044695F9303C4BB300F5405695F8BE
:1033F000442C96F89030DB43C3F3C01363F3C3024D
:1034000000F5984700F5964085F8442C24307CF070
:1034100021F8DFED3E7A303720EE670A38465CF05F
:1034200085FA95F8883C53B938465CF02BFAD6F803
:10343000C03093F8CB301BB9354B00221A80F8BD51
:1034400095F8443CDB07FAD4D6F89C0003689B6BE4
:1034500098470028F0D096F99030002BECDB2C4EEA
:1034600033884BB9B5F9363C33B1642213FB02F310
:10347000D5F8182B9A42E2DB38465CF073FAD5F89F
:10348000403B9FED247AD3ED367A67EE877AB3EE30
:103490000E7AF4EEC77AF1EE10FA05D83388002BD5
:1034A000CDD0013B3380CAE7B4F9A4301BB9B4F8DE
:1034B000A230A4F8A4303388B4F8A420B4F9A4004E
:1034C000154993423CBF013333803388D5F8F02A45
:1034D000012B01D10A60B2E709689142ACDD18B94D
:1034E000B4F8A220A4F8A420B4F8A4209A42A6D844
:1034F000002333804DF0B8FD02220C214DF010FD69
:103500002046BDE8F840FFF759BF00BF0AD7233C6B
:103510002C810020E02E65422881002008B500F5AE
:10352000804292F9303C6BB300F5405393F99030F0
:10353000002B0EDA00F53950134A062134304FF0D3
:103540008FFD4DF091FD0322BDE808400F214DF0A5
:10355000E7BCB2F9363C8BB1D2F8182B642113FBCF
:1035600001F39A420ADA00F53950084A0121343051
:103570004FF076FD4DF078FD0222E5E7BDE808400A
:10358000FFF71CBF08BD00BF784D0C088A4D0C0822
:10359000F0B52DED028B00F540555A4ED5F8C030F0
:1035A00093F8CB308DB0044643B195F99030002BA1
:1035B00004DB00F5005393F9A6332BB900233380C5
:1035C0000DB0BDEC028BF0BD00F5804797F8883C4C
:1035D000002BF3D101F06AFB002879D1D5F89C00CB
:1035E00003689B6B98470028E8D004F59540743039
:1035F0004FF070F929F0F4F8F0EE087AB4EEE70A2B
:10360000F1EE10FAF0EE408AD8DA04F5A253D3EDC9
:10361000997A93ED980A20EE270AA5F09FFADFED3C
:103620003A7A20EE270AB2EE0E7AB4EEC70AF1EE2D
:1036300010FAC3D9D7F8403B93ED368A28EE278A93
:10364000F3EE0E7AB4EEE78AF1EE10FAB6D904F58D
:10365000A250002309A9183009930A930B930EF086
:10366000B5F900283DD13388B4F9A42001339BB2C9
:103670003380002A40D0B4F8A420B3EB420F9FDB84
:103680004DF0F2FC01220C214DF04AFC1F4B0022B0
:1036900018EE900ACDE90623F8F736FF1C4BCDE96A
:1036A0000401002218EE100ACDE90223F8F72CFFDE
:1036B00004F539543434CDE90001164A204600217E
:1036C0004FF0CEFC01220C211348FAF77DFC77E77E
:1036D000D5F89C000368DB6C984700287FF47EAF28
:1036E0006CE709A829F07CF8F2EE047AB4EEE70A58
:1036F000F1EE10FAB7DB61E7B4F8A220A4F8A42039
:10370000B9E700BF24810020E02E65420000084098
:1037100000003E40A04D0C08AC590020F0B52DED46
:10372000028B8BB0002307930893099305AB0446E3
:10373000019300F5A25007AB009302AA04AB03A9C2
:1037400018300EF05BF804F50056054686F8680E52
:1037500028B9002528460BB0BDEC028BF0BD84F0E3
:1037600003F8D6F86C3E9FED2F7AC31A07EE903A15
:10377000F8EE677A074667EE877A04F5395006AAAD
:1037800002A90430CDED067A4FF0F0F804F5395077
:1037900006AA03A910308DED020A4FF0E7F804F5F0
:1037A000395006AA04A91C308DED030A4FF0DEF84B
:1037B00096EDEA8AC6F86C7EB5EEC08AF1EE10FA94
:1037C000C7D9DDED080A9DED070AA5F093F8DDEDF8
:1037D000090AA5F08FF8DDED037A38EE087AB4EE29
:1037E000C08AF1EE10FAB4EEE77A94BF0123002309
:1037F000F1EE10FA0AD80233DDED027AB4EEE78A70
:10380000F1EE10FA0AD8002BA3D0A3E7B4EEE78AB2
:10381000F1EE10FA9CBF0133DBB2EDE7012B99D832
:1038200097E700BFBD37863570B500F540550446B3
:1038300095F8B53043F0040385F8B5304DF014FC2D
:10384000012211214DF06CFBD5F8C03093F8CB303C
:10385000002B43D0D5F89C0003681B6898470928C3
:103860000AD1204607F0E8FA30B104F5A440183038
:10387000BDE8704007F0C8BA194BD3F89C00036844
:103880001B69984704F5005340B993F9A533032BFE
:1038900024D10621204607F0BBFA0DE093F9A513C9
:1038A0000229F6D195F8B530DB07F2D4062220467E
:1038B00002F00EF80028ECD00A4BD5F89C0001224B
:1038C0005A7303681B6C9847034604F53950064A3F
:1038D000BDE87040022134304FF0C2BB70BD00BF64
:1038E000B85B0020A5820020D44D0C0808B500F577
:1038F000405292F8B530590717D56FF3820382F81A
:10390000B5300A4B5A7B42B1002200F539505A7348
:103910000221074A34304FF0A3FB4DF0A5FBBDE870
:103920000840002211214DF0FBBA08BDA5820020FD
:10393000F84D0C08F0B5054685B005F5A257684668
:10394000183713F025FE694638460EF033F880B17B
:1039500005F50053D3EDEA7A374CF5EEC07AF1EE77
:1039600010FA08D8354A002328462380D373FFF77E
:10397000BDFF05B0F0BD2846FFF7D0FE064628463D
:103980000BF0FAF910B928460BF0D0F9A378002E05
:1039900018BF00200343DBB2A370002BE9D063788B
:1039A000A8BB83BB23780133DBB2082B237003D180
:1039B0004EB338460DF08EFF2378092B02D13846DE
:1039C0000DF080FF2378092B1DD94FF485732380D8
:1039D0004DF04AFB022210214DF0A2FA83F0D0FEF6
:1039E0006368C01A47F23053984209D905F5395037
:1039F000134A022134304FF033FB83F0C1FE606084
:103A00002846FFF711FF0D4B6278DA73B1E726788D
:103A1000002EF8D0013EF6B22670002BF3D0002E17
:103A2000F1D166704DF020FB324610214DF078FA4E
:103A30002846FFF75BFFE6E730810020A5820020E3
:103A4000104E0C0800F5405393F8B5305B0701D5D4
:103A5000FFF7EABE7047000073B5044600F5A250B8
:103A600001A9183004F500550DF012FDD5F8303ECF
:103A7000834206460CD004F58043D3F8400B76F021
:103A800065FEC5F8306E4DF0EFFA3E214DF028FA94
:103A900004F5805695F9341E96F9682796F868372C
:103AA00091421BD0FF2B19D004F58043D3F8400B73
:103AB00076F04CFE96F8683785F8343E4DF0D4FA2F
:103AC00095F8342E18214DF02BFA04F5395095F95C
:103AD000343E034A042134304FF0C2FA02B070BDC4
:103AE000204E0C082DE9F0438FB0054683F048FEC8
:103AF0000023059306930793089309930A930B9366
:103B00000C930D9305F5A25804AB019308F1180826
:103B100003AB009306460BAB08AA05A940460DF07F
:103B20004DFEDFED487A9DED077AB4EEE77AF1EECF
:103B300010FA074632DB9DED0A7AB4EEE77AF1EE31
:103B400010FAACBF0124002405F50059404699F84D
:103B5000683E002B08BF00270DF042FE8046FFB9EB
:103B6000444699F9343C012B2BD174B105F54053EF
:103B7000D3F8C02092F8CB403CB1D3F89C00036846
:103B80005B69984780F00100C4B299F8383ECBBB1E
:103B9000CCB9C9F83C6E0FB0BDE8F0830024D3E780
:103BA000002CDDD005F5395010304EF06FFE90ED51
:103BB000007AF7EE007AB4EEE77AF1EE10FAD0DC94
:103BC000CEE70024E1E7D9F83C0E301AB0F57A7F51
:103BD000E1D9C9F8403E012405F5804389F8384E03
:103BE000D3F8483B83F80C444DF03EFA22461D21A1
:103BF0004DF096F9144A05F53950022134304FF052
:103C00002FFAC8E714B1C9F8406EC4E7D9F8400EDE
:103C100043F69823361A9E42BDD905F58043C9F86C
:103C20003C4E89F8384ED3F8483B83F80C44C9F829
:103C3000404E4DF019FA22461D214DF071F9034A0C
:103C4000D9E700BF00000034384E0C08524E0C0873
:103C50000B4B10B5012204465A7283F091FD04F516
:103C60008042D2F8743CC31A142B08D9C2F8740CE1
:103C700004F5A0500430BDE8104040F0F5BD10BD83
:103C8000A58200202DE9F743044604F5405600F5CF
:103C90000E50002320300DF107018DF8073044F05D
:103CA000E1FBD6F8C00090F9C030026883B3083B4E
:103CB000DBB2012B95692BD93221A84704F1100002
:103CC00011F072FB204B04F539581F684FF00009C2
:103CD00008F13408F86A0368DB69984701281ED1A7
:103CE00083F04EFD41F28733A0EB09029A4205466C
:103CF00005D9164A062140464FF0B2F9A94620469A
:103D0000FFF7A6FFB86A036803215B689847E1E7FD
:103D100004F500539269B3F8B4139047CEE701213C
:103D2000D6F8C0007CF036FBD6F8C0000368DB6A2A
:103D3000984758F085FCF86A03681B68012103B0B6
:103D4000BDE8F043184700BFE8800020704E0C0823
:103D500070B5044600F539502DED028B184A194E06
:103D60009FED198A062134304FF07AF92046FFF78B
:103D700089FF2046FFF76CFF20460AF049FD3368B3
:103D8000986A036803215B68984758F0CBFF0546A3
:103D900058F062FF04F50053D3F8D83CB3F908306B
:103DA00000EE103A04F54053B8EEC00AD3F8C00054
:103DB00020EE080A7DF0C8FF284658F055FFD8E7E6
:103DC000944E0C08E88000206F12833A2DE9F047EA
:103DD000044600F539502DED028B2A4ADFF8AC90ED
:103DE000062134304FF03CF92046FFF74BFF58F0E6
:103DF00099FF04F54056054658F02EFFB7EE000A2D
:103E0000D6F8C0007DF0A0FF284658F02DFF83F0C3
:103E1000B7FC41F2873A074683F0B2FCC01B50451D
:103E2000D9F8008017D99FED188A284658F014FF5A
:103E3000B0EE480AD6F8C0007DF086FF284658F05C
:103E400013FF2046FFF704FFD8F82800036803217A
:103E50005B689847E9E7284658F0FEFEB7EE000A8F
:103E6000D6F8C0007DF070FF284658F0FDFE2046D1
:103E7000FFF7EEFED8F82800036803215B68984737
:103E8000CAE700BFC44E0C0800000000E880002014
:103E9000F7B500F540530446D3F8C03093F9C0306D
:103EA000032B2BD0364E652500F58047013D15F0DC
:103EB000FF050CD0D7F8703C4BB93368986A03689B
:103EC00014215B68984720460AF0A2FCEEE704F54F
:103ED000375001213430F9F75FFE04F5005378B90B
:103EE00093F9A03353B1092B08D08DF8070004F5DE
:103EF0000E500DF10701203044F0B4FA03B0F0BDCC
:103F000093F9A023032A34D8DFE802F002252D30EC
:103F1000D3F8D83CB3F9082040F2B5339A422ADDF1
:103F200004F50E5001250DF1070120308DF80750E2
:103F300044F098FA04F53950124A022134304FF017
:103F40008FF8114B5D720E4B1C68A06A0368052147
:103F50005B689847F9E7D3F8D83CB3F9082040F2FA
:103F6000B5339A4207DD2046FFF7F2FE2046FFF701
:103F70002DFF092AC2D000238DF80730B7E700BF14
:103F8000E8800020E84E0C08A582002000F539509A
:103F90000B46024A042134304FF062B8084F0C0837
:103FA00010B504464DF060F8002205214CF0B8FF32
:103FB00004F53950034ABDE81040042134304FF075
:103FC0004FB800BF144F0C0813B50B464AB100F5AB
:103FD000395000920421054A34304FF041F802B0C4
:103FE00010BD02B0BDE81040FFF7D0BF2C4F0C0849
:103FF00008B500F53950064A042134304FF030F846
:104000004DF032F8BDE80840002208214CF088BF8E
:10401000404F0C0838B504460D4683F0B1FB04F55B
:1040200040533DB9D3F8AC20C3F8B0000AB9C3F887
:10403000AC0038BDD3F8B020801A642884BF0022B9
:10404000C3E92B22F5E7000037B5044600F596409A
:1040500024307BF0E5F904F54052C0F3803592F846
:104060009230C3F34001A9421DD065F3410304F52A
:10407000395482F8923034346DB14CF0F5FF02229D
:104080000B214CF04DFF094A0221204603B0BDE848
:1040900030404EF0E5BF4CF0E7FF2A460B214CF0D4
:1040A0003FFF034AF0E703B030BD00BF584F0C0894
:1040B000744F0C0838B50A460C460621054601F037
:1040C00007FC28B1054A137843F00803137038BD84
:1040D00021462846BDE8384006F09ABEC48200203A
:1040E00038B50A460D461521044601F0F1FB28B10A
:1040F000094A137843F00803137038BD04F53950AA
:1041000004213430054A4EF0ABFF29462046BDE875
:10411000384006F07DBE00BFC4820020844F0C08EA
:1041200038B50A460D461521044601F0D1FB28B1E9
:10413000094A137843F00803137038BD04F5395069
:1041400004213430054A4EF08BFF29462046BDE855
:104150003840FFF7AFBF00BFC4820020AC4F0C084F
:1041600038B50A460D461B21044601F0B1FB28B1C3
:10417000094A137843F00803137038BD04F5395029
:1041800004213430054A4EF06BFF29462046BDE835
:104190003840FFF78FBF00BFC4820020C24F0C0819
:1041A00038B50A460D461121044601F091FB28B1AD
:1041B000094A137843F00803137038BD04F53950E9
:1041C00004213430054A4EF04BFF29462046BDE815
:1041D000384006F01DBE00BFC4820020D44F0C083A
:1041E00010B500F5405494F892309A0623D4D4F8D0
:1041F0009C0003681B689847032808D005D802284C
:104200000ED194F89000C00914E01B28F9D194F85D
:10421000900000F0A000A0F180035842584109E04E
:10422000B4F8900020F4FE4020F07F0080B2003807
:1042300018BF012010BD0120FCE7000038B500F5D3
:104240004055044695F8B530184A43F0080300F588
:10425000395085F8B530022134304EF001FF4CF072
:1042600003FF012217214CF05BFE2046FFF7B8FF49
:1042700040B104F537500122BDE8384015213430F3
:10428000F9F7A2BED5F89C0003681B68984706287A
:1042900006D104F5A6403030BDE8384007F0C4BF71
:1042A00020460B21BDE83840FFF704BFE84F0C085B
:1042B00070B500F54055D5E92B239B1A41F28832A1
:1042C0009342064611D9D5F89C0003681B6D9847A8
:1042D000044695F8B530C3F3C003A34213D034B1FC
:1042E0003046BDE87040FFF7A9BF0024F1E74CF06D
:1042F000BBFE224617214CF013FE95F8B53064F34F
:10430000C30385F8B53070BD0B46013B1146062B43
:1043100018D8DFE803F00406080A0C13150006F0AD
:1043200077BDFFF7C7BEFFF7FBBEFFF7D9BE00F5AD
:104330003750012214213430F9F746BEFFF710BF81
:10434000FFF72EBF70470000F8B5044604F500578C
:104350004CF08AFE012205214CF0E2FD97F88A33E9
:10436000072B98BF304A204694BFD55C0125FFF744
:1043700037FF68B12D4A2E492046FFF725FE04F588
:104380003750012210213430F9F71EFE002514E0C9
:1043900004F54056D6F89C000368DB6C984798B14A
:1043A00096F8153683B196F91436012B0CDC214AA8
:1043B00021492046FFF708FE012529462046032211
:1043C000BDE8F840FFF7A0BFD6F89C000368DB6C9F
:1043D000984718B1D7F8383C190715D4D6F89C007F
:1043E00003681B689847032803D1D7F8383CDA07DD
:1043F0000DD4D6F89C0003685B6A984768B90C49ED
:104400002046FFF7C3FDD8E70A4A0949D1E70B4A1E
:1044100007492046FFF7D8FDB8E7D7F8383C5B07D7
:10442000EDD5074AF4E700BFD0500C0808500C083F
:1044300012500C0818500C082B500C083B500C085C
:104440004B500C0838B5044615464CF00DFE0122C1
:1044500006214CF065FD2046FFF7C2FE98B104F539
:104460003750012207213430F9F7AEFD144A1549BF
:104470002046FFF7A9FD0025294620460422BDE875
:104480003840FFF741BF04F54053EDB2D3F89C002C
:104490000368DB6C984768B104F50053D3F8383CE7
:1044A0001B0707D535B1084A06492046FFF78CFDA2
:1044B0000125E1E703492046FFF768FDDCE700BF7F
:1044C00008500C086A500C0818500C082DE9F041EF
:1044D000044604F500574CF0C7FD012208214CF0BA
:1044E0001FFD56F00DFE97F87933072B98BF384A19
:1044F00004F5405698BFD55CD6F8C03093F8CB8011
:1045000088BF0225B8F1000F0BD132492046FFF7D2
:104510003DFD0025294620460522BDE8F041FFF774
:10452000F3BE2046FFF75CFE60B104F53750012270
:1045300012213430F9F748FD274A26492046FFF773
:1045400043FDE6E7D6F89C000368DB6C984768B14A
:1045500096F8153653B196F91436012B06DC1F4A2E
:104560001F492046FFF730FD0125D3E7D6F89C0010
:104570000368DB6C984718B1D7F8383C190713D497
:10458000D6F89C0003681B689847032803D1D7F826
:10459000383C9A070BD4D7F8383CDB0609D40D49D0
:1045A0002046FFF7F3FCB5E70C4A0A49D9E70D4A64
:1045B000C3E7D6F89C000368DB69984706460028E5
:1045C000EDD1094A03492046FFF7FEFC3546A1E735
:1045D000D8500C08533C0C0808500C0818500C0814
:1045E00064500C0872500C0887500C08F8B500F5A0
:1045F0000055044695F97933B3B300F54056376A50
:1046000097B383F0BDF805F5496595ED000ADFED38
:10461000177A9FED171ADFED170AC71B20EE270A3E
:104620008D2024F0D1FABCEEC00A10EE103A9F4261
:104630000CD296F8B5309A0716D520460021F9F726
:104640001DFE2046BDE8F840FFF7D2BC0CD996F815
:10465000B5309B0708D420460121F9F70FFE20460C
:10466000BDE8F840FFF732BFF8BD00BF00007A4454
:104670000000804F000000002DE9F341074600F5DF
:10468000964024307AF0CCFE07F54054C0F38048C1
:10469000019083F075F894F8B830434545460646D6
:1046A0000DD007F5395084F8B8803430002D41D052
:1046B0003B4B3C4AC4F8BC6002214EF0D1FC94F85C
:1046C000B83007F5005843B394F8B9302BBBB8F9AC
:1046D000A63C9FED350A9FED351ADFED350A07EE52
:1046E000903AF8EEE77A40F2571027EE800A24F06D
:1046F0006BFABCEEC00AD4F8BC0010EE103A361AC1
:104700009E420AD9012307F5395084F8B930294A65
:10471000234B022134304EF0A3FC98F9A53C002B2A
:1047200094F8B5300DDC6FF3451384F8B53002B062
:10473000BDE8F0811A4B204AC4F8BC8084F8B980E7
:10474000BAE7C3F34012AA42F1D065F3451384F8E7
:10475000B5309B06EBD5194BD3F89C0003681B6959
:1047600098470028E3D04CF07FFC01221F214CF039
:10477000D7FB3846FFF734FD48B107F53750012223
:104780002121343002B0BDE8F041F9F71DBC98F8A2
:10479000A51C3222384602B0BDE8F041FFF7B4BD97
:1047A000A0500C08AF500C0800007A440000804F65
:1047B00000000000C5500C08BA500C08B85B00207F
:1047C00008B5044B01221A7082F0CEFF024B18602C
:1047D00008BD00BF398100203C810020014B002230
:1047E0001A707047398100202DE9F041044682F0AB
:1047F000BBFF2A4BB4F8BE201988294E91420546CA
:104800000ED01A80274B18603378A3B1002434707F
:104810004CF02AFC22461321BDE8F0414CF080BB4D
:104820003378214FDBB93B782BB11E4B1F4A1B68F5
:10483000C31A934201D8BDE8F0810123337004F517
:104840004053D3F8C00090F8CB3013B103689B6A93
:1048500098474CF009FC012213214CF061FB3B7896
:10486000002BE8D03378002BE5D00E4A10491368AE
:10487000EB1A8B42DFD904F540541560D4F8C00020
:1048800090F8CB30002BD6D000217BF083FDD4F8FC
:10489000C0000368BDE8F0415B6A18473A81002018
:1048A000388100203C8100203981002080841E0056
:1048B00040420F002DE9F84300F5405500F500583F
:1048C0000446D5F89C0098F88C720368DB6C984716
:1048D000014650B995F99030002BA5BFD5F8C030EE
:1048E00093F8CB00012180F0010104F5095909F189
:1048F0001009484660F0AEFAD5F8C03093F8CB30D6
:104900000646002B7BD0002865D03E4B93F99030B3
:10491000002B04DB02463C4948465FF075FE98F9DF
:10492000567257B195F99030002B0EDA04F53750D6
:1049300001220F213430F9F747FB4CF095FB32464A
:10494000BDE8F84309214CF0EBBAD5F89C000368A8
:104950005B69984758B195F99130002B07DA95F8C3
:10496000B530DA0703D498F88C32DB07DED5314650
:10497000484660F0D5FADFED257AB4EEE70AF1EEAD
:1049800010FA05DD0A220921204600F0A1FFD4E734
:10499000023F032F11D801A353F827F085490108DE
:1049A000AD490108CB490108D14901080A22152166
:1049B000204600F08DFF0028BFD10A2206212046A4
:1049C00000F086FF0028B8D1DCE70A221121F6E7C3
:1049D0000A221521F3E797B198F88C327BB9094B7D
:1049E00093F99030002B06DB04F53950084A052175
:1049F00034304EF035FB4CF037FB0022A0E7BDE829
:104A0000F88300BFB85B0020E0500C080000C842EB
:104A1000E9500C0870B500F5005300F596452435B3
:104A200086B093F8381E044628467AF0A7FC02A800
:104A300012F0AEFD04F5A25002A918300CF06AFF86
:104A400004F58043049AC3F81C2B059AC3F8202B65
:104A500028467AF0E5FC82061AD528467AF0EEFC64
:104A600004F59645FDEEC07A143504F5805417EE32
:104A7000901A0222284617EE906A12F08FFD94F8E1
:104A8000D436DB0706D401223146284612F086FDD3
:104A900006B070BD0121284612F012FE0028F2D0A7
:104AA000F6E7000070B500F5804486B0B4F8A43C89
:104AB0008B420D46164603D1D4F8A03C934221D038
:104AC00082F05EFED4F89C3CC31A132B1AD9C4F8AA
:104AD000A06CA4F8A45CC4F89C0C4CF0C5FA044685
:104AE00082F056FE084B094A1B68CDE90453084B77
:104AF0000193084B0093CDE90201074B074920467B
:104B00004CF054F806B070BD4081002000510C08F4
:104B100018510C08D8260C08140A0C0813510C085C
:104B200038B500F540540D4694F89130C3F3801326
:104B30008B420BD021B14CF097FA11214CF0D0F9F7
:104B400094F8913065F3861384F8913038BD0000F5
:104B5000F0B52DED048B00F540568BB0D6F8C03083
:104B600093F8CB30054600F58044002B67D096F9CA
:104B70009030002B63DBD6F89C0003685B69984794
:104B8000002861D1D4F8400B9FED440A6C3027F027
:104B900029FA0AAACDED080A8DED091A8DED070A4A
:104BA00012E9070004AB01AF83E8070087E80700BC
:104BB000384626F085FFD4F8403B05F59540743023
:104BC000D3ED368AB0EE409A4DF084FE27F008FE11
:104BD000D4F8483BD6F89C00D3EDDB9A0368DB6C35
:104BE000B0EE408A9847DFED2E7AB4EEE79AF1EE08
:104BF00010FA02DC96F898300BB100283AD0DFEDBD
:104C0000297A68EEA78AF3EE0E7AF4EEE78AF1EEDF
:104C100010FA2FDCF0EE087AB4EEE78AF1EE10FA23
:104C200028DCF5EEC09AF1EE10FA23DAD4F8400B46
:104C300003689B6F98470BB0BDEC048BF0BDD4F8B4
:104C4000400B03689B6F0FE005F50055D4F8400B4F
:104C5000D5F8D82C0368B2F90820002A03DCD6F86E
:104C60009420022AEED1DB6F0BB0BDEC048BBDE8C3
:104C7000F0401847D4F8405BDFED0B0A2B68D3F8FF
:104C80008060D4F8483B40F2AB1093EDC90AB7EE10
:104C9000001A23F099FF2846B047CCE79F0CB34594
:104CA0000080BB44E02E65420000000000F540504B
:104CB00090F89800704700002DE9F04100F540554C
:104CC000064695F89030B1EBD31F0C4648D0254BE3
:104CD00000221A6000293FD04CF0C6F912214CF096
:104CE000FFF895F8903064F3C71385F8903084F09E
:104CF00001086AF0AFFF41466AF088FF06F50057E9
:104D0000B8F1000F06D097F80E331BB982F038FDCA
:104D1000C7F8100387F80E8314B3B7F85C335B074A
:104D20001ED5D5F8C03093F8CB30CBB1D5F89C0068
:104D300003685B69984798B9D5F89C0003682021FF
:104D40009B69984760B106F537500122BDE8F041F4
:104D50000D213430F9F738B94CF086F91C21BEE743
:104D6000BDE8F081408100202DE9F04F2DED0A8B48
:104D700000F540558DB0D5F8C03093F8CB600446AF
:104D800000F580471EB90121FFF796FF0BE095F96A
:104D90009020002A65DAD5F89C0003689B6C984740
:104DA0000646002841D04FF0000B95F99020B24EF6
:104DB000002AC0F25581D6ED007AB4F9A420B8EEED
:104DC000677A1AB9B4F8A220A4F8A420B4F8A430E1
:104DD000DFEDAA6A07EE903AF8EEE77A67EEA67A78
:104DE000B4EEE77AF1EE10FAACBF012100212046C3
:104DF000FFF796FE95F99020002A95F89120B8BF0C
:104E00004BF0010B530697F8882C48BF4BF0020B70
:104E10000AB14BF0080B3268594620460DB0BDEC84
:104E20000A8BBDE8F04FFFF73DBED5F8C0302046F5
:104E300093ED0C8AF9F7F2FAB4EEC80AF1EE10FA23
:104E4000B1D5D5F8C03093F8A130032BABD14AF0DF
:104E50005DFC4FF4801142224AF010FC314620469E
:104E600092E797F888ACBAF1000F03D0824A00238A
:104E7000136098E7D7F8400B93F8079003685B6FCF
:104E8000984780460090D5F89C0003685B69984776
:104E900020B1D5F89430022B00F0E480B9F1000F76
:104EA0000CBF4FF0000B4FF4007BB7EE00BAB8F127
:104EB000000F02D04BF4806B009604F5984808F17F
:104EC0005008404663F0A4F90130D7F8400B9FED3D
:104ED0006C0A9FED6CCADFED6C8A0CBF01230223C4
:104EE0006C3008EE103A27F07DF80CABCDED0A0AD5
:104EF0008DED0B1A8DED090A13E907000DF10C0E6B
:104F00000DF1180C8CE807008EE80700704626F0BB
:104F1000D7FDD7F8402BDFED5D7A92ED36AA2AEE69
:104F200027AAB4EECC0AF3EE0EBAF1EE10FA04F5AD
:104F30009540B4EEEBAAC8BF4BF4807B7430F1EE21
:104F400010FAC8BF4BF4807BF0EE40AA4DF0C2FCD3
:104F500027F046FCB8EEC88A04F59640B4EEC80ABD
:104F6000F1EE10FA00F1240098BF4BF0800BF0EE48
:104F7000409A7AF06FFA68EE288AB0EEC09AB4EEE2
:104F8000E89AF1EE10FA204648BF4BF0400B09F0CA
:104F90002DFD002846D14BF0200B0196404663F0D2
:104FA00037F901284FD14BF0100BB2463249B9F115
:104FB000000F53D0009B002B50D0F4EECCAAF1EEA2
:104FC00010FA4BDCB4EEEBAAF1EE10FA46DCF4EE8C
:104FD000C89AF1EE10FA41D8B4EEE89AF1EE10FA60
:104FE0003CD5019BD3B3BAF1000F37D00A68B4F9AE
:104FF000A40007EE902AB8EE677A18B9B4F8A200B8
:10500000A4F8A400B4F8A43007EE903AF8EEE77ADA
:1050100067EE8B7AB4EEE77AF1EE10FA19D5013229
:105020000A60C2E604F5335034304DF02FFCDFED5A
:10503000187A90ED007AB4EEE77AF1EE10FAAAD47D
:1050400000230193AAE7404663F0E2F80130ADD1B6
:10505000A9E701212046FFF72FFEA6E60022DFE7A1
:105060000121C4E6B9F1000FB0EE08BA0CBF4FF051
:10507000000B4FF4007B1DE740810020CDCC4C3E5F
:105080009F0CB3450080BB440000C842E02E65423F
:105090000000484330B500F5BD530833044693E89B
:1050A000070089B002AD85E807009FED1D7ADDEDB0
:1050B000047A77EE877A9FED1B7ACDED047AD4EDF2
:1050C0002B7AF0EEE77AF4EEC77A04F59540F1EE2C
:1050D00010FA00F174000BD5B4F9A23007EE903A43
:1050E000F8EEE77AF7EE006A86EEA77A84ED2B7A7F
:1050F000D4F8AC30019301AA29464DF05DFC20465E
:10510000FFF732FE2046FEF769F92046FEF740FA27
:105110002046FEF709F82046FEF7B0F809B030BD8A
:105120000AE81C410000003410B504462DED028B46
:105130001D2057F015FC60B304F54053D3F89C00D4
:1051400000F0C4FA192108EE100A04F5706043F06B
:1051500025FE02281AD00338012808D804F5335058
:1051600034304DF093FB90ED008ABDEEC88AB8EE66
:10517000C88A9FED090A28EE000ABDEC028B04F5EF
:1051800098405030BDE8104063F0C8B89FED038AE6
:10519000EDE7BDEC028B10BD0AD7233C00000000F8
:1051A000134A0260134A426002F17401816012499D
:1051B000C16002F5205101610839416124398161E2
:1051C000A2F6F861C1610D49016202F557614162C1
:1051D00002F51861816202F68411C16202F688113B
:1051E00002F68C124263064A01638263704700BF75
:1051F0004C620C08084F002004770020F87600204D
:10520000D02C00201C2952D8DFE801F0130F171B07
:1052100027232F1F512B51335151373A3D414551CF
:1052200051495151515151514D0000F599402C3087
:10523000704700F5A7403C30704700F599406C304E
:10524000704700F59A402830704700F5A2400430BE
:10525000704700F5A4406030704700F5A34054301B
:10526000704700F5A4401830704700F5A640303074
:10527000704700F5A2404430704700F5A3407047E6
:1052800000F59E40704700F5A5401C30704700F5C2
:10529000A1404030704700F5A7407830704700F5D6
:1052A000A8404830704700F5A9406430704700209E
:1052B0007047000073B50B6805461B6C08460C462A
:1052C00016469847034605F539500F4A00960421C3
:1052D00034304DF0C5FE4BF0C7FE236805461B6811
:1052E000204698470A21024628464BF019FE074BF4
:1052F00093F891309B0641BF054A137843F00403AD
:10530000137002B070BD00BF1C510C08B85B0020C8
:10531000C482002038B50C4A182305460C464AF0D2
:105320006BF878B121462846FFF76CFF30B1014693
:10533000064A2846FFF7BEFF002038BD284649F040
:10534000A1FFF9E70120F8E79C510C083C510C083B
:1053500010B500F50053002283F8882D094B044650
:1053600093F8901000F5804304F54054D3F8400BB7
:10537000C90973F097FED4F89C000368BDE810409B
:10538000DB681847B85B002070B5054608680368FD
:105390005B690C461646984790B1306803685B69B4
:1053A000984768B905F54053D3F8C02092F8CB2050
:1053B00032B193F99030002B02DB2846F9F744F81C
:1053C00004480AF0D9F820680368BDE870409B687B
:1053D000184700BF0082002070B500F54055044614
:1053E000D5F89C000B4E0368DB6998473074D5F8FC
:1053F0009C0003681B689847F070D5F89C00036810
:105400005B6C9847014604F5A0500430BDE870403D
:105410003FF074BAA582002070B52DED028B244BAD
:1054200093F8B530DB0782B006460D461446B0EE61
:10543000408AF0EE608A06D500232B60236002B01C
:10544000BDEC028B70BD55F05BFF037F002BF3D0EA
:10545000F36A9FED181A1B689FED170AB3F908301D
:1054600007EE103AB36A1B68B3F9083007EE903ABA
:10547000B8EEC77AF8EEE77A67EE000A68EE811AAE
:1054800027EE800A28EE011A01A9684624F090FA56
:10549000DFED0A6A9DED007ADDED017A27EE267ACE
:1054A00067EEA67A85ED007AC4ED007AC7E700BF03
:1054B000B85B00200AD7233C530469390000C84276
:1054C00070B52DED028B88B0002302930393364B09
:1054D00093F8B53013F0010F0646B0EE408A06ADE2
:1054E00002AC03D155F00CFF037F5BB994E80300D5
:1054F00085E803009DED060ADDED070A08B0BDEC66
:10550000028B70BDB36ADFED296A1B68B3F90830FE
:1055100007EE903AF36A1B68B3F9083007EE103AC9
:10552000B8EEC77AF8EEE77A27EE267A67EEA67A23
:10553000F1EE476ACDED026ADFED1D6ACDED037A2B
:10554000B0EEC77AB4EEE67AF1EE10FA06D5F0EED8
:10555000E77AF4EEE67AF1EE10FAC7D403AA214610
:105560001448F8F7A1FFDDED027A9DED037AF0EE25
:10557000E77AB0EEC77AF4EE477AF1EE10FACCBFD4
:10558000B0EE670AB0EE470A204626F0E7F904A815
:105590008DED040ACDED050A26F092FA204688EE3C
:1055A000000A26F00BFAA1E7B85B00205304693922
:1055B00000000034B82B0020094B93F99020002AFA
:1055C0000CDAB5EEC00AF1EE10FA07D9D3F8C03004
:1055D00093F8A100C31E58425841704700207047FD
:1055E000B85B0020436A1B6893F8CB3043B1054B8E
:1055F00093F8900000F0A000203818BF01207047F9
:1056000001207047B85B002010B5436A0446186853
:10561000D1B102217AF0CEFE236A9FED0C1A1868F0
:105620000368F0EE410ADB6AB0EE410A9847236A4C
:10563000074A1868D2EDD60A03689FED040A5B6E2C
:10564000BDE81040002118470121E3E700000000F9
:10565000B84B002010B5436A04461868002930D0C2
:1056600002217AF0A7FE236A186873F0EBFC636AE4
:105670001B6893F8A130012B04D8236A0121186814
:1056800074F07AFA6369186877F086FB63691868C2
:1056900077F0E2FB63699FED0C0A186877F008FE6B
:1056A0006369186877F076FE236A9FED071A186819
:1056B0000368BDE81040DB6AF0EE410AB0EE410A33
:1056C00018470121CDE700BF0000000013B50446D4
:1056D00001A90C4809F01AFA10B1019802B010BDE6
:1056E0006369186876F062FA18B9074BD3F8180B9B
:1056F000F4E7064801AA032111F086FF0028F4D040
:10570000EBE700BFB82B0020B86B0020CC76002060
:1057100070B504462DED028B00296AD18368B3F978
:105720006258642DB8BF6425FFF7D0FFA8426268B5
:10573000A4BF324B93F89150B2F93430ACBFC5F3EB
:1057400080150125002BDBBF63691B685B4293ED6D
:10575000C48AC8BF07EE903AB2F93230C8BFB8EE7B
:10576000E78A002BB8BF5B429BB25B4207EE903AE0
:10577000A368F8EEE77AB3F96268F4EEC87AF1EE5E
:1057800010FAD8BFB0EE678A2046642EB8BF6426F0
:10579000FFF79CFF6369A26B1B68D2ED001A93EDC3
:1057A000C61AD3ED0E0A311A00EE101AB8EEC00A6E
:1057B00023F0ECFC6368B3F93230002BB8BF5B42D6
:1057C0009BB25B4201EE103A40F29720B8EEC11A4C
:1057D000F0EE480A23F0F8F963692946186876F074
:1057E00089FABDEC028B6369BDE87040186877F0F8
:1057F000D1BD9FED030A0025EEE700BFB85B002096
:1058000000000000436A186803681B69184700001D
:1058100038B52DED028B03680446D3F880309847E5
:10582000236B2A481B68F0EE408AB3F9085009F050
:105830007BF84FF47A72041E4FF000012846D8BF5F
:105840004FF4FA7423F0FEF98442B6EE000A2ADD22
:1058500007EE900AB8EEE77A07EE904A27EE007A54
:10586000F8EEE77A87EE278A4FF46D7038EEC00ABB
:10587000F5EE087AB1EE400A80EE270AB7EE001A7C
:10588000FEEE000A23F0A0F9F7EE007A77EEC07A78
:1058900028EE000A20EE080A20EE080AA7EE880A81
:1058A000BDEC028B38BD031B07EE103AC4F57A74C9
:1058B000B8EEC77A07EE904A27EE007AF8EEE77A5C
:1058C00087EE278A38EE008ACEE700BFB82B00208B
:1058D0002DE9F04F2DED028B00F5804900F5405881
:1058E00099F8A84C89F8A82C0546D8F89C000368BC
:1058F00083B01B680F4616469847B84221D105F57C
:1059000000551A2E85F80C6307D130B905F66C45A1
:10591000D9F8403B2A68C3F8FC208C4B93F89130AF
:10592000980606D40124204603B0BDEC028BBDE8E6
:10593000F08FB442F6D0864A137843F00203137016
:10594000F0E7022E0CD01B2F12D105F59A403146FC
:10595000283003B0BDEC028BBDE8F04F01F05AB91E
:1059600039462846FFF7D6FC04460028EBD1DAE793
:1059700039462846FFF746FC0446019018B92846E8
:1059800049F080FCCFE7D8F8C03093F8CBB003687B
:105990005B699847019A05F5A24344338BF0010AED
:1059A0009A4208BF0120BBF1000F08D1019803689B
:1059B00051465B689847044648BB664A22E098F91E
:1059C0009030002B80F2B480002800F0B180DFF826
:1059D0007CB1DBF89C0003685B69984704460028AB
:1059E00040F0A6800198FFF713FFABF54050B0EEF2
:1059F000408AF8F713FDB4EEC08AF1EE10FA40F3D6
:105A00009780554A01992846FFF754FC8BE705F526
:105A1000425101AA1C31284605F50054FFF7B4FC99
:105A20000198C8F89C0084F80C6303681B689847C9
:105A3000014605F58D50324610304AF03DFE05F521
:105A400039500021343054F089FD94F9563223B195
:105A500005F5095010305FF087FAD8F89C0003680C
:105A60001B689847C21E5042504104F63C4289F8D8
:105A7000D00BD9F8403B1268C3F8F82004F66C420A
:105A8000D9F8403B1268C3F8FC20012F01D00B2F3E
:105A900006D104F65444D9F8403B2268C3F8FC20F0
:105AA0002846FFF799FC294B93F891309B063FF568
:105AB00042AF37E705F5005393F85022002A3FF430
:105AC00075AFB3F86C22D1077FF570AF93F88C22D5
:105AD000002A3FF46BAFD8F8C02092F8CB20002A00
:105AE0003FF464AF93F80C330A2B7FF45FAF98F95F
:105AF0009030002BFFF65AAF184A01992846FFF75D
:105B0000D9FB00240FE7164809F076F90028D1D117
:105B1000D8F89C0003685B6998470028CAD00198B0
:105B200003685B69984704460028C3D10D4A69E7BA
:105B3000019803681B6998470028E4D0084809F0D9
:105B400049F904460028DED1074A5BE7B85B00202C
:105B5000C482002006DE0D0864510C0888510C0830
:105B6000B82B002076510C0806910D080148FFF76C
:105B7000AFBE00BFB82B002013B504468DED010A5F
:105B800062F0DEFA6369A26B1B6892ED001A93ED76
:105B90000E0AD3EDC60A01A961F060F99DED010A74
:105BA00002B010BD436A186803685B6A18470000BA
:105BB00038B5436A1C6894F8CB10054661B9204695
:105BC0007AF0F8FB6B6A1B6893F8A10018B1012802
:105BD00014BF0320022038BD164803783BBBFFF7F3
:105BE000EBFC20BB144A92F8903003F0A003202B6A
:105BF00017D0B5EEC00AF1EE10FA10D592F8923037
:105C00005B070CD4012120467AF0D4FB6B6A1B6839
:105C100093F8A130012B0CBF02200320DBE7022107
:105C2000F1E7204602217AF0C5FB0420D3E70120EA
:105C3000D1E700BF00820020B85B002010B52DED39
:105C4000028B134B93F8B530DB07044604D59FED68
:105C5000110ABDEC028B10BD55F052FB037F002BE7
:105C6000F5D0636B186855F075FCA368DFED0A7A10
:105C700003F6AC0292ED008A03F50B63D3ED000A44
:105C800028EE278A23F04EFE28EE000AE1E700BF47
:105C9000B85B0020000000000000C8420148F8F78F
:105CA0002DBC00BFB82B00200148F9F7ADB800BFEC
:105CB000B82B00200148FFF70BBE00BFB82B002017
:105CC00070B52DED028B7D4D95F891308CB000268E
:105CD000044658060496059603D56369186875F05E
:105CE000D9FD95F8B530D9075DD463689B899A07CB
:105CF0001BD573484CF0CAFDDFED727A90ED007A47
:105D0000B4EEE77AF1EE10FA0FDD4BF0ADF93D217C
:105D10004BF0E6F86C4809220521FFF7D9FD20B9C0
:105D2000092202212046FFF7C5FF636893F954302A
:105D3000CBB365489FED658AF9F766F8E3689FED98
:105D4000647A1B68D3ED0A7AF4EEC87AF1EE10FAA1
:105D5000B8BFF0EE477AB6EE000A27EE800A20467A
:105D6000FFF7AEFB8DED040AB0EEC00AB4EEC80A30
:105D7000F1EE10FACDED050A06D5F0EEE00AF4EEEC
:105D8000C80AF1EE10FA0ED495F892301B0704D42D
:105D90004BF06AF949214BF0A3F895F8923043F0A3
:105DA000080385F8923095F893306FF3820385F8F5
:105DB0009330606909960A9609AD2A4604A90068DD
:105DC000012375F0D1FD6369186877F045F86369C0
:105DD000186876F01DF9A3688DED060ACDED070A67
:105DE0008DED081AD3ED007AF5EEC07AF1EE10FAD7
:105DF00052DD384B9FED388AB3F94C3300EE903AC0
:105E0000F8EEE00A2046CDED030AFFF75FFCA36839
:105E1000DDED030AD3ED001A9FED2A0AB7EE002A42
:105E200007EE900A31EE822AB8EEE71A22EE082A2F
:105E300061EE881A22F008FEDFED287A20EE270AAC
:105E4000DFED277A20EE270AA2F024FEDFED257A87
:105E500020EE270A06A820EE088A25F031FEB4EECF
:105E6000C08AF1EE10FA17D5C8EE006A63699DED9D
:105E7000067ADDED077A27EE267A67EEA67A8DEDB3
:105E8000067ACDED077A1B68D3F88823C3F89423EC
:105E9000D3F88C23C3F89823236A13491C68284637
:105EA000FCF708FB0B9B009395E80C0006A9204625
:105EB00073F07AF90CB0BDEC028B70BDB85B0020BA
:105EC000C076002000002F44B82B002000000034D2
:105ED00000007A43B84B00200000C8420AD7233C98
:105EE00035FA8E3C0AE81C41F480002013B50446C4
:105EF0000191FFF7E5FE0199204602B0BDE8104090
:105F0000FFF706BC0148FEF7D7BE00BFB82B002044
:105F1000004870472C5A00200148F8F7DDBA00BF4E
:105F2000B82B002030B50F4D87B0002304466946DA
:105F3000D5F8480B00930193029376F081F8D5F8D9
:105F4000480B02A976F0D0F8009B0393019B0493C1
:105F50000222029B059303A9204611F025FE20464C
:105F600007B030BDB86B002000207047002070479C
:105F700000207047002070470020704700207047C5
:105F800000207047002070470020704700207047B5
:105F90009FED010A704700BF00000000002070471D
:105FA0000020704700207047012070470020704794
:105FB0000020704701207047002070470120704783
:105FC0000120704700207047012070470120704772
:105FD0000020704700487047B4510C0800487047D3
:105FE000B4510C08836893F8C038DB0706D500234A
:105FF00080F83C30024B0222C3F894200120704705
:10600000B85B002090F83C3043B9836893F8C038FF
:10601000DB0742BF034B0122C3F89420002380F822
:106020003C307047B85B0020012380F83C3070475B
:106030002DE9F0432DED0C8BF0EE409A20EE000A96
:1060400097B00025A0EEA00A04468946B0EE41CAEA
:10605000F0EE60AA90461F460195029503950495BF
:1060600005950695A2F02CFFF7EE00CAB4EEEC0AF7
:10607000F1EE10FAC8BFCCEE807AA36803F67C027A
:1060800003F5086392ED009A9FEDC5DAD3ED000A9F
:10609000C4BF69EEA79A6AEEA7AAB0EE690A23F018
:1060A00041FCA36829EE0D9A03F67C0203F5086310
:1060B000D2ED008AD3ED000A29EE009AB0EE6A0A0A
:1060C00023F030FCA36868EE8D8A03F6940203F691
:1060D0009803D3ED000A92ED008A68EE808AB0EE54
:1060E0004C0A23F01FFC636828EE0D8A93F9703088
:1060F00028EE008A002B00F0D980236A9FEDA90AC0
:1061000018686C3025F06EFFB0EE60AACDED080A7D
:106110008DED091A8DED070A22F000FDBDEEC0BA23
:10612000A14940F6B8321BEE100A22F07BFD434233
:1061300007EE903A6368F8EEE77A93ED1A7A67EE25
:10614000877AB0EE4A0ACDED017A22F0E7FCFDEE47
:10615000C0BA40F6B83294491BEE900A22F062FDB4
:1061600042426368039507EE902A93ED1B7A93F9F8
:106170007030F8EEE77A022B67EE877ACDED027A7F
:106180006ED18A4BB3F94C330AEE103AB8EECBBA63
:10619000B8EECAAA236AB4EECABAF1EE10FA1A68C7
:1061A0003DDDA368DFED820AA16B92ED051AD1ED0A
:1061B000001A03F67C0393ED007A27EE0D7A3AEE8F
:1061C0004B0AC7EE200A22F0E1FFDDED017A37EE3F
:1061D000800A8DED010AB8EEEB0A236AB4EECA0A12
:1061E000F1EE10FA1A6834DDA368A16B92ED061A7D
:1061F000D1ED001A03F67C03D3ED000A20EE8DDA10
:10620000DFED6B0A3AEE400ACDEE200A22F0BEFF27
:10621000DDED027A37EE800A8DED020A20E0B1EE64
:106220004A0AB4EEC0BAF1EE10FAD4D5A368A16B55
:10623000DFED5F0AD1ED001A92ED051A03F67C033B
:1062400093ED007A27EE0D7A30EE4B0AC7EE200A66
:10625000B9E7B1EE4AAAB4EECA0AF1EE10FAC3D415
:10626000236AD3F800C00CF184030FCB12AD85E88C
:106270000F000EAE0AAD86E80F0085E80F0004ABF4
:1062800001AA2946604673F02BFC636893F97030CD
:10629000022B16D1DDED047A39EE279ADDED057A71
:1062A00078EEA78ADDED067A38EE278A89ED009A26
:1062B000C8ED008A87ED008A17B0BDEC0C8BBDE8F5
:1062C000F083F0EEE99AF0EEEAAAF4EEE9AAF1EE34
:1062D00010FA48BF6D46CDED009ACDED0AAAD5ED76
:1062E000007ADFED340AB0EECCCAF4EECC7AF1EEEF
:1062F00010FAD8BF35468DED0ECA95ED007ADFED68
:106300002E7A87EE270AAD20B7EE001A3CEEC00ABF
:1063100022F05AFCE369D3ED937A04A820EE270A11
:1063200025F060FEF0EEC07A8DED061AB0EEC91AC7
:1063300031EE671A8DED040AB0EEC11A39EE000A8B
:10634000CDED050AB520F1EE410A22F03DFCB0EE9C
:10635000409A9DED050AB0EEE81AF0EEC07A31EEF3
:10636000671A38EE800AB0EEC11AF1EE410ABA207F
:1063700022F02AFCF0EE408A9DED060AB0EEC81A23
:10638000F0EEC07A31EE671A38EE000AB0EEC11AAC
:10639000BF20F1EE410A22F017FCB0EE408A85E7FB
:1063A0000000C8429F0CB34548F4FFFFB84B0020E3
:1063B00000007A440000000000A08C4510B52DEDCF
:1063C000028B836A044686B0186855F0C3F8E36A06
:1063D0001868B0EE408A55F0BDF8636B8DED010A88
:1063E000186855F0B7F805ABB0EE401A03A920467F
:1063F000DDED010A04AAB0EE480AFFF719FE636A50
:10640000186890F8CB1000293AD179F0D3FF2046D4
:10641000FFF7FEF9636A1B6893F8A1100129B0EE3B
:10642000408A3DD0032944D051B9236A012118681C
:1064300074F058FA236A186872F0EEFD9FED208A16
:10644000236AA268186892F8C02803689DED030AC1
:10645000DDED040A9DED051A92074CBFDB6B9B6BCB
:106460009847236A174A1868D2EDD60A03680021B4
:106470005B6EB0EE480A984706B0BDEC028B10BDCB
:10648000114B93F99120002A06DBD3F89430022BAC
:1064900004D190F8A1300BB90121B6E70221B4E78D
:1064A000236A186874F01EFA236A186872F0CAFD2D
:1064B000C4E7D9790029C3D12046FFF723FDBFE700
:1064C00000000000B84B0020B85B0020836893ED0B
:1064D000140AB5EEC00AF1EE10FA01DCFFF792B92A
:1064E000704700007047000000207047012070478F
:1064F000022070470020704700207047012070473D
:106500000020704781F001007047000001207047B3
:1065100001207047004870474C520C0800487047F3
:1065200058520C0838B543690446186875F060FC89
:1065300018B96369186876F0DFFD636920461D6845
:10654000FFF7EAFC6368B3F93820B3F9363000EEA0
:10655000903A434201EE102A00EE103AB8EEC11A0A
:10656000F8EEE00AB8EEC00A284675F02DFB636924
:1065700020461D68FFF7D0FC6368B3F93820B3F9F3
:10658000363000EE903A434201EE102A00EE103A07
:106590002846B8EEC11AF8EEE00AB8EEC00A75F067
:1065A0008DFB012038BD000030B52DED028B044677
:1065B000436985B01D68FFF7AFFC6368B3F9382005
:1065C000B3F9363000EE903A434201EE102A00EE65
:1065D000103AB8EEC11AF8EEE00AB8EEC00A284642
:1065E0005B4D75F0F1FA2046FFF75EFBB5F94C33D1
:1065F00008EE103A236A186803689B6E9847B8EE55
:10660000C88AF0EE400A02AA01A9B0EE480A204664
:10661000FEF702FF2046FFF711FB236B1B68B3F95F
:106620000830F0EE408A00EE103A2046B8EEC00A7C
:10663000FFF734FB2046B0EE408A8DED030AFFF7EA
:106640006BFC6368B3F9363001EE103A434200EE5A
:10665000903AB8EEC11AF8EEE00A2B20B0EE480AE4
:1066600022F0B2FA20468DED030AFFF7A1FA0428C2
:1066700013D8DFE800F0032F252A4B00236A18689F
:1066800072F0CAFC236A0021186873F075FA636916
:106690009FED300A186876F00BFE236ADDED020AE2
:1066A00018689DED010A0368B0EE681ADB6A984726
:1066B0006369186876F06EFE05B0BDEC028B30BDE4
:1066C000236A0121186873F057FA236A186872F078
:1066D000B9FCDCE7204D2B7863B963689FED1F1A86
:1066E000DFED1C0A93ED040A452022F06DFA2846DE
:1066F00008F02AFF20469DED030AFFF73DFA1648F1
:106700008DED030A03A908F059FFC6E7636A022169
:10671000186879F04FFEB5F94C33114800EE103A85
:1067200002AA01A9B8EEC00A60F0C8F820469DEDA3
:10673000030AFFF721FA0B488DED030A08F002FA6D
:1067400063699DED030A186875F0C4FAA5E700BFF8
:10675000B84B0020000000000082002000007A44B6
:1067600098770020345900200020704790F8B93104
:10677000002B14BF1B20032070470000002070472F
:106780000120704790F89001062804D0A0F1090379
:10679000584258417047012070470000012070475F
:1067A0000120704790F8B901034A044B002814BF38
:1067B00010461846704700BFF0520C0809A40D0897
:1067C00090F8B901034A044B002814BF104618463C
:1067D000704700BFFC520C0809A40D0890F8900106
:1067E0000A3818BF0120704790F8B9312BB9044B13
:1067F000D3F8880C00F0010070470020704700BFFC
:10680000B84B002090F8903123B9034B187880F0F2
:106810000100704700207047E481002038B590F8EF
:106820009041012C054601D0002038BDC36818688E
:1068300003681B6998470028F6D1EB681B6820465F
:1068400083F8B848F1E70000C3681B68002283F8AA
:10685000B82801207047000070B52DED028B002391
:1068600080F8B931B0F87030012B84B004460D4681
:1068700001D8002946D0636A254E1B6893F8CB30B7
:1068800073BB2448072384F890310368022B02D19C
:106890000021FBF751FC9FED208AE368F0EE480AE7
:1068A0001868B0EE481AF0EE481AB0EE480A012512
:1068B00077F0F6FF84ED738A84ED748A84ED758A2F
:1068C00084F8B85104F59A7026F074F8134803F070
:1068D000B7FD96F892306FF3C30386F8923011E05B
:1068E00096F99030002BCCDA04F13C0028F014F932
:1068F00005460028C5D12046FFF70AFB084A0221B9
:106900004CF0AEFB284604B0BDEC028B70BD00BF5E
:10691000B85B0020F4800020000000008C7D002087
:1069200004530C0810B50446064890F8683D012B46
:1069300003D100F6645026F0A5F8002384F8B9319D
:1069400010BD00BFB86B002010B52DED028B094BB8
:106950000446D3F84C0BB0EE408A77F039FB9FED3C
:10696000060A28EE008A012084ED748ABDEC028BB1
:1069700010BD00BFB86B00200AD7233C10B52DED29
:10698000028B094B0446D3F84C0BB0EE408A77F0EB
:106990002FFB9FED060A28EE008A012084ED758A00
:1069A000BDEC028B10BD00BFB86B00200AD7233CA2
:1069B00010B52DED028B094B0446D3F84C0BB0EE0D
:1069C000408A77F023FB9FED060A28EE008A01201B
:1069D00084ED738ABDEC028B10BD00BFB86B002044
:1069E0000AD7233CC3681B68186975F043BC0000D4
:1069F00038B5D0F8943104460D461BB980F0C0FE7E
:106A0000C4F8940180F0BCFED4F89431C01A4FF45D
:106A10007A73B0FBF3F0B4F89231984209D3204670
:106A2000FFF776FA2B88044A06214CF019FB012067
:106A300038BD0020FCE700BF20530C0890F89031CF
:106A4000052B05D1054BD3F8543BD86875F08ABBAC
:106A5000C36818680368DB68184700BFB86B00207C
:106A600008B590F89031052B0BD1094BD3F8543B66
:106A7000D868243025F024F8BCEEC00A10EE100AC5
:106A800008BDC368186803689B689847F4E700BFAF
:106A9000B86B002090F890318B4206D00A2B80F81A
:106AA000901102D10148FCF7CDBF7047B82B0020F0
:106AB00073B501231E4E80F87530D6F89C308342A2
:106AC00005460A4614D1012485F8B941D6F89C0040
:106AD000019203681B689847019A0146154849F0DE
:106AE000EBFD96F891309A061BD4204602B070BD9B
:106AF00001910321FFF7DEF8019A04460028E2D154
:106B000085F875004AF0B0FA1B220A214AF008FA0B
:106B100096F891309B06E8D5074A137843F00403B2
:106B200003E0054A137843F002031370DDE700BF6A
:106B3000B85B0020683D0020C482002030B585B0DD
:106B400004460D4601466846FFF7ECF9694604F134
:106B50003C0028F093FDC8B94AF086FA1B220A21AE
:106B60004AF0DEF90D4B93F891309B0604D50C4AA0
:106B7000137843F0040313702046FFF7C9F9094A5C
:106B800004214CF06DFA002005B030BD29462046A6
:106B900005B0BDE83040FFF78BBF00BFB85B0020F9
:106BA000C482002034530C0830B585B004460D462D
:106BB00001466846FFF7B6F9694604F13C0028F043
:106BC00081FDC8B94AF050FA1B220A214AF0A8F9FF
:106BD0000D4B93F891309B0604D50C4A137843F083
:106BE000040313702046FFF793F9094A04214CF07F
:106BF00037FA002005B030BD2946204605B0BDE873
:106C00003040FFF755BF00BFB85B0020C4820020B2
:106C100070530C087FB505460E4605F13C0401464D
:106C20006846FFF77FF96946204628F04BFDC0B95A
:106C30002046694628F022FD044690B94AF014FA2D
:106C40001B220A214AF06CF90D4B93F891309B06F8
:106C50000FD42846FFF75CF90A4A04214CF000FAE9
:106C600004E031462846FFF723FF0446204604B0DF
:106C700070BD054A137843F004031370E9E700BFC1
:106C8000B85B0020A8530C08C482002030B504462D
:106C900085B00F4808F09EF80546B0B1072384F888
:106CA00090310023019302930393E36801A91868CC
:106CB00077F028F9E3681868036801A95B68002287
:106CC000984704480021FBF737FA284605B030BD45
:106CD000B82B0020F4800020F0B5424FD7F8202BCD
:106CE000D7F81C3B2DED028B1343D7F8182B134319
:106CF00087B005460C460CD148F008FD40F27512ED
:106D00004FF4801107B0BDEC028BBDE8F04048F0B5
:106D1000B5BC806978F092FB2046B0EE408A10F056
:106D200067FC03283AD1EB6801A9186877F0C6F927
:106D3000064698B3DDED017A6368009338EE678A02
:106D4000294BDFED2A7A93F990309FED290A2948E3
:106D5000002BA8BFB0EE670A38EE008A009BBDEE9C
:106D6000C88A002118EE102A9342ACBF009300920B
:106D7000FBF7E2F96B69186876F0BEF9DDED007A91
:106D80001D48B8EEE70A314608F098FE0021284673
:106D9000FFF780FE07B0BDEC028BF0BD94E80F005A
:106DA00002AE86E80F00D7F81C3B04936A46D7F87A
:106DB000203B05930221304610F026FC78B94AF0BA
:106DC00053F9022215214AF0ABF8DDED037AF8EE13
:106DD000E77A77EE887AFDEEE77ACDED007A002645
:106DE000AEE700BFB86B0020B85B002000000000D9
:106DF0000000C842F4800020E481002030B52DED71
:106E0000028BC36887B0044618680D4677F04AF9CC
:106E100000284BD194F89021002300930193029312
:106E20006AB93148039303A90493059308F078FEE7
:106E300028B1039B0093049B0193059B029394ED5F
:106E4000730A9FED2A8AE368DDED000A9DED011AC1
:106E5000DDED021A1868B4EEC80AF1EE10FAAABF06
:106E6000DFED237A9FED230A20EE270A77F018FD45
:106E7000D4ED747AF4EEC87AF1EE10FA07DBE36829
:106E80009FED1B0A186827EE800A77F0A1F8D4ED71
:106E9000757AF4EEC87AF1EE10FA07DBE3689FED3D
:106EA000140A186827EE800A77F0A2F8E3682946EA
:106EB000186877F01DFC054688B10F4B1B68022B44
:106EC00009D0032B03D10D4B93F97D331BB10A4835
:106ED0000021FBF751F901212046FFF7DBFD284691
:106EE00007B0BDEC028B30BDE4810020000000340F
:106EF0000000C84200000000F4800020B84B0020D1
:106F000010B52DED028BC368DFED348A1B68426932
:106F1000D3ED0A0A9FED328A93ED060AF4EEE80AF1
:106F20000446F1EE10FA1068B8BFF0EE480A74F0AB
:106F300031FCE36862691B681068D3ED0A0A93EDBF
:106F4000060AF4EEE80AF1EE10FAB8BFF0EE480ACD
:106F500074F098FC6369186874F028FE18B96369C6
:106F6000186875F063FEE36862691B68106893ED4A
:106F7000080A93ED0C1AD3ED070AB0EEC00A74F0BC
:106F800023FEE36862691B68106893ED080A93EDBD
:106F90000C1AD3ED070AB0EEC00A74F08FFE6369D5
:106FA000186874F025FF18B96369186876F0A4F8BA
:106FB00000210C48FBF7C0F80B4861F047FA0B4A78
:106FC000B2F8923023F48163A2F89230BDEC028BC8
:106FD00020460221BDE81040FFF75CBD00000034F0
:106FE00000007A43F480002008780020B85B00207D
:106FF00010B50C4B0446D3F8540B90ED0B0A90F8E7
:10700000502000F11C0176F0C5FC07480368022BF4
:1070100002D00821FBF790F820460521BDE810407A
:10702000FFF738BDB86B0020F4800020F0B52DEDDF
:10703000028B4A4DDFED4A8AB0EE408A8FB004469B
:10704000D5F8540B0E46174676F01AFBF0EEC87AC8
:10705000F4EEE87AF1EE10FA07D49FED420AD5F883
:10706000540B28EE000A76F071FBD5F8540B90ED26
:107070000B0AB0EEC00A0FB1B1EE400A76F056FB33
:107080000023D5F8540B079302AA07A90893099384
:1070900076F078FBDFED347A9DED027AB4EEE77A94
:1070A000F1EE10FA56DD022207A90AA810F07CFDC5
:1070B00071680191304610F09BFA019902460AA8C6
:1070C00010F06CFAE3680AA9186877F011FB10B9A0
:1070D0002648FDF7B3F8A06978F0AEF90268436876
:1070E000D5F8540B049303A91C30039224F01AFC26
:1070F00005A88DED050ACDED060A24F0E1FC1C4B38
:107100001B68022B1BD0D5F8543B1948D3ED0A7AE3
:10711000F4EEE87AF1EE10FAB8BFD3ED047AF4EEAB
:10712000C07AF1EE10FA4FF0000110D5DFED117AC0
:10713000B4EEE70AF1EE10FA09DDFBF71DF80421C1
:107140002046FFF7A7FC0FB0BDEC028BF0BDFAF7AD
:10715000F3FFF4E72046FFF74BFFF4E7B86B00209E
:10716000000000340000C84200009643B82B002005
:10717000F48000200000FA4308B50748D0F8883CA6
:107180009B0704D50121A0F50050F7F713F8BDE8DF
:107190000840024808F0F2BAB84B0020E481002011
:1071A00030B589B00446FEF71DFA30B10021204603
:1071B00009B0BDE83040FEF74DBA636A0221186895
:1071C00079F0F8F8E368186803685B699847014646
:1071D0001048FCF71FFF6369186876F0DBF8236A34
:1071E0001D686369186874F013FF05AC20460A49EE
:1071F0008DED020ACDED030A8DED041AFBF75AF965
:10720000079B009394E80C0002A9284671F0CCFF7C
:1072100009B030BDB82B0020F480002038B50446FA
:10722000FEF7E0F9054628B120460021BDE83840C8
:10723000FEF710BA636A0221186879F0BBF8294694
:107240002046BDE83840FEF751BE0000014800214D
:1072500005F004BCE87E002030B5174D9FED170AFD
:1072600005F5804389B00446D3F8540B76F0F2FB61
:1072700001462846FCF7CEFE6369186876F08AF866
:10728000236A1D686369186874F0C2FE05AC204665
:107290000B498DED020ACDED030A8DED041AFBF7C3
:1072A00009F9079B009394E80C0002A9284671F0A5
:1072B0007BFF09B030BD00BFB82B002000000000EC
:1072C000F480002030B589B00446FEF78BF930B168
:1072D0000021204609B0BDE83040FEF7BBB9636A23
:1072E0000221186879F066F8E368186803685B693A
:1072F000984701461048FCF78DFE6369186876F0E0
:1073000049F8236A1D686369186874F081FE05AC4A
:1073100020460A498DED020ACDED030A8DED041ACF
:10732000FBF7C8F8079B009394E80C0002A92846D5
:1073300071F03AFF09B030BDB82B0020F480002076
:1073400030B52DED028B83B00446FEF74BF920B922
:10735000636A1B6893F8CC3043B90021204603B020
:10736000BDEC028BBDE83040FEF774B994F898315B
:10737000DA071DD4E3681D682B6828469B68984788
:10738000D5ED097A94F89831B4EEE70AF1EE10FAE7
:107390004CBF0122002262F3000384F8983107D425
:1073A000204603B0BDEC028BBDE83040FFF7F8BECD
:1073B00094F898319B0734D4E368DFED458A1B6865
:1073C0006269D3ED0A0A9FED438A93ED060A1068BD
:1073D000F4EEE80AF1EE10FAB8BFF0EE480A74F0E5
:1073E000D9F9E36862691B681068D3ED0A0A93ED66
:1073F000060AF4EEE80AF1EE10FAB8BFF0EE480A19
:1074000074F040FA6369186874F0D0FB18B96369C6
:10741000186875F00BFC94F8983143F0020384F877
:1074200098312D4BD4F8A021D3F8183B9B1A07EEC6
:10743000903AB8EEE78AF1EE047AB0EEC87AB4EE8C
:10744000E77AF1EE10FA38D594F8983143F0040356
:1074500084F89831204684ED678AFEF731FC636931
:10746000A26B1B68D2ED001A93EDC61AD3ED0E0A7B
:10747000B1EE480A21F08AFE63691B6840F2AA4017
:1074800093EDC31AD3EDC40A21F09EFB2046FEF70C
:1074900073FB12488DED010A07F054FB63699DED03
:1074A000010A186874F016FC6369186803B0BDEC33
:1074B000028BBDE8304075F06DBFD4ED677A68EEA1
:1074C000277AF5EEC07AF1EE10FAC3D5BCE700BF1B
:1074D0000000003400007A43B86B002034590020CB
:1074E00030B52DED028B83B00446FEF77BF820B952
:1074F000636A1B6893F8CC3043B90021204603B07F
:10750000BDEC028BBDE83040FEF7A4B86369DFED47
:10751000347A1B6894ED710A93EDC31AD3EDC40A53
:1075200020EE270A40F2C44021F04EFB2046FEF731
:1075300023FB236A186803689B6EB0EE408A984765
:10754000284BB3F94C3307EE903AB4F8BC316425BC
:10755000F8EEE77A13FB05F3B4EEE70A07EE103A0C
:1075600094F9BE31F1EE10FAD8BFF0EE407A13FB79
:1075700005F39FED1D0AF8EEC76A07EE103AF4EE28
:10758000407AB8EEC77AF1EE10FA58BFB0EE670A4B
:107590006846CDED006A8DED017A24F0E3FA236AA6
:1075A000DDED010A1868B4F8C03102689DED000AEB
:1075B000126B13FB05F301EE103A0121B8EEC11A6C
:1075C00090476369B0EE480A186874F083FB6369FA
:1075D000186875F0DFFE03B0BDEC028B30BD00BF54
:1075E0000000C842B84B002000007A4430B590F843
:1075F000B83185B00446F3B168460FF0C9FF3F4883
:1076000069460AF0D7F950B104F13C0028F022F89D
:10761000002384F8B83104F59A7025F0CBF994F87A
:1076200090310A2B2DD8DFE803F0294B4F534B57ED
:107630002C5B5F2C630000F59A7025F0BBF904F118
:107640003C0590B194F84030012B0ED194F8903164
:10765000012B0AD1284627F06BFE50B12046FEF7D9
:1076600057FC274A02214BF0FBFC284627F08EFEF0
:10767000D5E72046FEF74CFC224AF3E72046FFF709
:107680007BFD94F844303BB994F8463023B994F824
:1076900040309A1E5342534194F8B92162B35BBB08
:1076A00084F8B931184BD3F89C0003681B689847DD
:1076B000014616482D2205B0BDE8304048F0FCBF19
:1076C0002046FFF76DFDDCE72046FFF7A7FDD8E772
:1076D0002046FFF7BBFDD4E72046FFF7BDFDD0E70E
:1076E0002046FFF7EFFDCCE72046FFF729FEC8E76D
:1076F0002046FFF7F5FEC4E705B030BD104000207E
:10770000F4530C081C540C08B85B0020683D0020A2
:107710002DE9F0412DED028B074684B008460E4658
:107720000FF066FF032880466D4628D1FB68186875
:1077300076F01EFB012822D12148294607F0E6F900
:107740000446B0B17B69DDED007A1B68F8EEE77A9C
:1077500093EDF27A77EEC77A4246FDEEE77A17EEBE
:10776000901AC829CDED007AB8BFC82130460FF075
:1077700015FF204604B0BDEC028BBDE8F081114B33
:107780000FCB85E80F0030460FF032FF0146284648
:107790000FF096FF04460028EBD07B69DDED017AFF
:1077A0001B68B8EEE78AD3EDF27A284638EE678A8E
:1077B0000FF01EFFBDEEC88A024618EE101AD5E77C
:1077C000B82B0020CC76002010B543699FED126ADB
:1077D0001B68D3EDF06A93EDF17AD3EDF27A86B0BF
:1077E00066EE866A27EE067A67EEC67A68460C462B
:1077F000CDED006A8DED017ACDED027A24F0B6FB75
:1078000003A920468DED030ACDED040A8DED051A7E
:1078100010F0FAF906B010BD0AD7233C30B5083293
:1078200004461D460FCA84E80F00134301BFAB682E
:10783000A360EB68E360636885B093B920460FF0FE
:10784000D7FE03AA014628460FF0DEFE60B1039979
:10785000019120460FF0CCFE0199024620460FF020
:107860009DFE204605B030BD696801912846F1E7CC
:1078700030B50B6985B004460BB94B6953B300238F
:10788000C4F8B43108310FC96D4685E80F002946A8
:107890002046FFF73DFF98B9124B0122D3F8181B81
:1078A00028460FF07BFE49F0DFFB0222152149F04C
:1078B00037FB2046FEF72CFB0B4A02214BF0D0FB96
:1078C00029462046FFF79AFA10B90848FCF7B6FC9B
:1078D00005B030BD0123C0F8B43105B0BDE830407B
:1078E000FFF70EBBB86B002050540C08B82B0020DB
:1078F00070B51A4B04460E460FCB88B06D4685E82E
:107900000F0020462946FFF75FFFE368186876F00E
:10791000C9FB98B1E368186803681B69984768B1A8
:10792000E3682946186876F02FFA38B947F0EEFE7A
:1079300040F295624FF4801147F0A0FE214604A862
:107940002B463246FFF76AFF04A92046FFF756FA96
:1079500010B90348FCF772FC08B070BDCC7600206B
:10796000B82B002070B5154B0C4606460FCB88B0DF
:107970006D4685E80F0029463046FFF725FF2B4668
:107980002246314604A8FFF749FF6288A388122ADD
:107990004FEA132305D1227ED20744BF03EB8303B2
:1079A0005B00227A07EE903AC2F34002B8EE670A13
:1079B00004A93046FFF73AFB08B070BDCC76002032
:1079C00038B504460D46FFF793FF0023C4F8943101
:1079D000AB88A4F8923138BD7FB50D460446FFF759
:1079E00087FF05F108010FC96E4686E80F001343B3
:1079F00006D1234BD3F81C2BD3F8203B02920393E0
:107A000004F5D072012130460FF0FEFD94F8983154
:107A100070B923F0050343F0050384F8983120463C
:107A2000FEF776FA174A06214BF01AFB04B070BD38
:107A300023F0070384F898310023C4F89C31E368ED
:107A400062691B68106893ED080A93ED0C1AD3ED78
:107A5000070AB0EEC00A74F0B7F8E36862691B6801
:107A6000106893ED080A93ED0C1AD3ED070AB0EEF7
:107A7000C00A74F023F908212046FFF70BF8D5E778
:107A8000B86B00207C540C082DE9F0438DB06D4696
:107A900088461C46074613460A4601462846DDE945
:107AA0001469FFF7BBFE95E80F0084E80F0007A8F4
:107AB0000FF06EFDB8F80430F3B9B8F800100131DA
:107AC00005AA89B207F13C0026F0DEFFA0B12346EB
:107AD00005AA39462846FFF7A1FE95E80F0086E87B
:107AE0000F00BDF81630A3F152025342534189F8FA
:107AF00000300DB0BDE8F08394E80F0086E80F0079
:107B00000023F4E770B58B8892B004460D46164604
:107B1000002B44D10DA80FF03BFD298801310BAAA1
:107B200089B204F13C0026F0AFFF002837D0BDF841
:107B30002E10132903D014D81039012913D8334635
:107B40002A46214603A8FFF769FE03AB214607A892
:107B50000BAAFFF763FEE36807A9186876F008FE32
:107B600001E0522901D012B070BD07AD03A80FF09B
:107B70000FFD28460FF00CFD0DF10B03CDE900536E
:107B8000324603AB0BA92046FFF77EFFE0689DF865
:107B90000B3000682A4603A976F0C0FDE3E7012018
:107BA000E1E7000070B5214B04460E460FCB88B0CC
:107BB0006D4685E80F0020462946FFF705FEE3687D
:107BC000186876F06FFA98B1E368186803681B6963
:107BD000984768B1E3682946186876F0D5F838B94F
:107BE00047F094FD40F216624FF4801147F046FDD5
:107BF000214604A82B463246FFF710FE04A9204672
:107C0000FFF7FCF820B90A48FCF718FB08B070BD74
:107C10000023C4F89431B388A4F8923104AA314601
:107C20002046FFF76FFF0028F0D1ECE7CC7600206C
:107C3000B82B0020F0B5324B04460E460FCB91B066
:107C400004AD85E80F0020462946FFF7BDFDE36837
:107C5000186876F027FA98B1E368186803681B691A
:107C6000984768B1E3682946186876F08DF838B906
:107C700047F04CFD4FF4DF624FF4801147F0FEFCFB
:107C80000CAF08A80FF084FC38460FF081FC0DF112
:107C90000F03CDE900732A4608AB31462046FFF7B3
:107CA000F3FEE0689DF80F3000683A4608A977F0C7
:107CB0007BF820B91348FCF7C1FA11B0F0BD0023DE
:107CC000C4F89431B388A4F8923108AA314620460A
:107CD000FFF718FF0028EDD00B4B1B68022B09D0D3
:107CE000032B03D1094B93F97D331BB106480021C7
:107CF000FAF742FA01212046FEF7CCFEDDE700BF8D
:107D0000CC760020B82B0020F4800020B84B002057
:107D100037B504460D467FF033FDC4F8A801D5ED14
:107D2000027AF5EEC07AF1EE10FA17DD9FED137AC4
:107D300067EE877AFCEEE77AC4ED697A2046FEF7B3
:107D4000E7F8D4F8A4214FF47A73B2FBF3F30C4AAA
:107D5000062103B0BDE830404BF082B95CF09AFBDD
:107D60000023009395F90D2095F90E3095F90C102C
:107D70005CF02CFBC4F8A401E0E700BF00007A44EB
:107D800094540C0810B5B1F90A30A0F8BC3191F93F
:107D90000C3080F8BE31B1F90D30A0F8C031B1F926
:107DA0000F3007EE903AF8EEE77A0446C0ED717AAC
:107DB0007FF0E6FC0A21C4F8C8012046BDE8104067
:107DC000FEF768BE38B504460D467FF0D9FCC4F80E
:107DD000B001D5ED027A9FED047A67EE877AFDEE69
:107DE000E77AC4ED6B7A38BD00007A444A7C0648D5
:107DF0000B46003A91F91010D3ED030A93ED020AF5
:107E000018BF0122FAF7C2B9F480002070B51B4EEA
:107E10000446D6F89C00036886B01B680D46984758
:107E2000042806D16B88102B0FD0732B20D0002094
:107E30001CE0D6F89C0003681B6898470328F6D11D
:107E400094F89031062BF2D1ECE705F108010FC947
:107E500002ACDFED0B0A84E80F0000230948009311
:107E6000B0EE600A1A46214602F02CF906B070BD49
:107E700020462946FFF7BAFF0120F7E7B85B00204C
:107E8000000000008C7D002038B5D1F8093007EEE5
:107E9000903AF5EEC07AF1EE10FA05460C4605DD93
:107EA0000B7A022B03D01ED9032B0ED038BD154BF5
:107EB0009FED150AD3F84C0B27EE800A76F088F870
:107EC000D4F80930C5F8D031F0E70E4B9FED0E0A1B
:107ED000D3F84C0B27EE800A76F08AF8D4F80930F4
:107EE000C5F8D431E2E7074B9FED070AD3F84C0BF6
:107EF00027EE800A76F08AF8D4F80930C5F8CC313C
:107F0000D4E700BFB86B00200000C84210B5044C95
:107F1000237813B1034860F093FA207810BD00BFB6
:107F2000E48100200878002013B5094B0191044634
:107F3000D3F84C0B03681B69984730B10199204670
:107F400002B0BDE81040FEF753BD02B010BD00BF47
:107F5000B86B002090F8983113F0010018BFC3F3FC
:107F600080007047094A034692F86D0368B192F8A1
:107F70006C23043A012A07D85B6A1B6893F8A100B6
:107F8000431E58425841704700207047B87B00207C
:107F900010B504467FF0F4FBD4F8B031C01AD4F821
:107FA000AC3123EAE37398424FF0000084BFC4F879
:107FB000AC01012010BD000010B503680446DB6D64
:107FC0009847D4F8AC3123EAE37398424FF00000AD
:107FD0003CBFC4F8AC01012010BD000008B5044846
:107FE0000321FAF7A9F8BDE808400148FAF790B96B
:107FF000F480002070B51C4B0446D3F84C0B03688A
:108000001B690E469847054610B90025284670BDE5
:10801000D4F894315BB97FF0B3FBB4F89231C4F873
:10802000940123B1114A537843F0010353707FF058
:10803000A7FBD4F89421B4F89231801A4FF47A72E5
:10804000B0FBF2F09842E0D323B9084A537843F0EA
:10805000010353702046FDF75BFF3388044A062175
:108060004AF0FEFFD2E700BFB86B0020C4820020B8
:1080700020530C0810B590F89031042B0446164B91
:108080000AD1D3F84C0B03681B69984718B12046F6
:10809000FEF7AEFF002010BD0A79D3F8543BDFEDA8
:1080A0000F6A93ED0E6A07EE902A0A7E920748BF88
:1080B0009FED0B7AF8EE677A48BF67EE877A86EE17
:1080C000267AB0EEC77AB4EEE77AF1EE10FAACBFDA
:1080D00001200020DFE700BFB86B0020DB0FC940A4
:1080E0000000803B13B5094B01910446D3F84C0BBB
:1080F00003681B69984730B10199204602B0BDE87A
:108100001040FEF775BC02B010BD00BFB86B002078
:1081100010B504467FF034FBD4F8A831C01AD4F867
:10812000A43198424FF0000084BFC4F8A40101209C
:1081300010BD000038B505460C467FF021FBD5F890
:10814000C831C01A23894FF47A725343984294BFBE
:108150000020012038BD0000C368186808B190F8FD
:10816000B808704710B5012104460A4803F0F6FF2D
:1081700028B120460321BDE81040FEF78BBC47F034
:10818000C5FABDE8104040F26B124FF4801147F081
:1081900075BA00BFE87E002090F89031022B04D021
:1081A000032B04D1034803F0A9BF0120704700202E
:1081B000704700BFE87E002038B50C4BD3F8885CD0
:1081C00090F89031032B044605F004050AD10848C5
:1081D00003F0ACFF94F8903135B110B9023B58422E
:1081E000584138BD0020F5E70120FAE7B84B0020E0
:1081F000E87E002010B50F4A137843F08003137017
:108200000D4B93F99020002A044609DBFEF73EFD52
:1082100070B920460822BDE810400921FDF74ABD8B
:10822000BDE8104001220E21A3F50370F5F7CCBE86
:1082300010BD00BFC4820020B85B0020F8B5D0F8A4
:10824000B44105465CB1012C1AD047F05FFA40F604
:1082500043024FF4801147F011FA012407E0184B54
:10826000D3F84C0B03681B69984710B900242046CB
:10827000F8BD2846FEF744FE0123C5F8B431F6E701
:10828000104F97F99030002BF0DA436A1B6893F88F
:10829000A160012EEAD13C3026F04CFC04460028B7
:1082A000E5D1D7F8C03093F8CB3033B132460D2149
:1082B000A7F50370F5F788FED9E73446D7E700BF86
:1082C000B86B0020B85B002038B5674BD3F89C2012
:1082D000664B9A4204460D4601D0002096E04B883A
:1082E0005D2B75D8512B2FD8103B9AB20F2A49D944
:1082F0002046FDF70DFE6B885D4A04214AF0B0FE72
:108300007DE0BC3B0D2BF3D801A252F823F000BF57
:10831000FF830108FF830108F1820108F18201084F
:10832000F1820108F1820108F1820108FF8301084E
:10833000F1820108FF830108F1820108F18201083E
:10834000F1820108FF830108523B0B2BD0D801A218
:1083500052F823F04B840108F182010815840108CA
:1083600029840108F1820108F1820108F1820108E3
:10837000F1820108F1820108F1820108F18201080D
:10838000518401080F2BB3D801A252F823F000BF8B
:1083900023840108DB820108318401083784010845
:1083A000458401082984010815840108F182010827
:1083B000F1820108F1820108F1820108F1820108CD
:1083C000F1820108F1820108F18201083D8401086F
:1083D000732B46D006D8702B40D0722B88D1FFF774
:1083E000EBFD1AE04AF2CF62934234D080D8C92B19
:1083F0000DD8BB2B85D8B23B012B3FF679AF204679
:10840000FDF786FD29884EF059FF012038BDCF2B9E
:10841000F5D06DE72046FFF779FD00283FF45DAF0A
:10842000EDE7FFF7E7FDF8E72046FFF707FFF4E782
:10843000FFF720FEF1E7FFF777FDEEE7BDE83840F4
:10844000FFF788BDFFF78EFDE7E7FFF74BFEE4E798
:10845000FFF75EFEE1E7FFF76DFEDEE7FFF798FD51
:10846000DBE7FFF7BBFDD8E7B85B0020E078002032
:10847000A4540C0890F89031032B0BD0062B06D097
:10848000012B0AD1C368186803681B6818470448A1
:1084900001F00ABA034803F0BBBE0020704700BFDA
:1084A0008C7D0020E87E00208B88012B05D00B6995
:1084B0003BB94B692BB9CB681BB904480021FAF7CB
:1084C00039BA024800220831FAF756BAB82B002010
:1084D00010B54B885D2B04460A464BD8512B05D866
:1084E000103B99B20F291FD9002091E0523B0B2B72
:1084F000FAD801A151F823F04B860108E98401085C
:10850000058601081B860108E9840108E984010841
:10851000E9840108E9840108E9840108E984010883
:10852000E9840108538601080F2BDDD801A151F819
:1085300023F000BF13860108258601082D86010857
:1085400035860108458601081B8601080586010855
:10855000E9840108E9840108E9840108E984010843
:10856000E9840108E9840108E9840108E984010833
:108570003D860108B32B76D016D8732B70D00ED859
:10858000702B6AD0722BAFD1D1ED027A9FED3A7A7F
:1085900067EE877AFDEEE77AC0ED6B7A37E0B22BB3
:1085A000A2D1FFF771FC32E0C92B23D8BB2B9BD99A
:1085B000BC3B0D2B98D801A151F823F00F86010880
:1085C0000F860108E9840108E9840108E9840108AB
:1085D000E9840108E98401086D860108E98401083D
:1085E0006D860108E9840108E9840108E98401082D
:1085F0006D8601084AF2CF6293427FF475AFFFF7B0
:10860000C1FB04E002F108012046FEF765FB0120F2
:1086100010BD1146FFF7C6FAF9E711462046FFF7ED
:1086200027F9F4E71146FFF763F9F0E71146FFF782
:1086300099F9ECE71146FFF7C3F9E8E71146FFF7B0
:10864000CBF9E4E7FFF78EFDE1E71146FFF7F2FA19
:10865000DDE71146FFF75CFBD9E7FFF7B3FBD6E791
:10866000FFF7C4FBD3E7FFF71FFFD0E7034802F192
:108670000801F9F729FECAE70000C842F48000208B
:1086800070470000704700007047000090F8280015
:1086900080F0010070470000024B436040F6050384
:1086A000038170470001020490F8550170470000F3
:1086B0000F2070470020704700207047002070474F
:1086C000002070470048704750550C08004870471C
:1086D0005C550C0810B50A4C04F500532046D3F83D
:1086E000D83CB3F9083000EE103AB8EEC00AF5F7FE
:1086F00005FF04F59E40BDE81040FDF73DBA00BF00
:10870000B82B002030B5154C2DED028B1D4604F51D
:10871000005383B0B3F94C3308EE103A04F58043AC
:10872000CDE90021D3F8400B03689B6E9847B8EE63
:10873000C88AF0EE400ADDE9002104F59E40B0EE63
:10874000480AFCF769FE04F59E40FDF777FA85EDCF
:10875000000A03B0BDEC028B30BD00BFB82B002077
:10876000F8B51C4D05F5005405F580462846D6F8A9
:10877000487BF5F7B1FEB4F9883301EE103AB4F94D
:10878000863300EE903A434200EE103AB8EEC11A3A
:10879000F8EEE00AB8EEC00A384673F015FA28463B
:1087A000D6F8486BF5F798FEB4F9883301EE103A25
:1087B000B4F9863300EE903A434200EE103A304668
:1087C000B8EEC11ABDE8F840F8EEE00AB8EEC00A0B
:1087D00073F074BAB82B002038B5124D124CD5F88E
:1087E000400B03689B689847692100F1940220467A
:1087F00047F06AFCD5F8400B0368DB6898476A21AC
:1088000000F19402204647F05FFCD5F8400B036866
:108810001B6998476B2100F194022046BDE838405F
:1088200047F052BCB86B0020683D0020014806F0BC
:10883000D1BA00BFB82B00203C307DF07BBB0000DC
:1088400008B546F063FFBDE8084072224FF480117E
:1088500046F014BF08B546F059FFBDE8084066224F
:108860004FF4801146F00ABF08B546F04FFFBDE84F
:10887000084080224FF4801146F000BF73B51F4DB1
:108880000646D5F89C0003681B6B9847044680B3E6
:1088900095F99130002B2FDBD5F8C03093F8CB4001
:1088A0003CB395F8903003F0A003202B24D1D5F8E9
:1088B0009C0003681B689847052808D0D5F89C00E1
:1088C00003681B689847A0F110035C425C410C4AA6
:1088D00002F624330193A2F500532146D3F8F03D6C
:1088E0000093D2F8483BD2F8402B30467DF0D0FAC6
:1088F0000446204602B070BD0024FAE7B85B0020B1
:10890000B86B00203C30FFF7B9BF000038B5114DFF
:1089100004461148F6F778FA95F99030002B14DAEE
:10892000236A93F8A120012A06D0D5F89C000021E3
:10893000BDE83840FCF78EBE0D21A5F50370F5F7B4
:1089400043FB95F99030002BEFDB2046BDE8384023
:108950007DF0DABDB85B0020B82B00203C30FFF77B
:10896000D5BF0000012070470120704701207047EB
:108970000120704711207047012070470020704788
:10898000002070470020704700487047A0560C0830
:1089900000487047A8560C0838B5436904461D685E
:1089A000806976F04FFD23F01BFFDFED1B0A2846A0
:1089B00072F0F0FE6369A0691D6876F043FD23F054
:1089C0000FFFDFED150A284672F05CFF6369186837
:1089D00074F02CF96369DFED110A18689FED0E1A27
:1089E000B0EE600A73F0F0F86369DFED0C0A186806
:1089F0009FED091AB0EE600A73F060F963691868B8
:108A000073F0F6F918B96369186874F075FB002300
:108A10002364012038BD00BF00803B4400007A433E
:108A200070B52DED028B88B00446FCF7DBFD70B10C
:108A300020460021FCF70EFE63699FED310A18689D
:108A400008B0BDEC028BBDE8704074F031BC636AC5
:108A50000221186877F0AEFC2A4B93F891305B0640
:108A600003D56369186872F015FF9FED258A606968
:108A70008DED018A8DED028A8DED038A8DED048ADC
:108A800003AA01A90068012372F06EFF63691868E8
:108A900074F0E2F9236A1D682B68DE6C636918685C
:108AA00073F0B6FA0122CDED060A8DED071A05A97D
:108AB0008DED050A2846B0EE480AB0476369B0EE6E
:108AC000480A186873F006F96369186874F062FC64
:108AD000236C8BB17EF054FEE36BC01A236C98427A
:108AE0000AD309480C220521FCF7F2FE20B90648FA
:108AF0000C220221FCF7ECFE08B0BDEC028B70BD2D
:108B000000000000B85B0020B82B002038B50446F8
:108B10000D467EF035FEC4E90F0538BD07207047CD
:108B200001207047002070470020704701207047E7
:108B30000048704740570C080048704748570C08D9
:108B400038B52DED028B002380F83C30C368DFED93
:108B5000338A1B684269D3ED0A0A9FED318A93ED8F
:108B6000060AF4EEE80A0446F1EE10FAB8BFF0EE99
:108B7000480A106872F00EFEE36862691B681068AC
:108B8000D3ED0A0A93ED060AF4EEE80AF1EE10FAC4
:108B9000B8BFF0EE480A72F075FE636920461D68A2
:108BA000FDF7BAF96368B3F93820B3F9363000EE4F
:108BB000903A434201EE102A00EE103AB8EEC11A84
:108BC000F8EEE00AB8EEC00A284672F0FDFF6369CD
:108BD00020461D68FDF7A0F96368B3F93820B3F9A2
:108BE000363000EE903A434201EE102A00EE103A81
:108BF000B8EEC11AF8EEE00AB8EEC00A284673F0E3
:108C00005DF8084BD3F8540B74F0E0FE06480821D9
:108C1000F9F792FABDEC028B012038BD0000003458
:108C200000007A43B86B0020F480002030B52DEDB1
:108C3000048BC3689FED898A1B684269D3ED0A7A69
:108C4000DFED870A93ED060AF4EEC87AF1EE10FA2A
:108C50000446A8BFF0EE670A106889B072F09AFD6A
:108C6000636920461D68FDF757F96368B3F938203A
:108C7000B3F9363000EE903A434200EE103A01EE7E
:108C8000102A2846774DB8EEC11AF8EEE00AB8EE81
:108C9000C00A72F099FFD5F8540B74F0D9FFA5F50E
:108CA000805393F8B530D90747D4D5F8543B1A8B85
:108CB000D20742D593ED0A9AB4EEC89AF1EE10FAB3
:108CC000B8BF93ED049AE36A186852F043FCD5F8F4
:108CD0004C3BD3ED067AA36B20EE270AD3ED007A46
:108CE000F0EE498AE0EE278AB0EE490AF5EEC08A36
:108CF000F1EE10FAD8BFDFED5C8AF0EE680A1FF0E3
:108D00005FFE28B9D5F8540BB0EE680A74F01EFD6A
:108D1000636893F95130272B0FD0A36A186852F07B
:108D200019FCF0EEC07AF4EEC87AF1EE10FAB0EE6B
:108D3000407A20D5002384F83C30236B1B68B3F9BC
:108D4000083000EE103A2046B8EEC00AFCF7A6FF45
:108D50002046FCF711FF2046B0EE408AFCF742FCAB
:108D6000002848D00021204609B0BDEC048BBDE8A6
:108D70003040FCF76FBCD5F8543B9FED3C0AD3ED77
:108D80000F7AD3ED0B6AA36B27EE800AF4EEC86A64
:108D9000D3ED007AF1EE10FA67EE277A10DB9FED43
:108DA000341ADFED310A552037EE800A1FF00CFF30
:108DB000012384F83C30D5F8540B74F0B7FCBCE7C1
:108DC0009FED2C7AF4EEC76AF1EE10FA05D89FED0C
:108DD000261ADFED290A5920E6E7F0EEE66AF4EEFE
:108DE000C86AF1EE10FAE3D594F83C30002B08BFC6
:108DF000B0EE670ADCE7636A0221186877F0DAFAF6
:108E00001E4805F09FFEB0EE480AD5F8540B74F0EA
:108E100021FE01461A48FBF7FDF86369186874F0F3
:108E2000B9FA236A1D686369186873F0F1F805AC34
:108E3000204614498DED020ACDED030A8DED041A8A
:108E4000F9F738FB079B009394E80C0002A9284629
:108E500070F0AAF909B0BDEC048B30BD00000034FD
:108E600000007A43B86B002000000000E02E65424D
:108E70000000B442000000B40000B4C23459002025
:108E8000B82B0020F480002008B5064BD3F8543BE3
:108E9000D868243022F014FEFCEEC07A17EE900A57
:108EA00008BD00BFB86B0020024BD3F8543BD86814
:108EB00073F058B9B86B00200B2070470120704741
:108EC000002070470120704700207047004870471D
:108ED000E0570C0800487047E8570C08012070471D
:108EE00008B5DFED237AF4EEE70AF1EE10FA2DED86
:108EF000028BF0EE408AB0EE608A35DDDFED1D7A40
:108F0000F4EEE70AF1EE10FA2ED5F6EE007A70EEE6
:108F1000E77ADFED196A9FED190ADFED190AF0EE25
:108F2000E77A87EEA67A8720B7EE001A30EE470A76
:108F30001FF04AFEDFED137A9FED131ADFED130ADF
:108F400020EE270A8A2020EE280A1FF03DFE30EE90
:108F5000080ABDEC028BDFED0A0ABDE808408D204F
:108F6000B7EE001A1FF030BE9FED050AEFE700BF15
:108F7000AC1C5A3ED578493F8FC2753E9A99993FAD
:108F800000000000FAEDEBBA9A99993E9A9999BEC1
:108F900030B52DED048B7D4BB3F94C3300EE903A98
:108FA000F8EEE00A83B0044601AA6946B0EE600A12
:108FB000FCF732FAA06976F045FAE369D0ED008A51
:108FC000D3ED946AD3ED977A90ED016AA3689FED93
:108FD000701ADFED700A27EEE80A68EEA68A03F63B
:108FE0009403E6EE278A05463B20DFED6B7AB0EE70
:108FF000E87AB4EEE77AF1EE10FA58BFB0EE677A8D
:10900000DFED667AC7EE275AF7EE007A77EEE57A5B
:109010009DED007A67EE877A93ED007A67EE877AA6
:109020009FED5F7AA6EE260A87EE879A1FF0CCFDA9
:109030003C209FED571ADFED570AB0EE408AB0EEA4
:10904000680A1FF0C1FD626B564B1268DFED567A5D
:10905000B2F90820D3ED006A9FED541ADFED540AEF
:1090600007EE102AB8EEC77AF0EE408A27EE277A8C
:10907000DFED507AA6EEA77A4520F4EE007AA7EE4F
:10908000678ABAEE000A28EE000A83ED007A8DEDB9
:10909000000A1FF099FDDDED017A9FED477A474BFD
:1090A0008DED000AF0EEE77AF4EEC77AF1EE10FAF1
:1090B00051D593ED007ADFED427A77EE277AB2EE62
:1090C000007AF4EEC77AF1EE10FA58BFF0EE477A64
:1090D000C3ED007A67EEA87ACDED017A636A18686D
:1090E00090F8CB10002939D177F064F9636A1B68D6
:1090F00093F8A110012939D0032940D039B9236A46
:10910000186870F039FD236A18686FF085FF236ACC
:10911000DDED010A18689DED000A0368B0EE491AFA
:10912000DB6A9847204695ED028AFCF771FB2046E2
:10913000F0EE400AB0EE480AFFF7D2FE236A6268FA
:109140001868D2ED020A036801215B6E984703B0EC
:10915000BDEC048B30BD00221A60BFE7194B93F9B8
:109160009130002BB4BF01210221BDE7236A1868AA
:1091700070F002FD236A18686FF064FFC7E7D979C1
:109180000029C4D12046FCF7BDFEC0E7B84B002043
:1091900000000C4400000CC40000FA4400409C4550
:1091A00000003442448100200AD7233D00A08C45B2
:1091B00000A08CC58FC2753F00000034488100209C
:1091C0008FC2F53CB85B00200E207047002070472E
:1091D0000020704700207047002070470020704733
:1091E0000048704780580C080048704780580C08A9
:1091F00070B52DED028B436A1B6893F8CB300446A3
:10920000FBB9052384F848302046FCF701FB636A6C
:1092100002211868B0EE408A77F0CCF894F950300B
:10922000E2696BB3D2F8F8515D4394F84820052AFF
:109230004FD8DFE812F02B005F008400B100DF00A0
:109240001E01836A1B68B3F90830002BB8BF5B426C
:109250009BB2B3F57A6FD4D2C36A1B68B3F90830F6
:10926000002BB8BF5B429BB2B3F57A6FC9D27EF0D8
:1092700087FAE36CC01A40F6C4139842C1D8C3E71A
:1092800094F95150D2F8FC215543CEE7226A94F963
:10929000511010689FED801A49F6404253435143E4
:1092A00000EE103A00EE901A0268F8EEE00A926BB7
:1092B000B8EEC00A9047DFED797A41F293139D42F0
:1092C00038EE278A05DD94F950308BB1012384F8FC
:1092D0004830236A62681868D2ED020A0368B0EE6B
:1092E000480ABDEC028B5B6EBDE870400021184758
:1092F0000223ECE7226A9FED681A106849F64042A3
:10930000534300EE103A0268B8EEC00A926BF0EEDA
:10931000410A9047DFED627A38EE678A05F50C5511
:10932000B5EEC08AF1EE10FA05F1270543F2BA4313
:10933000D8BF9FED598A9D42CBD80423C7E7236A43
:109340009FED551A186894F9513049F6404253433D
:1093500000EE903A0268F8EEE00A926BB0EE410A35
:109360009047DFED4F7AE36938EE678AD3F8F8313A
:10937000B5EEC08AF1EE10FAD8BF9FED478A002BF8
:10938000B8BF5B4242F228329342A2DD41F294130D
:109390009D429EDD03239AE7236A9FED3F1A1868DA
:1093A00094F9513049F64042534300EE903A026836
:1093B000F8EEE00A926BB0EE410A9047DFED387AA2
:1093C000E36938EE678AD3F8F831B5EEC08A03F561
:1093D0000C53F1EE10FA03F1270344F24E62D8BFAA
:1093E0009FED2D8A93423FF674AF2E4B9D42FFF6C0
:1093F00070AFA2E7236A94ED111A1868D4ED100A31
:10940000036894ED0F0A1B6B00219847DFED237A68
:1094100094F95020E36938EE278A1AB393ED7E7AE7
:10942000D4ED0F7AB8EEC77A77EEC77A9FED1E7A41
:10943000F0EEE77AF4EEC77AF1EE10FA3FF649AFB4
:109440000D2294F849101948FCF742FA024618B95F
:1094500001461648FCF73CFA47F006FE162147F095
:109460003FFD36E793ED7F7AD4ED107AB8EEC77AF8
:10947000DAE70D2294F849100C48FCF729FA024665
:1094800018B901460948FCF723FA47F0EDFD02221E
:109490000D2147F045FD1CE700000000CDCC4C3EFF
:1094A0008FC2753E6DEEFFFF0000FA43B82B00201F
:1094B00073B5474D0446D5F89C0003685B6B98472D
:1094C00018B90026304602B070BD95F99130002BD6
:1094D0005FDBA36A1B68B3F90830002BB8BF5B429F
:1094E0009BB2B3F57A6FECD2636A1B6893F8CB60DA
:1094F000002EE6D095F99030002BE2DBD5F89C00E9
:1095000003681B689847002584F8490084F8485090
:109510007EF036F9E36AE064A4F850501B68B3F9B2
:109520000830B3F5967F43DD012384F8513047F0CE
:109530009BFD152147F0D4FC264BB3F94C3301EECB
:10954000103AE369B8EEC11A93ED7E0A8DED011A67
:10955000F1EE410A5320B8EEC00ACDED000A1FF02B
:1095600033FBE36984ED0F0A93ED7F0A9DED011A49
:10957000DDED000AB8EEC00A54201FF025FBE369B8
:1095800084ED100AD3ED807AF8EEE77AC4ED117A13
:1095900098E7D5F89C0003681B689847012890D08D
:1095A000D5F89C0003681B689847002891D188E78C
:1095B00013F5967F01DAFF23B7E7A36A1B68B3F9B7
:1095C0000830002BACBF0123FF2384F85030AEE7F6
:1095D000B85B0020B84B0020042070470120704782
:1095E00000207047012070470048704718590C0848
:1095F0000048704720590C08012909D0232907D0B9
:10960000042905D0034BD3F88C0C00F001007047FF
:1096100001207047B84B0020C36B23B990F841007C
:1096200080F001007047002070470000034BD3F822
:109630008C0C80F00400C0F380007047B84B002011
:10964000012380F84230184670470000002380F85C
:10965000423001207047000070B52DED028BC368C9
:109660000446186890F9BB3886B0B0EE408A0BB358
:1096700090F8BC68F6B174F07BFB01281AD127483A
:1096800019213FF0BBFB07EE900AF8EEE77AF4EE03
:10969000C87AF1EE10FA0DDD214BB3F9EE3C07EE7E
:1096A000903AF8EEE77AF4EEC87AF1EE10FA18DBA9
:1096B000002012E01B4B0FCBFDEEC87A02AD85E80F
:1096C0000F0017EE901A012228460DF067FF01AA3D
:1096D000022128460DF098FFE8B906B0BDEC028BD8
:1096E00070BDBDEEC88A8DED018A002529460E4861
:1096F000E563F8F721FD6369186873F0FDFCDDEDA3
:10970000017A0A48B8EEE70A314606F0D7F984F83C
:1097100041500120E1E70026E7E700BFB83A00200A
:10972000B84B0020CC760020F4800020E48100209B
:1097300010B52DED048BC2689FED149A1268436931
:10974000D2ED0A0ADFED128AF4EEC90AF1EE10FA40
:109750000446B8BFF0EE680A1868B0EE408A72F0AE
:1097600019F8E268636912681868D2ED0A0AF4EE23
:10977000C90AF1EE10FAB8BFF0EE680AB0EE480A76
:1097800072F080F8BDEC048B012010BD00000034A5
:1097900000007A4313B5C36842691B68F0EE400AC3
:1097A00093ED080A93ED0C1ACDED010A0446B0EED4
:1097B000C00A106872F008FAE36862691B681068F2
:1097C00093ED080A93ED0C1ADDED010AB0EEC00A24
:1097D00072F074FA012002B010BD000010B52DED3A
:1097E000028BC36842691B68044693ED0C1AD3EDE3
:1097F000070A1068B0EE408A72F0E6F9E368626921
:109800001B68106893ED0C1AD3ED070AB0EE480AF6
:1098100072F054FABDEC028B012010BD1FB5C36B72
:10982000022B0BD0032B1DD0012B22D1C36818684B
:109830000368DB6805B05DF804EB1847806975F0D4
:10984000FBFD0D4B59689A6802911B68019301A9B1
:10985000039220F0EFF9FDEEC07A17EE900A05B002
:109860005DF804FB4369186805B05DF804EB72F01D
:1098700079BC0020F3E700BF80810020C36B012B7F
:109880000AD003DC2BB19FED070A7047023B032B84
:10989000F9D84369186802E0C3681B68186972F058
:1098A000E9BC00BF0000000030B5C26B012A89B0DE
:1098B0000C4604D0022A0AD0002009B030BDC3688B
:1098C000186803681B6809B0BDE8304018470B4BA7
:1098D000586899681B680193094B02901B780391A3
:1098E000002B04AD18BF032201A928460EF05CF935
:1098F00095E80F0084E80F000120DEE7808100205A
:10990000C48100207FB5C36B022B0FD0032B23D063
:10991000012B25D1C368186803689B689847BCEE83
:10992000C00A10EE100A07B05DF804FB806975F0FC
:1099300083FD0D4B014658689A6804901B68039399
:1099400003A8059221F0EEFF01A88DED010ACDEDEF
:10995000020A22F0B5F8E2E7436918682430F8E714
:109960009FED020ADDE700BF8081002000000000BB
:1099700010B52DED028B01239FED1C8AC363C368D4
:10998000044684B018688DED018AF0EE480AB0EE06
:10999000481AF0EE481AB0EE480A8DED028A8DEDB5
:1099A000038A74F07DFFE3688DED018A8DED028AF4
:1099B0008DED038A186801A974F0A4FAE3681868A9
:1099C000036800225B6801A9984730B945F09EFE04
:1099D000BB224FF4801145F051FE05480021F8F7F5
:1099E000CBFB04B0BDEC028B10BD00BF000000003B
:1099F000F480002030B589B00446FBF7F3FD70B168
:109A00001D4805F04DFD014618B1636A1B6893F8C7
:109A1000CC10204609B0BDE83040FBF71BBE636A9E
:109A20000221186876F0C6FCE368186803685B6971
:109A3000984701461048FAF7EDFA6369186873F021
:109A4000A9FC236A1D686369186872F0E1FA05AC25
:109A500020460A498DED020ACDED030A8DED041A68
:109A6000F8F728FD079B009394E80C0002A928460C
:109A70006FF09AFB09B030BDB82B0020F4800020B5
:109A800010B52DED028BC368DFED298A1B68426992
:109A9000D3ED0A0A9FED278A93ED060AF4EEE80A51
:109AA0000446F1EE10FAB8BFF0EE480A106871F003
:109AB00071FEE36862691B681068D3ED0A0A93EDD2
:109AC000060AF4EEE80AF1EE10FAB8BFF0EE480A22
:109AD00071F0D8FEE36862691B68106893ED080AAC
:109AE00093ED0C1AD3ED070AB0EEC00A72F06CF8D1
:109AF000E36862691B68106893ED080A93ED0C1A1D
:109B0000D3ED070AB0EEC00A72F0D8F8636918689E
:109B100073F0F2FA6369186873F088F80648002158
:109B2000F8F72AFB054B00221A70BDEC028B10BD22
:109B30000000003400007A43F4800020C48100203B
:109B40000223C363FFF79CBF0523C363FFF798BFDE
:109B50000423C363FFF794BF10B50446FFF7F8FF73
:109B6000074A0023936053601360064A9360536072
:109B70001360002384F8403084F84230012010BD87
:109B80008C810020988100200323C363FFF778BFF6
:109B900030B50623C363C36842691B6893ED080AA6
:109BA00093ED0C1AD3ED070A044685B01068B0EEA9
:109BB000C00A72F009F8E36862691B68106893EDE7
:109BC000080A93ED0C1AD3ED070AB0EEC00A72F042
:109BD00075F86369186872F00BF918B96369186849
:109BE00073F08AFA7DF0CCFD0C4D0346284601A99E
:109BF00040F8043B236A1B6800245B6F03930194C5
:109C0000029421F0D5FA0023EC61AC616C616C62C6
:109C10002C6285F82C3005B030BD00BF508100208B
:109C2000024BD3F88C0CC0F3C0007047B84B002037
:109C30002DE9F0432DED028B9946C36B274C062B83
:109C400085B080460E461746B0EE408A36D0FFF704
:109C50009FFF96E80F00224D85E80F0097E8070068
:109C6000103585E8070084F82D900023B9F1000F26
:109C700030D084ED0A8A63627DF082FD03AB206000
:109C800002AA01A9304621F0C5FB94ED092ADFEDB7
:109C9000157AD4ED0A1A9DED031ADDED020A9DED49
:109CA000010AD8F83C10104822EE272A3A46F7F766
:109CB000DDF905B0BDEC028BBDE8F083B9F1000F12
:109CC000C7D194F82D30002BC3D04369186873F0C6
:109CD00013FABEE7A36284ED098ACDE75081002024
:109CE000548100200AD7233CB82B002038B50B4DF7
:109CF0000446284605F042FD2B786BB194F84130BC
:109D000053B90123064884F841305AF03FFDBDE8BD
:109D1000384004485EF094BB38BD00BFE4810020A9
:109D2000084E00200878002070B52DED028B88B019
:109D30000446FBF757FC054680B1294805F0B0FB07
:109D4000014618B1636A1B6893F8CC10204608B02E
:109D5000BDEC028BBDE87040FBF77CBC636A9FEDF5
:109D6000218A1868022176F025FB60698DED018A51
:109D70008DED028A8DED038A8DED048A2B4603AAB0
:109D800001A9006871F0F0FD63698DED008A186823
:109D90000368B0EE480A2A4669465B6898476369DB
:109DA000186873F059F86369186873F0F3FA236A56
:109DB0001D682B68DE6C6369186872F029F901224E
:109DC0008DED050ACDED060A8DED071AB0EE480AB5
:109DD00005A92846B04708B0BDEC028B70BD00BF96
:109DE000B82B002000000000A1B1DFED0F7A20EEBB
:109DF000270A33B1DFED0D0A0D4801220021F8F7E3
:109E0000C5B922B160EEA70A0948F8F73DBADFEDFF
:109E1000070AF9E722B10648B0EE600AF8F770BA0F
:109E20000348F8F7A9B900BF0AD7233C0000000097
:109E3000F48000202DE9F0432DED028B8BB0044619
:109E4000164606A802220F461D46B0EE408AF0EEE6
:109E5000608A0DF0A9FE284806A95AF059FE8046EE
:109E600058B947F001F90522162147F059F8404644
:109E70000BB0BDEC028BBDE8F083E36B032B02D08B
:109E80002046FFF781FE9DF858309DF854209DF83C
:109E90005010F0EE680AB0EE480A2046FFF7A4FF23
:109EA0007DF06EFC154BD7F800901860144BD7F876
:109EB00004E0D7F808C0134AC3F80090C3F804E0E0
:109EC000C3F808C00023137096E807000E4F0F4E2A
:109ED000CDF80C9087E8070095E8070086E80700B2
:109EE000CDE90076E16B0A48CDF810E003AACDF881
:109EF00014C0F7F777F8BAE7084E00204C8100202D
:109F000080810020C48100208C8100209881002065
:109F1000B82B002010B588B000240594069407944F
:109F20009DF82C4002949DF82840CDE9003405AB03
:109F3000FFF780FF08B010BD2DE9F04F2DED028B2B
:109F40008FB091469DF86C709DF868B0002F14BFDB
:109F50000322022204460AA80D46B0EE408A9A4621
:109F6000F0EE608A0DF020FE4D480AA95AF0D0FDAF
:109F7000064658B947F078F80522162146F0D0FF7A
:109F800030460FB0BDEC028BBDE8F08F454AE36B65
:109F9000D2F88C2C12F0400F0DF11C082AD0012BA6
:109FA00002D02046FFF7E4FC5B46F0EE680A52461A
:109FB000B0EE480A49462046FFF716FFE3681868E6
:109FC00003683A465B682946984700230493059343
:109FD000069307930893099304AB0093CDF804808C
:109FE0003B462A46E16B3048F6F7FCFF012384F834
:109FF0004030C5E7022B02D02046FFF7A1FD002F1D
:10A0000049D0E3684146186874F058F840B92268AE
:10A0100003905268012120469047039B1E46AFE7FC
:10A02000224B1B782BB963699DED070A186871F004
:10A0300093FF52464946DFF874A0DFF884905B46F0
:10A04000F0EE680AB0EE480A2046FFF7CDFE296818
:10A050006A68AB68164D8AF80070164F29606A600E
:10A06000AB600023BB607B603B60C9F80830C9F877
:10A070000430C9F800307DF083FB0F4B6A68296813
:10A080001860AB680892CDE90079099307919AF8B6
:10A0900000304246A6E763699FED080AC6E700BFA5
:10A0A000084E0020B84B0020B82B0020C4810020AF
:10A0B000808100208C8100204C8100200000000065
:10A0C000988100202DE9F0472DED028B8EB00446DB
:10A0D0006F489DF860A00E469046B0EE408A9946C3
:10A0E000F0EE608A5AF014FD054658B946F0BCFF00
:10A0F0000522162146F014FF28460EB0BDEC028B57
:10A10000BDE8F087634BD3F88C3C590648D5E36B28
:10A11000012B02D02046FFF72BFCE368314618687C
:10A1200074F0E6FA054618B946F09EFF0222E0E711
:10A1300053464A46F0EE680AB0EE480A41462046C9
:10A14000FFF752FED6ED027AE16B0391F8EEE76A73
:10A15000D6ED037ACDED056AB8EEE77AD6ED017A51
:10A160008DED067AF8EEE77A3046CDED077A0DF000
:10A170003FFA00220BAB089209920A920B920C92C2
:10A180000D920193C21E08AB0093039953425341B1
:10A1900005AA4148F6F726FF012384F84030ABE7D3
:10A1A0000027E068089709970A97006805AB08AA96
:10A1B000314674F05DFA054600289DD0E36B022B12
:10A1C00002D02046FFF7BCFC5346F0EE680A4A4630
:10A1D000B0EE480A41462046FFF706FE9DF81430CF
:10A1E000002B50D0E3680BA9186873F067FF804616
:10A1F00030B9236801215B682046984745467BE7D4
:10A20000264B1B782BB963699DED0B0A186871F01A
:10A21000A3FE234B089A1A60099ADFF89080DFF8B2
:10A2200090905A60DFF874A00A9A9A609DF81430F2
:10A230008AF80030C8F80870C8F80470C8F80070D0
:10A24000C9F80870C9F80470C9F800707DF098FA70
:10A25000D6ED027A134BE16B1860F8EEE76AD6EDA3
:10A26000037ACDED0B6AB8EEE77AD6ED017A8DED83
:10A270000C7ACDE90089F8EEE77A9AF80030CDED56
:10A280000D7A0BAA85E763699FED070ABEE700BF59
:10A29000084E0020B84B0020B82B0020C4810020BD
:10A2A000808100204C810020000000008C81002073
:10A2B000988100202DE9F0470E4611461A46C36BDF
:10A2C0008AB0052B9DF84C9005460DD0CDED050AC2
:10A2D00004928DED030A0291FFF736FCDDED050ACD
:10A2E000049A9DED030A0299184C194F9DF84830C5
:10A2F000DFF868A0DFF868802846FFF775FD0023C7
:10A300000022A36063602360BB607B603B608AF8CF
:10A31000002096E8070088E807007DF031FA0D4B31
:10A320001860B9F1000F0ED06268A3682168079128
:10A3300008920993CDE900789AF80030E96B064855
:10A3400007AAF6F74FFE0AB0BDE8F087808100202B
:10A350008C8100204C810020B82B0020C48100207B
:10A36000988100202DE9F0470F461946C36B8AB04B
:10A37000042B9DF85090054616460BD0CDED050AEE
:10A380008DED040A0391FFF7E3FBDDED050A9DED7A
:10A39000040A03991A4C9DF84C309DF84820DFF8C8
:10A3A00070A0DFF870802846FFF71EFD0023A36031
:10A3B0006360236000238AF8003097E8070088E88C
:10A3C000070096E807000F4F87E807007DF0D8F9EF
:10A3D0000D4B1860B9F1000F0ED06268A3682168B8
:10A3E000079108920993CDE900879AF80030E96B4C
:10A3F000064807AAF6F7F6FD0AB0BDE8F08700BFE9
:10A4000080810020988100204C810020B82B002002
